:020000040000fa
:080000000001040000000000f3
:020000040000fa
:100200006f5f22000e7f22000e01880000000000b8
:100210000c000700a086210011002000110007003b
:10022000000020000000e000020032000000020098
:10023000000000005c010200010000000040da0044
:100240000000fe004440a90000f820000000e0008b
:100250000300320000002000a00188004440a800f4
:100260000000060091018800800078000000eb008b
:1002700015003700e280400032a0b4009101ba00be
:10028000e280400032a0b4009102ba00e280400057
:1002900032a0b4000002eb00472bde00f507b200ed
:1002a000602ce10004003a000059eb008301e900f2
:1002b000fdff3e00040037006128e100010032002c
:1002c0000082eb00040007001101ba000200e00008
:1002d000e8ff3a00000006003159ba008301e90046
:1002e0000c0032002159ba008301e90008003200f5
:1002f0000400e00003003a00e280400032a0b400b5
:10030000f5ff370011d9ba008301e900faff3a007e
:100310008100e800e180400032a0b4000000060047
:10032000480f0400010000005a4f040001000000c3
:10033000c00e040001000000404d04000100000058
:100340004a0c040001000000fc430400010000000e
:10035000e4440400010000001e5c040001000000f1
:100360000040da000000fe0003f0a200889fbe00fb
:100370008a9fbe008c1f7800dc010700e301330078
:100380006450e1004f0032006420e100520032006e
:1003900003826c0007003b000905d0000306d00073
:1003a000820f54000c065d0002003900020032008a
:1003b00089017800030678008582550004003d001d
:1003c0000003fd008103fd008502ea008b854200e9
:1003d000840f720002003b0060001000e0801800f3
:1003e0006011b8000005eb007a28e1000a0039002e
:1003f00006007800c75ddd00f707b2008780750052
:100400002d003700828171000a01780061056000cb
:100410008180d1000080d3008502e900f9ff3b0014
:10042000060440008784480002003b00600414007a
:10043000e0841c000988a300070032008a81710053
:1004400082817100610164008904d1000884d300b5
:100450008b05e800170037000978a30013003a0065
:100460000b00e000130034008b05e9000804440091
:1004700089844c000a4474000978a3000d003a00f6
:100480000b00e000070034008b05e900080444007d
:1004900089844c0001003a000b0020000978a30079
:1004a000f7ff32000001eb0002003700828171008b
:1004b0000a017800520107000cf0a70001f0a0002b
:1004c0009b0137006420e10002003a00838f6c003a
:1004d0009b0133000801be000200be0094013700fa
:1004e000889fbe008a9fbe008c1f78007f01070096
:1004f0001002200002003b001063880083013700d7
:100500008a0062006408e10002003a00106388007b
:100510008b0137006108e100fcff32000800be00db
:10052000030478007000070001f0a1000900070033
:1005300008f0a600040037000001be00910424006a
:10054000b0fd200088ff070009f0a70001f0a2001d
:1005500077013700889fbe008a9fbe008c9fbe0037
:100560000004be004c0107000800be0089067800a8
:100570006420e10008003900040032000160a0009e
:1005800012022000126388005300370091fc230000
:10059000b0fd20004e0037000006eb0009f0a1007e
:1005a00003f82300020020000800be009f0007009f
:1005b0000600340001f82300000020000801be00fe
:1005c000490007000004be002c0020000800be0007
:1005d00093e82300320a230094000700120034003d
:1005e0000801be00d1fd2300703d2b005fff070016
:1005f0000005be00b3f32300f27a26000800be0017
:100600005201070003f823000200200056ff0700f4
:100610000801be0055ff07000a01be0032000700b6
:100620000004be000c06e8000800be0001f0a100b6
:1006300002002000039823007c0007000800be0091
:10064000160035000801be00400107000005be008d
:1006500032cd2c0043fb230044ff0700809fbe00e7
:100660001269280003d52b000a00be0037010700dd
:10067000620f210013ef2b003cff07000a01be00b0
:10068000320107004f01be00170007000801be003d
:100690002e0107000801be0034ff07000c00e00037
:1006a0000b0032000c10a70001f0a200b2fd2000e8
:1006b00093fc23006260e1000400320022a92000c4
:1006c00063f023000c10a70063f8230027ff070046
:1006d0000df0a70001f0a2004f06be004f05be00be
:1006e0004f04be0000000600889fbe008a9fbe0027
:1006f0008c1f7800fd0007000401330003866c00a6
:100700006450e1002e0032006420e100330032002a
:100710006150e1002f0032006120e1003100320021
:1007200085855500eb07b000090020000804200073
:10073000050037000804440089844c000a00310099
:100740000603430087834b000001530081815b0057
:10075000f8ff33000203be000800a00008044400b4
:1007600089844c00f6ff3900c639dd00830173002f
:1007700001003200130020008904d1000884d30056
:100780000998a300050032000800a7000300a0009c
:100790008904d1000884d3008b05e8008904d100c6
:1007a0000884d3000001eb000281d200940007000e
:1007b00001f0a1000cf0a70001f0a000dc00370060
:1007c0006420e100de0032000801be000200be002d
:1007d000f7ff37006120e100d90032006000b80067
:1007e000f3ff37000000200001f82700f0ff37007a
:1007f000839f68000100e00002003d0060001000df
:10080000e08018000300e00002003d0060011100dc
:10081000e0811900360107004f00e00002003b00b4
:1008200060001000e08018000000060014002000a6
:1008300066013700f4ff2f00640137000001be009d
:10084000950007000470a70003f0a1006509b1003e
:10085000160032000d0035006828e1000600350062
:10086000f0ff2f00f1ff27000300e00013003b0022
:1008700001002800000005000000400081804800c1
:100880008502e900fcff3a0008003700f88f4200bb
:1008900002003c008000eb00000005008100d10058
:1008a0000080d3008502e800fcff3a000300e0006e
:1008b00002003b0060001000e0801800000006000d
:1008c0000001be00740007000470a70003f0a1003f
:1008d00003f8a30013003a006509b10010003200cc
:1008e000090035006928e1000200350001002800f8
:1008f0000000050000004000818048008502e900fa
:10090000fcff3a0000000600f88f420005003500a9
:100910008100d1000080d3008502e800fcff3a008e
:10092000000006008000eb0000000500889fbe006c
:100930008a9fbe00010578000100e0000400350038
:1009400008003c000000e0002000320005003700f5
:1009500060001000e080180002003b0001f02c0055
:100960001a0037000004be006011b8006b092000b7
:100970000982cf00020039000882cf000441b00094
:10098000694252000e00320008003b008281710073
:10099000610164008904d1000884d3008b05e8005c
:1009a0000442e800f9ff3a0005003700080444005b
:1009b00089844c008b05e9000442e900fbff3a0002
:1009c0000f0007000af0a70001f0a0004f05be00cd
:1009d0004f04be00000006000001eb00d400070039
:1009e000040032000200200003f8230001f0a700f9
:1009f0005dfe07000000060004002000f300370041
:100a000081002000618055000b003d000b0020009c
:100a100061fe2f000100e1001d00340082817100a1
:100a2000610164008904d1000884d3000000e8005b
:100a3000faff3a00710020006100640003007000ba
:100a4000020060000900320061044400e0844c00b0
:100a50000988a500050032008b05e8006808e10060
:100a600002003a008904d1000884d300f20f20006c
:100a70000258e10005003d00c75ddd00f907b20046
:100a80008980750008007800000006000bf8270038
:100a90008b00780000000500c70ade00f107b200f5
:100aa000f50fb20008003200e1cf42000200320030
:100ab0000170a00024000500810f700001003200c9
:100ac0000408050044000500810f700002003a0090
:100ad000140005008502e9000000400081c04800c4
:100ae000fcff3b000170a000240005000004be00d4
:100af000e9ff07000003be000405be000200be00bf
:100b0000e5ff0700844f7500000006000200be00ec
:100b10006450e100050036006420e1000200360068
:100b20000968a30001003a000800be000160a000af
:100b30004f0678004f05be004f04be0000000600bf
:100b4000f0ff2f00f1ff2700f9ff3700889fbe005c
:100b50008a9fbe008c1f7800e4ff0700ebff330084
:100b600003866c006450e100240032006420e10040
:100b7000270032006150e100220032006120e100d4
:100b8000210032008b854200eb07b1000134b80030
:100b9000003ab8000804420089844a00013ab800cb
:100ba0000030b8008880400009014a00040033008a
:100bb0000000400081804800020149008b05e900e7
:100bc000c909dd008301700001003200130020001c
:100bd000c814de004814dd004709de001200b20030
:100be000c808de000884700085ff070001f0a1003e
:100bf0000cf0a70001f0a000cdff37006120e1005c
:100c0000cfff32000801be000200be00f7ff370030
:100c10006150e100fcff3a00c9ff3700889fbe0029
:100c20008a9fbe008c1f78000004be009aff070058
:100c30000478a30026003a006120e100250032007c
:100c400009f8a30025003a006420e10021003200e9
:100c5000f507b1000508a3000200320000004000c3
:100c6000818048006044b80003102000020020008a
:100c700000004000818048000805440089854c0040
:100c80000a0541008b8549000a0550008b855800f4
:100c9000030033000a00be00020474008384740061
:100ca0008301d1000281d300830f7100f0ff3a006d
:100cb0008904d1000884d3006001490082017800d2
:100cc000c1adde00fb07b0004dff070098ff370005
:100cd0000960a0000800be0095ff37001202200046
:100ce00012638800f0ff2f00f1ff270090ff37000c
:100cf0006022b800060220000000d0008180d200ef
:100d00000482d2008582d2000000a00002025200bc
:100d100083825a00030031000202420083824a00ab
:100d20000000a1000603e900f3ff3a0000000600fe
:100d3000889fbe008a9fbe000003be0056ff0700ca
:100d40008505780082815200020020006220e100c7
:100d500004003a00f307b100040035007718e10001
:100d6000040035000600be00140037006000b80023
:100d70000f003700f50f2000faff2f008502d10089
:100d80000a85d3008301e900fcff3b0081846200f7
:100d900000046500890f7400f2ff32008582ea00ca
:100da0000a85ea00818462000004650014ff0700e0
:100db00007f0a70001f0a0000081eb000200e000b6
:100dc0004f05be004f04be0000000600889fbe0015
:100dd0008a9fbe00841f780044ff07004f00780000
:100de00011003300f0ff2f00838f6c0006003b00e2
:100df000040565000a00a7000800370009f0a600f6
:100e00001000200008003700820f5400838f5c0020
:100e1000030039001000200001003e000000200007
:100e200009f0a7000000ea004f05be004f04be0015
:100e30000000e00000000600800078001106b1000c
:100e4000030035009101b10001003c000050a100f9
:100e5000000006000001780000c2b3000100370066
:100e60000201e8009240780080cf5000fcff320081
:100e7000e9cf5000faff3200d0c2b30080cf50005b
:100e800003003a000201e80014c0b3000500370077
:100e90000042eb00b0c2b30080cf500001003a0026
:100ea0000201e8008000eb0005fd2f000400370080
:100eb0006a08b90000804100850040000201e80096
:100ec0009201fb0005804100e90f5000f8ff360059
:100ed0000404e000010032008100ea000100780013
:100ee00000000600000478000900070008007800f0
:100ef000cd0a07008001eb00020037008171780005
:100f00008301e800828f5100fcff3a0000000600d8
:100f1000881f7800402b81000000e00001003200b3
:100f200000000100084722000800780012090700ad
:100f30006c04440040492200800f5400faff3a003c
:100f40004f04780000000600800078003004e000c4
:100f5000feff3a00010050000000e900000006001a
:100f60000c00fa00a0bf9f00c0bf9f00f6ff070063
:100f7000b0bf9f00f0bf9f00100c2000d0bf9f00ab
:100f800074815700efb097006c8057002e00070067
:100f90000080fa0000000600889fbe000004780070
:100fa0008144780000fd2f0000004400e90f50004c
:100fb00002003e00000178000d00370008007800b4
:100fc000e00807000000e00003003200080078009d
:100fd000e20807000004780008007800c70807004e
:100fe0000000e0000700320090fa2f0000014400ea
:100ff0000980fb00800f510002003d000280fb00d1
:1010000001003700f00f20004f04be000000060072
:10101000881f7800502b81000f090700000478001a
:10102000c00807000000e000faff3a00e10f4400aa
:1010300003003200512b810008007800840907006a
:101040004f04780000000600ec874700889fbe0030
:101050008a9fbe008c9fbe008e1f780081bf9f00bc
:1010600002077800502b89008046eb00040137000e
:101070008884fb0009007800aa0807008000780037
:101080000000e00002003200e1ff0700fc00370032
:1010900050c2b300804f5400f0003a000fbd9700db
:1010a00020c0b300c0ef9f00d1ef9f0081ef9f00f1
:1010b0000300370040c0b300c0ef9f000fbd970092
:1010c0000fb99700b240780082bf9f008184fb0077
:1010d00090c6b30080cf50003500320017003e00ac
:1010e0006640500080cf5000620032000c003e008d
:1010f0007740500080cf50002800320006003e00ac
:101100000104e0009b003200a0c2b30080cf500079
:101110006e003a001d00370080c5b300160037008e
:1011200040c6b30080cf5000210032006440400030
:1011300080cf500065003a001200370030c7b3007e
:1011400080cf50001e00320007003e006740500074
:1011500080cf5000110032006340400080cf50002b
:101160005a003a001400370050c7b30080cf500037
:101170000f0032006340400080cf500053003a001f
:101180006500370020c0b300cbff3700dfe89700d1
:101190008140e800d1ef9f00c8ff37004fe997007a
:1011a00080c0b300e24f5100c3ff3a00c1ff3700d7
:1011b000acc0b300590037008cc0b30057003700f3
:1011c00093ff0700dfe897000104e00002003a0007
:1011d0004e017800d2b79f00502b81009e08070077
:1011e00000047800e10f4000a20032008fec97006d
:1011f000120037000a85e8008abf9f0016003700fa
:101200008fb897001100fb00800f5400f9ff3200e7
:101210005fe997000204e00003003a005fb0970026
:1012200008587800d0b79f008944e9000a003200ce
:10123000502b810088080700000478000800e800af
:10124000e10f500004003600080078003508070060
:101250000000e000eaff3200dfe897000104e00050
:1012600087003a008d46e8005fb197000149780099
:10127000830037005fe897000004e00003003a00b5
:101280008d46e800ce007800d1b79f00502b81003a
:1012900071080700e10f4000760032005fe9970017
:1012a0000204e00003003a00dfb0970080587800a5
:1012b000d1b79f000fe997000241e90082ef9f003c
:1012c0004240a9006e003400f0ff37000180fb00af
:1012d00008fd2f0008004000e90f50005f003e00ad
:1012e0000a007800dbfe070080ef9f00880078008e
:1012f000030037000fb897000000e80080bf9f0090
:101300000fb997001200fb0001004000e90f5000e8
:10131000f8ff360069ff37000cc1b3003cff07003f
:10132000502b81004c080700000578000040eb00be
:10133000e0ef9f00d0022000800f550005003a002a
:10134000502b8100440807000005780011c0b3004d
:10135000e1ef9f008c4078000a0078000eff070044
:10136000e14f40000a003a00512b81000a0078004a
:10137000b70807000d04e0004b003a00502b810035
:10138000300090000048a3004300320048003700be
:101390008fed97006044b8000c81fb000300200033
:1013a0000800be00a60c07000004be008c407800b8
:1013b0000a007800f8fe07000080fb000100200012
:1013c00008044000898448008b45e900070032008a
:1013d000502b810020080700000578008c40780021
:1013e000edfe0700e14f4000ebff3a008c40780033
:1013f0000a007800e8fe0700e14f400003003a00d1
:10140000512b81000a007800910807006fe99700ce
:101410000204e0000200320060041400e0841c00ba
:101420005fe897000004e00015003a008d46e800f0
:10143000cfe89700e4cf500003003a004e00780058
:101440000888be000e0037000e81e9000207780010
:10145000120078000808780009003700502b81003e
:10146000fd070700808f540005003200e10f4000a7
:101470000b003a000d04e0000d0032000a003700b6
:101480008fb897003144780081bf9f000804e000c6
:10149000f7fe3a00040037000000eb0005003700bb
:1014a000512b81006a0807000d80fb000100370006
:1014b0000080eb004f0778004f06be004f05be00ce
:1014c0004f04be00cf00b100000006000c00fa007f
:1014d000889fbe0000047800cfb09700f0ff27007f
:1014e000d0bf9f008004eb0099bf9f0088bf9f0082
:1014f000a8bf9f00200c2000b0bf9f00788157003c
:10150000708057005f0007000fb897000948780007
:101510000fb8970008045000080078004f04be0080
:101520000080fa0000000600889fbe008a1f780035
:10153000804078000004e00021003d008040ea0087
:10154000d0c6b30080cf5000090034008104fb00f6
:1015500042062000110009008204d8000001780032
:10156000010078004311dd002af621001f0037003a
:101570000100fb0023f6210039003700a200200003
:10158000110009000200d800000178000100780075
:101590004311dd00030141004300dd000300400072
:1015a0003002be002003be0042209000d2209000f6
:1015b000f2219000622190007f0b07002e0037007f
:1015c000d0c6b30080cf5000230034008104fb005c
:1015d00042062000110009008204d80000017800b2
:1015e000010078004311dd002a0122000a014100b8
:1015f000a8002000110009000800d8004300dd0009
:101600000a00400040229000d02290006023900009
:10161000f02390000288900092889000b289900098
:1016200022899000640b0700801f78000102780077
:10163000110009008804d8000102fd004f00780065
:101640000402fb004322dd000a0242005403be00f4
:101650004402be00d8ff37000100fb002301220036
:10166000eacf5000c5ff3c004300dd00030040000e
:101670005001be004000be004f0578004f04be0080
:10168000000006008f03b000889fbe008a9fbe0046
:101690008c9fbe008e1f7800e0b79f00f1b79f00bf
:1016a00082bf9f000000eb00a0b79f00e604370058
:1016b0008001eb0050c2b30080cf5000090032001f
:1016c0000100fb00efb0970097070700e10f400013
:1016d000dd043200afb097008100e800a1b79f00a1
:1016e000d90437007fb1970092407800d0c2b30090
:1016f00080cf50000c00320007003c006d405000cd
:1017000080cf50000d0032006b40400080cf500071
:1017100019003a000e00370000c3b30080cf50001c
:1017200015003a000f0037000330a0007fb2970089
:101730000402e800f4b79f00eaff37000300a000ae
:10174000ffb297008502e800f5b79f00e5ff37007c
:101750000310a0007fb697000c06e800fcb79f00be
:10176000e0ff37000320a0007fb097000000e800f2
:10177000f0b79f00dbff37000318a3000100320021
:101780000300a1000338a300010032000320a100e0
:101790000100fb0002fd2f0002004000e90f500095
:1017a00010003e008000eb00c1b79f0002027800ed
:1017b0004fb197006a10b900ffb297001501fb0006
:1017c0000001410004014100c2b79f005500fb0029
:1017d000f5b79f0004004000e90f50000d003e00e7
:1017e000f3ff37000006eb00ccb79f00a0c2b300a8
:1017f00080cf500007003a000fb89700c000780073
:1018000080bf9f00c1b79f007fb197000201e80031
:10181000f2b79f00e0c2b3007fb29700944f100070
:1018200021003a00830678000de0a0008400e80063
:1018300064405000914f100004003200f1b79f0047
:101840008002eb00b5b79f00100037000fbe970075
:101850004c0078008cbf9f00b0b79f00ffb097008e
:101860008180e800f1b79f00130037003fb2970076
:101870006a20b9000000410003004000b0b79f009b
:10188000ffb297008502e800f5b79f007fb697008a
:101890001c01fb0003fd2f0003004100e90f500075
:1018a000f2ff360004003700830678000dc0a00068
:1018b0000000eb00b0b79f007fb19700b240780006
:1018c000f2b79f00c17f9f00c0c6b30080cf500019
:1018d0002700320014003c006840500080cf5000c8
:1018e0009d00320009003c006c40500080cf500049
:1018f000290032006b40400080cf5000720032005f
:101900000104e000560432008e00370060c6b300c8
:1019100080cf50001c0032006340400080cf500058
:1019200088003a008c00370030c7b30080cf5000e9
:101930001c00320007003c006440500080cf500083
:10194000130032000040e80080cf50007d003a00d4
:101950001100370050c7b30080cf50007d00320027
:101960006340400080cf500076003a000b00370003
:10197000000028000d48a30001003a0000012000eb
:1019800080867600ccff37000da0a00072003700e3
:101990000d60a000700037000d50a0000d70a00079
:1019a0006d0037008fb997004300780083bf9f0018
:1019b000000478000000e00001003a0048442200e2
:1019c0008004eb00010037008104e8008900780002
:1019d000088044001004e000fbff3a003fb297008b
:1019e0000400e00003003200890f520001003100c2
:1019f000840478000007eb00cfb29700898f520073
:101a000001003600098752004368de00e1066000ed
:101a100019003a000d06780009003700efb0970072
:101a200000022000c0060700e10f40000300320062
:101a30002fb097000000e800a0b79f000c06e80058
:101a40008e0f5600f5ff3a000087eb000a003700c2
:101a5000880078003100fb0001047800efb09700a7
:101a6000b1060700e10f400003003200afb097005d
:101a70008100e800a1b79f000900e9008004780018
:101a8000e10f4000f2ff3a000006eb000d00e0001d
:101a90000a003a00ec033700efb097000002200084
:101aa000a1060700e10f4000030032002fb19700ac
:101ab0000201e800a2b79f000c06e8008e0f560056
:101ac000f5ff3a00e00337008fb997004300780034
:101ad00083bf9f00cf80de00010178008201780083
:101ae0000205be000004be000203be000002be00ec
:101af0004822de00482edd0004027600c47f9f00ed
:101b00000d48a3000a0032000404e000080032007f
:101b1000e14f420006003200d1fb2f000180470058
:101b2000044878001840980029002000020037007f
:101b3000d07f9f0019002000d2fb2f0002844700b5
:101b4000a6ff3700c3fb2f000384470019002000c5
:101b5000a2ff37000d0cb300007020000082660069
:101b6000270232000dc8a3000200320064002000ea
:101b7000b4b79f000d48a300050032000fba9700cc
:101b80004401be004400be0084bf9f000400370033
:101b90008fba97004500be0085bf9f007c090700f3
:101ba000e0af9f00f1af9f0082b79f0093b79f0007
:101bb0006022b8006033b8006fa89700ffa89700b4
:101bc0000fb197009fb19700c30807000000e00025
:101bd0000a003d006fa89700ffa897000fb197007b
:101be0009fb1970003f0a200e0af9f00f1af9f000c
:101bf00082b79f0093b79f003d00b3000000eb0049
:101c000080a79f006022b8006033b8006fa89700db
:101c1000ffa897000fb197009fb197001209070026
:101c20000000e000340032006fa89700ffa8970082
:101c30000fb197009fb19700560a070003fc2f00d1
:101c400003814700d90907000fa097000000e900b1
:101c50006300b900a2002000110009000200d800b2
:101c60008000fd0081a79f000100e00002003d0010
:101c70000100e90080a79f000fa497000840ea0038
:101c800029fe07006faa9700ffaa97000fb39700dd
:101c90009fb39700c8090700a0af9f00b1af9f0096
:101ca000c2af9f00d3af9f006022b80006002000a3
:101cb00007ff2300880807000000e00002003d0045
:101cc0000800e9000b0037006022b8000600200081
:101cd000470224002fa89700bfa897004fa997009c
:101ce000dfa99700810807000000e000020035002e
:101cf0000800e80080a79f003fb29700f80f52004d
:101d000057003c00d0c6b300804f52002900360077
:101d10000485fb0042062000110009000285d8005e
:101d200000017800010478004311dd002bf621004a
:101d30000b0141006022b8000600200007fe2300ce
:101d40000288900092889000b289900022899000c9
:101d500099090700a9002000809fbe00110009001a
:101d60000984d800000478004f00be004344dd0021
:101d70000b04440048229000d82290006823900071
:101d8000f82390008c090700801f7800010278007a
:101d9000110009000985d8000102fd004f007800fc
:101da0004322dd000b0242005403be004402be0089
:101db0001f0037000480fb0029f62100ea4f520083
:101dc00014003600a2002000110009000280d80093
:101dd00000017800010478004311dd000901410091
:101de0006022b8000600200007fe23004220900079
:101df000d2209000f2219000622190006e0907002d
:101e00004344dd00090444003802be002803be003c
:101e1000070037004300dd00090040006022b800e1
:101e20000600200007fe23005001be004000be0057
:101e3000610907000002be000203be006fa8970000
:101e4000ffa897000fb197009fb19700a507070063
:101e5000e0af9f00f1af9f0082b79f0093b79f0054
:101e60000fa49700e90f540015003c006022b80051
:101e70006033b8006fa89700ffa897000fb19700d4
:101e80009fb19700780807000000e00032003200a0
:101e90006fa89700ffa897000fb197009fb1970018
:101ea000da080700e00f5000e08f5800e00f5900fb
:101eb000e08f590028003a00e10f5400260034005a
:101ec0000400200005002e00b6e0220017012400c7
:101ed0002fa89700bfa897004fa99700dfa99700e8
:101ee000fd0707000000e00002003d007300540001
:101ef000010037007200540080a79f000fc09700b8
:101f000089fd0700a0af9f00b1af9f00c2af9f0047
:101f1000d3af9f000002be000203be006fa897006f
:101f2000ffa897000fb197009fb19700f407070033
:101f3000b60807000205be000004be006000b8003d
:101f40006011b800a0a79f00b1a79f00c2a79f0083
:101f5000d3a79f002e0037006fa89700ffa8970017
:101f60000fb197009fb19700a80807000205be00b7
:101f70000004be00e00f5000e08f5800e00f590051
:101f8000e08f590002003500d10807001300370028
:101f900010002000010020006011b800080060005f
:101fa000898060000a0161008b8161008b03d10090
:101fb0000a83d3008982d3000882d3000000720014
:101fc000818072000201730083817300c0080700e2
:101fd0000002be000203be00420707000002be006e
:101fe0000203be006fa89700ffa897000fb19700eb
:101ff0009fb1970065090700a0a79f00b1a79f00a8
:10200000c2a79f00d3a79f000000eb0080a79f00fe
:1020100014c0b300a52e22000b0037000400fb0003
:102020004300dd00050040005001be004000be003e
:102030000040e10001c8e10002d0e10003d8e10066
:10204000030039000442e800f44f5200f3ff3a0065
:10205000c47f9f000400fb00bfb0970000804000d9
:102060008fa09700010040004fb19700000751007a
:10207000bfb197000300e000010032000e07e90045
:1020800063806600010032000e07e9000d28a300fe
:1020900026003200e18066000d18a3000c0032001b
:1020a000d00220000100e00001003a000080e900b9
:1020b000efb097001c050700e10f40001800320048
:1020c0002fb297000402e800a4b79f001400370065
:1020d0000100e00012003200efb097000002200083
:1020e00011050700e10f40000d003200afb297006c
:1020f0008502e800a5b79f0009003700efb0970000
:102100000003200008050700e10f40000300320033
:102110002fb697000c06e800acb79f000e07e90049
:102120000e00e000f5ff3c003d0037000d38a30035
:102130000a0032000b003700efb0970000022000c9
:10214000f9040700e10f4000030032002fb09700b0
:102150000000e800a0b79f000e07e9000e00e000b5
:10216000f5ff3c00e18066000d18a3000c00320072
:10217000d00220000100e00001003a000080e900e8
:10218000efb09700e8040700e10f400024003200a0
:10219000afb097008100e800a1b79f002000370092
:1021a0000100e0001e003200efb0970000022000a6
:1021b000dd040700e10f4000190032002fb1970045
:1021c0000201e800a2b79f00150037000000fb00e5
:1021d0004300dd00a12e2200010040003002be00bd
:1021e0002003be000800be000a01be00c1090700ae
:1021f000a4002000050020006033b800c4090700d7
:102200000003b000efb09700c7040700e10f4000e3
:1022100003003200afb197008301e800a3b79f002d
:102220004f7a97000440e900c07f9f00e14f4000d3
:10223000e6ff3a000b003700efb0970000032000e4
:10224000b9040700e10f400003003200afb297006d
:102250008502e800a5b79f000fa097000000e900e5
:1022600080a79f000fa097000000e000f2ff3c0055
:102270003fb6970020c1b300f20f560001003c00aa
:102280006fe09700c07f9f00cf7897000100fb00b0
:102290003fb1970000005100e0a79f000104e0005b
:1022a00008003200efb09700e00220009e04070013
:1022b000e10f400003003200afb197008301e80056
:1022c000a3b79f004f78970097fc07000002be005d
:1022d0000203be002fa09700bfa097004fa1970058
:1022e000dfa1970034080700c80707001e00370069
:1022f0000000fb004300dd00ac2e22000c0040007b
:102300003002be002003be000800be000a01be006d
:1023100078090700a4002000050020006033b80001
:102320007b0907000003b000efb097007e040700b0
:10233000e10f4000030032002fb297000402e800d2
:10234000a4b79f00cf7a97000500fb004300dd0093
:102350000c0040003002be002003be000800be009a
:102360000a01be006a0907000205be000004be00a3
:102370004f7e97000c40e900c07f9f00e14f400076
:10238000dbff3a000006eb0009003700efb09700d2
:102390000003200064040700e10f40000300320046
:1023a0002fb097000000e800a0b79f000c06e800df
:1023b000efa09700810f5600f4ff3a000d38a300fc
:1023c000a10132000e00e0009f0134000006eb0086
:1023d000efb097000002200053040700e10f400017
:1023e000030032002fb197000201e800a2b79f005e
:1023f0000c06e8008e0f560093013200f4ff370000
:102400000d007800000cb20028003a000d00e0003a
:1024100005003d008fb997004305be004304be0090
:1024200083bf9f00140037000d48a3000b0032004b
:102430000fba97004400be0084bf9f004f89de00a2
:10244000cf91de000002be00020378008203780014
:102450000605be000404be00070037008fba9700cf
:102460004500780085bf9f0000047800cfc4de00df
:10247000090578008a057800e00f5400e08f5c00c1
:10248000e00f5d00e08f5d0020003d003d00b300e7
:102490006000b8006011b80008045000898458003a
:1024a0000a0559008b855900180037000d00e0001f
:1024b00005003d000fbe97004c05be004c04be0059
:1024c0008cbf9f00110037000d48a30008003200a8
:1024d0008fba97004500be0085bf9f0004017800b9
:1024e000840178000205be000004be00070037002a
:1024f0000fbe97004c0078008cbf9f00000478004e
:10250000090020000a0020000b0020003fb09700c7
:102510000000e00007003a00e00f5400e08f5c008c
:10252000e00f5d00e08f5d0002003a001100200026
:10253000b1b79f000d0778000e0cb2000004200018
:10254000800f57002f00320003003c000e00e00017
:10255000070032003f00370000082000800f5700be
:1025600014003200000c2000800f570039003a00a0
:1025700014c0b300a52e22000b0037000400fb009e
:102580004300dd00050040005001be004000be00d9
:102590000040e10001c8e10002d0e10003d8e10001
:1025a0002b0039000442e800f44f5200f3ff3a00d8
:1025b0002700370000012000010020006011b80052
:1025c00014c0b3000040e10001c8e10002d0e10006
:1025d00003d8e1001e003900450020000000d000b3
:1025e0008180d2000281d2008381d2008502e9007d
:1025f000faff3a000442e800f04f5200f1ff3a00bf
:102600001300370080002000010020006011b80096
:1026100014c0b3000040e10001c8e10002d0e100b5
:1026200003d8e1000a0039003c0020000000d0007f
:102630008180d2000281d2008381d2000c06e900a1
:10264000faff3a000442e800f54f5200f1ff3a0069
:10265000c47f9f00cf7897000100fb003fb1970037
:10266000820f500002003d00c27f9f00040037002f
:10267000bfb19700808f510001003d00b0b79f00af
:102680004fb297000400e00004003200638066004f
:10269000020032000402e900c4b79f000de8a30065
:1026a0000b003200cfb297003fb697008c8f5200dc
:1026b00003003c000000eb00c0b79f00040037009f
:1026c000cfb097003fb1970082805000c1b79f0004
:1026d000cf7997000300fb000002eb0094a79f0056
:1026e000cfb29700808f5200020034000080520069
:1026f00090a79f000d28a30037003200e1806600fc
:102700000d18a3000c003200d00220000100e000f0
:1027100001003a000080e900efb097008203070053
:10272000e10f40000e0032002fb697000c06e800c3
:10273000acb79f000a0037000100e000080032003b
:10274000efb097000002200077030700e10f400080
:10275000030032002fb097000000e800a0b79f00f0
:102760009fa097000100e0000f0032000006eb0080
:10277000efb09700000320006b030700e10f40005b
:10278000030032002fb197000201e800a2b79f00ba
:102790000c06e8009fa19700830f5600f4ff3a0053
:1027a0000002eb0094a79f00bfb29700c328dd0092
:1027b000202e22008080400091af9f004228dd0043
:1027c0006400500080af9f006328b900f0a79f000d
:1027d00063065000820037001fa697000c00e0003f
:1027e00011003200688066000f003a000006780091
:1027f000efb09700000220004b030700e10f4000fc
:10280000030032002fb097000000e800a0b79f003f
:102810000c06e8009fa09700810f5600f4ff3a00d5
:102820000001eb0092a79f00e18066000d18a30055
:102830000c003200d00220000100e00001003a004c
:102840000080e900efb0970037030700e10f400078
:10285000d5ff3200afb197008301e800a3b79f0016
:10286000d1ff37000100e000cfff3200efb097004a
:10287000000220002c030700e10f4000caff3200d5
:102880002fb297000402e800a4b79f00c6ff3700ec
:1028900000042000800f57003000320003003c008d
:1028a0000e00e000070032003d0037000008200065
:1028b000800f570011003200000c2000800f5700dd
:1028c00037003a001fa897003002be002003be0068
:1028d0000800be000a01be0006080700a400200090
:1028e000050020006033b8000908070004c3b300e6
:1028f00004424000c47f9f0029003700b5442200f5
:10290000d5b79f000d58a30002003a00c045220031
:10291000d0b79f0014002000050020006033b800ed
:102920008fa897008100e900050033000402d00061
:102930008582d2000683d2008783d200f9ff370058
:102940000800be000a01be00ea0707006f00600031
:102950005fb197006240780010003700140020003b
:10296000050020006033b8008c0178008301e90085
:10297000050033000402d0008582d2000683d20015
:102980008783d200f9ff37000800be000a01be00ad
:10299000d8070700674060000043b000c07f9f0079
:1029a0004f7a97000400fb00efb09700de020700ab
:1029b000e10f400003003200afb297008502e8004b
:1029c000a5b79f001fa897006800500090af9f0018
:1029d0008fa89700e480500081af9f0063065600e7
:1029e000d0ff2f003fb197000090b900ffa19700e2
:1029f0000080410063005000800f5600a4ff3a00a1
:102a00000d38a300100032001fa297000400e00060
:102a10000d0034000006eb00efb09700000220002c
:102a2000c1020700e10f400003003200afb297007f
:102a30008502e800a5b79f000c06e8001fa09700dc
:102a4000800f5600f4ff3a007fb19700b240780043
:102a5000f2b79f00c17f9f000104e00014fb3a0021
:102a60002fb097004f0778004f06be004f05be00fd
:102a70004f04be008f03b100000006000c00fa00f6
:102a8000a0bf9f00c0bf9f002ff90700b0bf9f00ed
:102a9000f0bf9f00100c2000d0bf9f007481570032
:102aa000efb097006c8057002e0007000080fa00fe
:102ab00000000600889fbe00000478008144780072
:102ac00000fd2f0000004400e90f500002003e000e
:102ad000000178000d003700080078001902070097
:102ae0000000e00003003200080078001b0207002d
:102af0000004780008007800000207000000e000f1
:102b00000700320090fa2f00000144000980fb000a
:102b1000800f510002003d000280fb0001003700e1
:102b2000f00f20004f04be0000000600881f780050
:102b3000602b81004802070000047800f9010700bb
:102b40000000e000faff3a00e10f44000300320009
:102b5000612b810008007800bd0207004f04780057
:102b600000000600ec874700889fbe008a9fbe00d9
:102b70008c9fbe008e1f780081bf9f0002077800e7
:102b8000602b89008046eb00040137008884fb003d
:102b900009007800e3010700800078000000e000f1
:102ba00002003200e1ff0700fc00370050c2b30012
:102bb000804f5400f0003a000fbd970020c0b300d2
:102bc000c0ef9f00d1ef9f0081ef9f00030037000f
:102bd00040c0b300c0ef9f000fbd97000fb9970032
:102be000b240780082bf9f008184fb0090c6b30092
:102bf00080cf50003500320017003e006640500084
:102c000080cf5000620032000c003e007740500040
:102c100080cf50002800320006003e000104e00092
:102c20009b003200a0c2b30080cf50006e003a007b
:102c30001d00370080c5b3001600370040c6b30042
:102c400080cf5000210032006440400080cf50000f
:102c500065003a001200370030c7b30080cf500043
:102c60001e00320007003e006740500080cf500039
:102c7000110032006340400080cf50005a003a00fb
:102c80001400370050c7b30080cf50000f0032004f
:102c90006340400080cf500053003a006500370089
:102ca00020c0b300cbff3700dfe897008140e80089
:102cb000d1ef9f00c8ff37004fe9970080c0b300f5
:102cc000e24f5100c3ff3a00c1ff3700acc0b30070
:102cd000590037008cc0b3005700370093ff07003e
:102ce000dfe897000104e00002003a004e0178009e
:102cf000d2b79f00602b8100d70107000004780045
:102d0000e10f4000a20032008fec97001200370064
:102d10000a85e8008abf9f00160037008fb8970029
:102d20001100fb00800f5400f9ff32005fe99700ab
:102d30000204e00003003a005fb0970008587800f2
:102d4000d0b79f008944e9000a003200602b81005f
:102d5000c1010700000478000800e800e10f5000fe
:102d600004003600080078006e0107000000e00053
:102d7000eaff3200dfe897000104e00087003a0034
:102d80008d46e8005fb19700014978008300370065
:102d90005fe897000004e00003003a008d46e80079
:102da000ce007800d1b79f00602b8100aa010700f8
:102db000e10f4000760032005fe997000204e00076
:102dc00003003a00dfb0970080587800d1b79f0029
:102dd0000fe997000241e90082ef9f004240a900fd
:102de0006e003400f0ff37000180fb0008fd2f006b
:102df00008004000e90f50005f003e000a00780024
:102e000014f8070080ef9f00880078000300370067
:102e10000fb897000000e80080bf9f000fb997002f
:102e20001200fb0001004000e90f5000f8ff3600df
:102e300069ff37000cc1b3003cff0700602b810025
:102e400085010700000578000040eb00e0ef9f00df
:102e5000d0022000800f550005003a00602b810051
:102e60007d0107000005780011c0b300e1ef9f006d
:102e70008c4078000a0078000eff0700e14f400008
:102e80000a003a00612b81000a007800f001070077
:102e90000d04e0004b003a00602b810030009000f0
:102ea0000048a30043003200480037008fed970030
:102eb0006044b8000c81fb00030020000800be0045
:102ec000df0507000004be008c4078000a0078008f
:102ed000f8fe07000080fb0001002000080440000d
:102ee000898448008b45e90007003200602b81008f
:102ef00059010700000578008c407800edfe0700be
:102f0000e14f4000ebff3a008c4078000a00780067
:102f1000e8fe0700e14f400003003a00612b81000a
:102f20000a007800ca0107006fe997000204e00078
:102f30000200320060041400e0841c005fe8970087
:102f40000004e00015003a008d46e800cfe8970045
:102f5000e4cf500003003a004e0078000888be001d
:102f60000e0037000e81e900020778001200780099
:102f70000808780009003700602b8100360107003f
:102f8000808f540005003200e10f40000b003a0032
:102f90000d04e0000d0032000a0037008fb89700e2
:102fa0003144780081bf9f000804e000f7fe3a003a
:102fb000040037000000eb0005003700612b8100a2
:102fc000a30107000d80fb00010037000080eb002b
:102fd0004f0778004f06be004f05be004f04be00ed
:102fe000cf00b10000000600889fbe008a9fbe008f
:102ff0008c9fbe0000017800e15022001100e0002b
:103000000b003a00205122007028890050288900c6
:103010009128890061288900214090000004a000c7
:10302000a0409800614090000004a000e04098009b
:10303000e7004100c208de00c20cdd006428810008
:103040006d572200605f22000d0550002200200015
:10305000811f7800110009000205d80000067800e1
:10306000cf007800c308dd00e48540008001eb005c
:1030700066572200e5502200010037000102780067
:10308000244090000008a300020032000a0037002c
:10309000110a780094007800214090000008a300f5
:1030a000fbff320009014200828f5000020039000c
:1030b000840f51004600310094007800848f500046
:1030c000eeff3e00868f500002003900858f5000d1
:1030d000eaff390050288100800f52004f003a006b
:1030e000858f50004d003a008301e800e18f5100c8
:1030f000e2ff36008c8f5400040036008a8f5400a3
:10310000020031000b04780012003700614ab80059
:103110006151b900b0ff2f000100200002005000f3
:1031200083805800800f5200818f5a0002003500c2
:1031300009047800070037000d805400925f2200d8
:1031400002004000110009000a80d8000a80b9007e
:103150000004780008007800bd02070080017800b4
:10316000e10f40002d003200502881000308780054
:103170005228810064004100a2409000808f5100dd
:10318000020032000104a000010037000104a10088
:1031900021419800088041006400500080097800b7
:1031a00050288900e250220002087800512881004e
:1031b000214090000004a000a0409800234090000f
:1031c0000004a100a041980002027800a7ff370088
:1031d00062288900828f5000090036009200780032
:1031e00080502200a24190000348780031288900d5
:1031f000140978008040eb0060288100214098008d
:1032000060288100000a7800244090000004a0009b
:103210002042980064004200010037000000eb00eb
:103220004f06be004f05be004f04be000000060062
:103230006400500060288900a04090000104a100b3
:103240002140980000000600889fbe008a9fbe00b3
:1032500000057800e401500013001000c285de0074
:10326000234090000008a300040032006328890076
:10327000234090000004a100a041980001007800c4
:1032800059ff0700000478000000e000170032003a
:103290008a0f50001500320060b8970008005000f7
:1032a000c284de00898f5500010036008905780050
:1032b0004259dd008a00780008007800d301070039
:1032c0008a0f5400090031004248dd00000044002c
:1032d0008a0f5000050036000a005000000044002c
:1032e00032288100432881000288be00080078004f
:1032f0004f05be004f04be00000006001004b100e0
:10330000070035009001b100040034007000b100e6
:10331000030035009001b10001003c0010000500e1
:10332000000005006900e100040035006d00e100c7
:10333000030034000002b10001003200000005006b
:10334000100005001004b100030035009001b10029
:1033500001003c001000050000000500800078001e
:103360001104b100030035009101b10001003c00df
:103370000050a00000000600889fbe008a1f780051
:1033800000047800300090006300600024003200e8
:1033900008007800e20007003805900080ef2f0059
:1033a0000000650030049800280090000000e00054
:1033b00004003200e804650002003a00d40007006f
:1033c0002904980048009000d8010700e10f400050
:1033d00013003200b80090000102b20010003a0061
:1033e0000ac8a30018003200702b81000000e00022
:1033f000150032000001780081047800012a2000c5
:1034000012289000880f5000070032004205b000db
:103410004905b000818f54000b003200f8ff3700df
:103420000080eb000900370002007800ff01070070
:10343000702b8100090040008000eb0011289800eb
:1034400001007800010037000000eb004f05780014
:103450004f04be0000000600881f780000047800ba
:10346000b00090000148a30007003a000108a30043
:10347000050032000198a3000800320010009000ff
:103480000000e00005003200380090000040a0007d
:10349000300498008080eb00200037000190a100ec
:1034a00031049800180090000000e000060034008d
:1034b0000000e9001004980018007800b080fb00bc
:1034c000000c780006003700380090000068a30068
:1034d000edff3a0008007800bb000700800078008c
:1034e000380090000078a3000c003a00fa8f5000da
:1034f00008003a00280090000000e000e2ff3200df
:10350000180090000000e80010049800180ce90072
:10351000ddff3700ed8f5000e2ff32000100780040
:103520004f04780000000600889fbe00000178006c
:1035300001047800b10090000118a300400032009f
:103540000198a30003003a00180090000000e0007a
:103550003b003a000190a0003104980082047800fa
:10356000f90fb200180090000000e00002003a00dd
:1035700028009000000c7800ea8f540006003a0002
:10358000380090000078a30003003a00880078001b
:10359000d0002000e4ff0700180290006121b9006c
:1035a00058009000e8009000800f5100818f590072
:1035b0000b0032000400e8001004980018007800a6
:1035c00009587800000c780011c0b3004055220063
:1035d00001487800ea8f54000600320019003700d5
:1035e0008800780009407800c50007008004780052
:1035f00014003700380090000088a300110032004a
:1036000018019000a80090004800900050010700a9
:1036100098009000810f50000400320038009000a4
:103620000003b300300498008084eb000000eb003e
:103630001004980028009000000c7800010037006a
:103640008084eb00090078004f04be0000000600f3
:103650000003780001027800e10f40001a003200f8
:10366000310090000008a300170032000098a3006a
:1036700015003a00a10390000700e000120032009c
:10368000910290006129b90051009000e100900082
:10369000800f5100818f59000b0032001400780018
:1036a000870f500002003a00000ae80002003700cd
:1036b0000500e800100298001400e900000a7800f4
:1036c00006487800010037000083eb000600780010
:1036d00000000600812b81000100e00003003200a1
:1036e00011007800802b89000300370020002000a3
:1036f0005701070080007800e18f400002003a0087
:10370000906e26001063880001007800000006001b
:10371000812b810001087800802b890000000600c1
:10372000881f780000047800300090000008a30093
:1037300007003200800078000120b20004003a0047
:1037400011049800a8009000010c780017003700c1
:103750000018a300190032000098a30017003200df
:10376000a80090000100e000140032001801900051
:103770000200e0001100320048009000f400070051
:1037800098009000810f5000030032003800900034
:103790000003b300300498000000eb001004980010
:1037a00028009000000c7800380090000058a3001a
:1037b000020032000080eb00010037000000eb0047
:1037c0004f047800000006000200fa00889fbe0047
:1037d0008a1f7800000478000000eb0010049800b5
:1037e000380090008080eb000008a3003f0032000a
:1037f000405522001004e00010003200094722006a
:103800006a4722001a0078006c0545002010b200bb
:1038100021102000810f500002003a0009007800ba
:10382000bfff0700ec84440040492200808f540011
:10383000f4ff3a00405522000048eb004800900099
:10384000580190000200e0000d003a0012049800b8
:1038500012002000e88057007b000700e10f5000b5
:1038600003003a000ff897008080fb001f0037002c
:10387000380090000040a00030049800120037008b
:10388000a800900070000700100498000000e000fd
:1038900003003200e10f40000d003a000300370042
:1038a000380090000040a00002003700380090006f
:1038b0000003b30030049800a8009000010c7800c9
:1038c0000000eb00100498008080eb000700370038
:1038d000a8009000010c78000000e9001004980096
:1038e00001007800b080fb00000c78000100780037
:1038f0004f0578004f04be000080fa00000006006b
:103900000200fa00889fbe00a0ff9f00010478001b
:10391000b1009000810478000904b2000200320076
:103920000000fb00360037000118a30005003a0034
:103930000103b30031049800190498000080eb00e3
:103940002f003700580090000000e00006003a0009
:103950004800900012002000e68057007c0007001d
:103960001904980024003700280090000000e000af
:1039700008003a000055220020049800000c78004e
:103980002000200050049800100498000130a0008e
:103990003104980018019000a800900048009000a1
:1039a0006b00070028009000000c78000080eb00fe
:1039b0001004980018007800aff8970001587800bc
:1039c000000c78002ff89700ea4f50000a003a00e8
:1039d000380090000088a300070032001801900012
:1039e000a8009000480090005900070019049800b2
:1039f000a8009000010c7800aff897000100fb00d0
:103a00004f04be000080fa00000006008001eb00b9
:103a10000200370061f079008301e800828f5100d5
:103a2000fcff3a00000006000c02e20004003d002a
:103a30000f42ab00020032000f02ab00feff32006b
:103a40000040da00feff37000a00fa00881f780005
:103a5000800178000000e00029003a00902b8100ee
:103a6000e10f500008003200e02120000000e000db
:103a7000050032006421200085212000c72120009c
:103a80008001780004003700c4202000e5202000d9
:103a90002721200043212000144090000004e00072
:103aa000040035008009eb00144090000074a00071
:103ab000104298000002eb000c003700130a2000af
:103ac000154478006140640002003a008301e90077
:103ad000fbff3a000402e8009541780061c06100f4
:103ae0000500320017007800805878000403510068
:103af000820f5200f1ff3a00060051000800370023
:103b000020002000a0bf9f00b3bf9f00c1bf9f0047
:103b1000d2bf9f006c80570000c0da005fb89700ea
:103b20004f0478000080fa00000006000a00fa0046
:103b300011002000b1bf9f00c0bf9f006a805700e6
:103b400000c0da004fb897000080fa0000000600bd
:103b50000a00fa0080017800e20f500028003e00c1
:103b6000902b8100e10f500008003200e02120007e
:103b70000000e000050032006421200085212000c3
:103b8000a62120008001780004003700c420200016
:103b9000e520200006212000432120001440900051
:103ba0000004e000040035008009eb0014409000a0
:103bb0000074a00010429800154090000028a30057
:103bc00003003a00154090000024a00090429800a5
:103bd0008001eb0007003700154090000008a300ab
:103be000fdff320063c078000000fb00000b78008e
:103bf0008301e800828f5100f7ff3a000800370088
:103c000030002000b0bf9f00c3bf9f00d1bf9f0006
:103c1000e2bf9f006a80570000c0da006fb99700ca
:103c2000020078000080fa00000006000a00fa0096
:103c300051002000b1bf9f00c0bf9f006a805700a5
:103c400000c0da005fb897000080fa0000000600ac
:103c5000889fbe0080047800a02b81000000e00057
:103c600003003a00100007000000e0000a003500e1
:103c7000a02b81000900e00002003a000004780057
:103c80000600370000047800090040000600070025
:103c90000000e00001003d000084eb000800780017
:103ca0004f04be0000000600800078000000e00025
:103cb00004003a0060572200a02b8900010178001f
:103cc000060037000081eb00605f2200808f50000b
:103cd00002003e00a12b89000001eb0002007800e9
:103ce000000006002800fa00889fbe008a9fbe00e0
:103cf0008c9fbe0007067800878669000c003b0099
:103d0000030478008704780008f0a10009f0a100fe
:103d1000840f5000858f5800860f5900890f5c0072
:103d2000030033000cf0a20001003a000cf0a100e7
:103d3000fe0007006400e1005f00320078014700e8
:103d40006408e100610032006c014700748557008f
:103d50003200be001201be003a04be001a05be00c9
:103d60001e039000be0a90008503530006003d002c
:103d70000004fd008104fd000205fd008305fd0037
:103d80008703ea00050378000df8a3000400320061
:103d900060041400e0841c0060051d00e0851d0027
:103da0006022b8007d0320000d38e1008006eb00a2
:103db0000b0039004433dd00f300b20083017300cf
:103dc00039003700848272000d027800e106640039
:103dd0008b85d1000a85d3008984d3000884d30061
:103de0008703e900f7ff3b00080040008980480096
:103df0000a0149008b81490004003b00600010006b
:103e0000e080180060011900e08119000358a30048
:103e1000090032008d8272008482720061026000ab
:103e20008301d1000281d3008180d3000080d300c0
:103e30000603e8001b0037000348a30017003a0000
:103e40000600e000170034000603e9000d00a3009f
:103e50000000480081804800020149008381490038
:103e60000348a3000f003a000600e00009003400f8
:103e70000603e9000000400081804800020149007b
:103e80008381490001003a000003eb000348a300ce
:103e9000f5ff32006022b800020037008482720011
:103ea000618266007500070003f0a1000cf0a70016
:103eb00003f0a000b1003700640147006408e1008e
:103ec00002003a000df8a300a9003a003200be003b
:103ed0001201be00a90037008f1fd10007030700a1
:103ee0008f87e9000000e00000000600809feb00e3
:103ef000020307008f87e9000000e00000000600d1
:103f00002800fa00889fbe008a9fbe008c9fbe00da
:103f100003866b00850007006400e1004400320066
:103f20006408e1004a0032006100e100460032000e
:103f30006108e10049003200ec0647006000b8006b
:103f40003d02be003d03be00f48657006011b8007c
:103f50003d04be003d05be007d0320000b00370080
:103f60000000a0008d06e9001300320004024200a8
:103f700085824a0006034b0087834b000000400007
:103f800081804800020149008381490008025200f3
:103f900089825a000a035b008b835b00f0ff3b00c1
:103fa0000802420089824a000a034b008b834b00bf
:103fb0008d06e900edff3a0084827200868272006d
:103fc000f707b2008782720001003200150020005e
:103fd0001e0490003e0b900006035400e63fb00024
:103fe0000368a300070032000000a7000500a0003e
:103ff0008301d1000281d3008180d3000080d300ef
:104000000603e8008301d1000281d3008180d30040
:104010000080d3000002eb000482d20017000700ea
:1040200003f0a1000cf0a70003f0a000530037003c
:10403000640247006408e1004d0032003400be0015
:104040003401be00f6ff37006108e100480032008d
:104050006011b8006000b800f1ff370003ff2700cf
:1040600002002000fbff3700801feb00a3020700c7
:104070008f87e9000000e000000006001800200023
:1040800057002000080453000d003d0006002000ea
:1040900097fc2f000740e1001e003400848272006c
:1040a000610260008301d1000281d3008180d300ce
:1040b0000080d3000804e800f8ff3a004700200021
:1040c0006104600005047400040464000d00320003
:1040d00061004000e080480060014900e081490043
:1040e00003b8a500070032000603e8006538e100c8
:1040f00004003a008301d1000281d3008180d30003
:104100000080d300f87f20000830e1000300350074
:10411000080378006000b8006011b8004433dd0087
:10412000f300b2008301730000000600680447003a
:104130000294be000094be00fc0447008694be00ba
:104140008494be0009007800b502070008007800da
:10415000b302070099007800814f70000b003b000c
:104160000800be008e0207004f00b10003003700b8
:10417000f3ff2700f2ff2f006110b9004f06be00c9
:104180004f05be004f04be000080fa00000006008c
:104190008103780040f207000001be006000b80013
:1041a0000478a30013003a006220e10015003e00ed
:1041b0000d0039008301d1000281d3008180d3003a
:1041c0008301d1000281d3008180d3008301d1001b
:1041d0000281d3008180d3000538b000c42add00fd
:1041e000f300b2008381720007f0a70003f0a00083
:1041f00000000600f3ff2700f2ff2f006110b90056
:10420000fbff370003ff2700f7ff37001400fa0019
:10421000889fbe008a9fbe008c9fbe000004be0027
:104220000205be00680047000a90be000890be006c
:104230007b0207000070a7000bf0a1000bf8a300a1
:1042400020003a009e0990000e099000fe009000a8
:104250006e0090009e029000344320008482520041
:10426000c6ff32000a003c00b4fc2f000428e10025
:10427000140034008301d1000281d3008180d30077
:104280000080d3008502e800faff3a00bbff370048
:10429000b40020000428e10007003c0000004000ba
:1042a0008180480002014900838149008502e900bc
:1042b000faff3a00b1ff3700030028000200200097
:1042c000010037006011b8006000b800abff370094
:1042d000889fbe00830478000300e0002c003500b6
:1042e00003003c00008270000402710026003200ce
:1042f00036432000c50020008383cf000a00390028
:104300000541b1008283cf00070039000541b100ab
:104310008183cf00040039000541b1008083cf00c4
:10432000010039000541b10085c353006022b80087
:10433000120032000a003b008482720061026000b9
:104340008301d1000281d3008180d3000080d3009b
:104350000603e8008743e800f7ff3a00070037004c
:10436000000040008180480002014900838149002b
:104370000603e9008743e900f9ff3a003fff070021
:1043800009f0a70003f0a0004f04be0000000600e3
:1043900060001000e080180060011900e081190041
:1043a000d3ff3b00033e2c00f7ff3700c601070098
:1043b00005097800000006002800fa00889fbe006a
:1043c0008a9fbe008c9fbe0003866b0057ff0700cc
:1043d0000028a30064003a000128a30067003a0007
:1043e0000008a30062003a000108a30065003a003b
:1043f0001e009000be08900081064000ed3fb10015
:10440000f4805700ee019000111ab8008e09900058
:10441000311bb8009e099000311cb800511db80036
:10442000f485570046000700fe0190003a0007009f
:104430008b85e8003e0007008e09900040000700d1
:10444000ee019000340007008b85e800380007007b
:104450008e099000400007009e0990001b18b800cc
:10446000890440000a854800fe01900034000700de
:104470008b85e80038000700ee019000300007004f
:104480008e0990001b18b800890440000a85480076
:104490000a98a30008003a000402420085824a00fc
:1044a00006034b0087834b0008044c0089844c00b2
:1044b0000a054d008d06e9008482720085027300b2
:1044c0004c3add0085027200010032001500200028
:1044d000443ade001400b2004538de00cb45dd0072
:1044e0000b007000c540de00cb4ddd008b807000fe
:1044f0004549de00cb55dd000b017100c551de00e2
:104500000d037800ddfe070003f0a1000cf0a7000a
:1045100003f0a00019ff37001b18b8008502400007
:1045200006834800e0834b0060044c00070037001e
:104530001b18b8000603400087834800faff3700c5
:104540001b18b8008703400008844800e0844c0032
:1045500060054d00000006001b18b800080440006c
:1045600089844800faff37000108a30000ff3a00e1
:104570005800be005801be00e3ff37000008a3004a
:10458000fbfe3a0009047800f9ff370007f0a200ab
:10459000d4fd37001400fa00889fbe008a9fbe0039
:1045a0008c9fbe000005be000206be0068004700ea
:1045b0000c90be000a90be00990107006400e10063
:1045c0001a00320016003e006100e1001a003200bd
:1045d0006e049000fe0490000e0b90009e0b900065
:1045e0006011b8009e0590000b38b100d501200085
:1045f00082817100610164008703d1000683d300ca
:104600008984d3000884d3008502e900f8ff3a00ca
:10461000fbf007000df0a70001f0a000d7fe370067
:10462000f1ff2700f0ff2f00d4fe370001f827002c
:1046300000002000f7ff37006000b800f5ff3700ea
:10464000020ab900001bb9000200b8008100420054
:104650008100430000000600881f780000047800f5
:104660005001be004000be000400400085804800ac
:104670000601490087814900009cbe000294be00eb
:104680000400e1000588e1000690e1000798e100e0
:1046900002003100680044001008e8004f04780070
:1046a00000000600f4874700889fbe008a9fbe0076
:1046b0008c9fbe008e1f78000205be000004be0065
:1046c000d4b79f00e5b79f00f6b79f0087bf9f0054
:1046d0000000eb00c0b79f00b0b79f00a0b79f00dd
:1046e00090b79f0080b79f000d042000bfb09700d7
:1046f0004fb09700000140000000e0000f003d00b7
:104700004f08de0000007100c0b79f004d00070099
:1047100001003d00120020005000070001003d0094
:104720001200200055000700610007006600070026
:104730000f004000c8ff0700220037004f08de00ce
:1047400000067100ccb79f003e00070001003d004d
:10475000120020004100070001003d00120020006f
:1047600046000700520007000fb297009fb2970063
:104770002fb39700bfb39700590007000000520005
:1047800081805a0002015b0083815b0080b79f003b
:1047900091b79f00a2b79f00b3b79f000007eb003f
:1047a0004f0007000020e10001a8e10002b0e10095
:1047b00003b8e100010031001e0020000e00560089
:1047c000c0b79f004fb297000400e000070035001b
:1047d00010002000010020006011b80008047000e3
:1047e000898470000a0571008b8571008d06e900cf
:1047f000beff3a000400e00003003d003200070065
:104800000f00400094ff07004fa897000000e00051
:1048100004003a000fb497009fb497002fb597009b
:10482000bfb597000800be000a01be004f07780020
:104830004f06be004f05be004f04be004f01b10041
:10484000000006000180400090b79f000001eb00cf
:104850008fb097000100e000000006000200700029
:1048600090b79f000180400080b79f000001eb00df
:10487000ffa897000100e0000000060002007000a1
:1048800080b79f00018040006faa9700cf20de0014
:1048900001007000f0af9f00040242000800be005b
:1048a0000a01be004f18de00000272000000060080
:1048b000e4af9f000804440089844c000a054d00c1
:1048c0008b854d00000006003fb29700cfb29700e5
:1048d0005fb39700efb3970000fe2f0000000600c3
:1048e0003fb09700cfb097005fb19700efb197004e
:1048f00000000600881f780018002000881f78003c
:1049000068ff07008f87e9004f0478000000060069
:10491000801feb0063ff07008f87e900000006009f
:10492000889fbe008a9fbe008c1f78000205be00d3
:104930000004be00e00f5000e08f5800e00f590067
:10494000e08f59000c003d006000b8006011b80015
:1049500008045000898458000a0559008b855900c5
:104960001c0020001f00070008003d001800070081
:104970000006eb00050037000006eb0019000700f9
:1049800002003d000f0007001c0020000800be00d0
:104990000a01be00d7ff07000203be000002be00ee
:1049a0000c00e00001003200060007000400be0019
:1049b0000601be004f0678004f05be004f04be0042
:1049c000000006006000b8006011b8000000370069
:1049d000040250008582580006035900878359005d
:1049e00000000600e00f5200e08f5a00e00f5b006d
:1049f000e08f5b0000000600889fbe008a9fbe001b
:104a00008c1f78000205be000004be00e00f5000bd
:104a1000e08f5800e00f5900e08f59000a003d0078
:104a20006000b8006011b800080450008984580084
:104a30000a0559008b8559001c002000180007004a
:104a400007003d00050037000006eb0014000700da
:104a500003003d006000b8006011b80015000700b9
:104a60000800be000a01be00a9ff07000203be0045
:104a70000002be000c00e000030032006000b8003d
:104a80006011b8000b0007000400be000601be0064
:104a90004f0678004f05be004f04be000000060020
:104aa000e00f5200e08f5a00e00f5b00e08f5b00e8
:104ab00000000600040250008582580006035900d9
:104ac00087835900000006000003be00f2ef0700d4
:104ad0006220e100020032000600be000500050071
:104ae000e507b100f107b20004f0230084807000f4
:104af00007f0a70001f0a00024000500889fbe0079
:104b00008a9fbe008c9fbe000404be000605be0046
:104b1000809fbe00829fbe002f0007000406780021
:104b20000800be000a01be002b00070084067800c2
:104b30004f03be004f02be008d4f76007fb097003e
:104b400013003300f0ff2f008b8f6b0006003b003b
:104b50000d0666000c00a7000a00370007f0a6004b
:104b6000100020000a003700880f5200898f5a0079
:104b70008a0f5b008b8f5b00030039001000200060
:104b800001003e000000200007f0a7000000ea003e
:104b90004f06be004f05be004f04be0000000600d9
:104ba000e48240001078a300070032006402400055
:104bb0001178a3003400be001401be0004003200ce
:104bc0000330a700000006003500be001501be003e
:104bd0000330a0000000060005ff270005826100e9
:104be000070032000428e100010032002400050023
:104bf0000600070001003a00440005000408050013
:104c000002000700f9ff3a00140005006f826100fe
:104c100081027000850271008502720000000600aa
:104c2000800078005002be005003be004439de0010
:104c3000f700b200f37f2000030161000900320099
:104c40000218e10016003a0085017200830173002a
:104c5000838173000008200015003a004000200006
:104c60001300370085017200830173008381730094
:104c700005003a0004a8be0006a8be0010002000ef
:104c80000b0037000201e9000402420085824a005d
:104c900006034b0087834b000748a300f9ff32004f
:104ca0000740a00004a8be0006a8be002000200007
:0c4cb000800098009200980000000600b0
:020000040000fa
:0200000401f009
:04000000e6bf000057
:020000040000fa
:0200000401f009
:04000400ff7f00007a
:020000040000fa
:0200000401f009
:040008007fff000076
:020000040000fa
:0200000401f009
:04001400ffff0000ea
:020000040000fa
:10000800b0010000b0010000b0010000b001000024
:10001800b0010000b0010000b0010000b001000014
:10002800dc5b0100b0010000b0010000b00100007d
:10003800b0010000b0010000ca590100b001000081
:10004800b001000000690100fe670100f81f01000f
:10005800b0010000b00100005c400100b0010000e8
:10006800b0010000b0010000b0010000b0010000c4
:10007800b0010000bc69010082620100b00100000b
:10008800be6801005e680100b0010000b001000018
:10009800b0010000b0010000b0010000b001000094
:1000a800b0010000b0010000b0010000b001000084
:1000b800b0010000b0010000b0010000b001000074
:1000c800b001000088670100b0010000b001000025
:1000d800b0010000b0010000b0010000b001000054
:1000e800b0010000b0010000b0010000b001000044
:0800f800b0010000b00100009e
:020000040000fa
:10010800b0010000b0010000b0010000b001000023
:10011800b0010000b0010000b0010000b001000013
:10012800dc5b0100b0010000b0010000b00100007c
:10013800b0010000b0010000ca590100b001000080
:10014800b001000000690100fe670100f81f01000e
:10015800b0010000b00100005c400100b0010000e7
:10016800b0010000b0010000b0010000b0010000c3
:10017800b0010000bc69010082620100b00100000a
:10018800be6801005e680100b0010000b001000017
:10019800b0010000b0010000b0010000b001000093
:1001a800b0010000b0010000b0010000b001000083
:1001b800b0010000b0010000b0010000b001000073
:1001c800b001000088670100b0010000b001000024
:1001d800b0010000b0010000b0010000b001000053
:1001e800b0010000b0010000b0010000b001000043
:0801f800b0010000b00100009d
:020000040000fa
:104cbc000c070000574500004c4300004f4d00000e
:104ccc0045200000746f000020740000686500002f
:104cdc002053000065720000436f00006d2000003f
:104cec00707200006f7400006f6300006f6c000046
:104cfc00206f00006e200000652d00005075000034
:104d0c00636b00000d0a0000746800006520000051
:104d1c0045500000464c0000206500006475000002
:104d2c0063610000746900006f6e00002072000067
:104d3c006f6200006f740000207400007970000036
:104d4c00652000002248000022200000666f000051
:104d5c0072200000686500006c7000000d0a0000f5
:104d6c00006100002c250000642c0000256400006c
:104d7c002c250000640d00000a000000612c0000ce
:104d8c00302c0000302c0000300d00000a00000018
:104d9c00622c00002564000020280000256400001f
:104dac0025250000290d00000a000000622c0000df
:104dbc00256400000d0a0000004200002c250000b4
:104dcc00640d0000006200000d0a0000006300008a
:104ddc002c250000640d00000a000000442c00008b
:104dec00256400002c250000640d00000064000008
:104dfc000d0a0000006500002c250000642c00004a
:104e0c00256400000d0a0000004600002c2500005f
:104e1c00640d0000006600000d0a00000067000031
:104e2c002049000052200000636800006563000008
:104e3c006b2000003a20000030780000257800003c
:104e4c002c20000061640000647200006573000097
:104e5c00732000003a200000307800002578000014
:104e6c002c2000006461000074610000203a0000f6
:104e7c002030000078250000780d00000a000000aa
:104e8c00672c0000256400002c250000642c000019
:104e9c00256400000d0a0000006700002c300000a3
:104eac002c3000002c3000000d0a0000000a00001d
:104ebc0000220000412200002020000020200000e1
:104ecc0020200000202000002020000020200000d6
:104edc00202000002041000063630000656c00008e
:104eec00657200006f6d0000657400006572000053
:104efc000d0a000000220000422c000023220000ba
:104f0c002020000020200000202000002020000095
:104f1c002020000020200000204200006f640000d0
:104f2c00792000006c65000064200000303d00001a
:104f3c006f66000066200000313d00006f6e0000bf
:104f4c00203200003d6900006e76000065720000a2
:104f5c00736500000d0a00000022000062220000b0
:104f6c002020000020200000202000002020000035
:104f7c002020000020200000202000002042000003
:104f8c0061740000746500007279000020760000e6
:104f9c00616c0000756500000d0a00000022000025
:104fac0062220000202000002020000020200000b1
:104fbc0020200000202000002020000020200000e5
:104fcc0020420000617400007465000072790000da
:104fdc00207300007461000074650000202800003c
:104fec00313d00006f6b00002c200000303d0000b4
:104ffc006c6f0000772900000d0a000000220000f1
:10500c00432200002020000020200000202000006f
:10501c002020000020200000202000002020000084
:10502c0020530000656c000065630000746f000085
:10503c0072200000706f000073690000746900003a
:10504c006f6e00000d0a000000220000442c0000ce
:10505c00232c000023220000202000002020000030
:10506c002020000020200000202000002053000001
:10507c0065740000206d00006f7400006f720000fa
:10508c00207300007065000065640000206c000057
:10509c0065660000742c00007269000067680000ef
:1050ac00740d00000a0000002245000022200000c0
:1050bc0020200000202000002020000020200000e4
:1050cc002020000020200000202000004765000068
:1050dc00742000006d6f0000746f000072200000df
:1050ec007370000065650000642000006c650000b2
:1050fc00667400002c720000696700006874000080
:10510c000d0a000000220000462c000023220000a3
:10511c002020000020200000202000002020000083
:10512c00202000002020000020460000726f0000ac
:10513c006e740000206c00006564000020300000dc
:10514c003d6f000066660000203100003d6f0000de
:10515c006e200000323d0000696e00007665000094
:10516c0072730000650d00000a0000002247000069
:10517c002220000020200000202000002020000021
:10518c002020000020200000202000002020000013
:10519c004952000020720000656300006569000040
:1051ac0076650000720d00000a0000002267000006
:1051bc0022200000202000002020000020200000e1
:1051cc0020200000202000002020000020200000d3
:1051dc0047790000726f00000d0a000000220000e9
:1051ec004822000020200000202000002020000089
:1051fc0020200000202000002020000020200000a3
:10520c0020480000656c0000700d00000a000000d2
:10521c002249000022200000202000002020000055
:10522c002020000020200000202000002020000072
:10523c00202000004765000074200000636100001e
:10524c006d6500007261000020700000617200004a
:10525c00616d000065740000657200000d0a0000ad
:10526c00002200004a2c0000232c0000232c0000fc
:10527c00232c0000232c0000232c000023220000f0
:10528c002020000020530000657400002063000003
:10529c00616d00006572000061200000706100000b
:1052ac00726100006d6500007465000072200000e2
:1052bc006d6f0000646500002c77000069640000cd
:1052cc00746800002c6800006569000067740000b9
:1052dc00682c00007a6f00006f6d00002831000010
:1052ec002c340000206f00007220000038290000d0
:1052fc002c780000312c0000793100000d0a0000e0
:10530c00002200004b220000202000002020000082
:10531c002020000020200000202000002020000081
:10532c002020000020430000616c00006962000036
:10533c00726100007465000020700000726f000044
:10534c00786900006d69000074790000207300001a
:10535c00656e0000736f0000727300000d0a000090
:10536c00002200004c2c0000232c00002322000003
:10537c002020000020200000202000002020000021
:10538c0020200000204c000065640000206e00000e
:10539c00756d000062650000722c0000303d00004d
:1053ac006f66000066200000313d00006f6e00004b
:1053bc00203200003d6900006e760000657200002e
:1053cc00736500000d0a0000002200004d22000051
:1053dc0020200000202000002020000020200000c1
:1053ec00202000002020000020200000204600008b
:1053fc006c6f00006f72000020730000656e00007f
:10540c00736f0000727300000d0a00000022000090
:10541c004e22000020200000202000002020000050
:10542c002020000020200000202000002020000070
:10543c0020500000726f0000786900006d69000058
:10544c00747900000d0a0000002200004f220000b9
:10545c002020000020200000202000002020000040
:10546c00202000002020000020200000204c000004
:10547c00696700006874000020730000656e00000e
:10548c00736f0000727300000d0a00000022000010
:10549c00502c0000232c00002322000020200000b0
:1054ac0020200000202000002020000020200000f0
:1054bc002053000065740000206d00006f74000024
:1054cc006f720000207000006f73000069740000a0
:1054dc00696f00006e2000006c65000066740000af
:1054ec002c72000069670000687400000d0a00004f
:1054fc00002200005122000020200000202000008b
:10550c00202000002020000020200000202000008f
:10551c00202000002047000065740000206d000072
:10552c006f7400006f720000207000006f73000039
:10553c0069740000696f00006e2000006c6500004b
:10554c00667400002c72000069670000687400002b
:10555c000d0a000000220000522200002020000052
:10556c00202000002020000020200000202000002f
:10557c002020000020200000205200006573000055
:10558c0065740000206500002d700000756300003c
:10559c006b0d00000a0000002253000022200000c6
:1055ac0020200000202000002020000020200000ef
:1055bc002020000020200000202000005374000058
:1055cc006f700000206500002d70000075630000f6
:1055dc006b200000616e00006420000074750000f8
:1055ec00726e0000206f000066660000206c0000e8
:1055fc0065640000730d00000a00000022540000d6
:10560c002c2300002220000020200000202000007d
:10561c00202000002020000020200000202000007e
:10562c00506c000061790000207300006f75000061
:10563c006e640000203100002d3500002065000054
:10564c006c73000065200000737400006f70000024
:10565c00207300006f7500006e6400000d0a0000de
:10566c0000220000742200002020000020200000f6
:10567c00202000002020000020200000202000001e
:10568c002020000020540000656d000070650000b3
:10569c007261000074750000726500000d0a000054
:1056ac0000220000552200002020000020200000d5
:1056bc0020200000202000002020000020200000de
:1056cc00202000002047000065740000206d0000c1
:1056dc0069630000726f0000706800006f6e00005c
:1056ec0065200000616d0000706c000069740000a2
:1056fc0075640000650d00000a00000022560000d1
:10570c00222000002020000020200000202000008b
:10571c00202000002020000020200000202000007d
:10572c005665000072730000696f00006e20000067
:10573c006f6600002053000065720000436f00008c
:10574c006d0d00000a00000022570000222000000e
:10575c00202000002020000020200000202000003d
:10576c0020200000202000002020000057720000a4
:10577c0069740000652000004932000043200000dd
:10578c00286d00006f6400002c720000656700003b
:10579c002c760000616c0000290d00000a0000004e
:1057ac0022590000222000002020000020200000b0
:1057bc0020200000202000002020000020200000dd
:1057cc0020200000526500006164000020490000a8
:1057dc003243000020760000616c00003d28000080
:1057ec006d6f0000642c00007265000067290000da
:1057fc000d0a0000002200004122000020200000c1
:10580c0020200000202000002041000063630000e5
:10581c00656c0000657200006f6d0000657400001f
:10582c00657200000d0a00000022000062220000d8
:10583c00202000002020000020200000204200003a
:10584c00617400007465000072790000207600001d
:10585c00616c0000756500000d0a0000002200005c
:10586c0062220000202000002020000020200000e8
:10587c002042000061740000746500007279000021
:10588c002073000074610000746500002028000083
:10589c00313d00006f6b00002c200000303d0000fb
:1058ac006c6f0000772900000d0a00000022000038
:1058bc0043220000202000002020000020200000b7
:1058cc0020530000656c000065630000746f0000dd
:1058dc0072200000706f0000736900007469000092
:1058ec006f6e00000d0a000000220000442c000026
:1058fc00232c000023220000202000002053000055
:10590c0065740000206d00006f7400006f72000061
:10591c00207300007065000065640000206c0000be
:10592c0065660000742c0000726900006768000056
:10593c00740d00000a000000224500002220000027
:10594c0020200000202000002020000047650000df
:10595c00742000006d6f0000746f00007220000056
:10596c007370000065650000642000006c65000029
:10597c00667400002c7200006967000068740000f7
:10598c000d0a000000220000472200002020000029
:10599c0020200000202000002049000052200000a0
:1059ac007265000063650000697600006572000096
:1059bc000d0a0000002200004822000020200000f8
:1059cc00202000002020000020480000656c000012
:1059dc00700d00000a000000224b00002220000085
:1059ec002020000020200000202000004361000047
:1059fc006c69000062720000617400006520000098
:105a0c00707200006f780000696d0000697400000e
:105a1c0079200000736500006e7300006f72000047
:105a2c00730d00000a000000224c00002c23000023
:105a3c002c23000022200000202000004c650000d8
:105a4c00642000006e7500006d620000657200003d
:105a5c002c3000003d6f0000666600002031000015
:105a6c003d6f00006e200000323d0000696e0000aa
:105a7c007665000072730000650d00000a000000de
:105a8c00224d0000222000002020000020200000d9
:105a9c0020200000466c00006f6f00007220000098
:105aac00736500006e7300006f720000730d0000d0
:105abc000a000000224e00002220000020200000de
:105acc002020000020200000507200006f780000a1
:105adc00696d000069740000790d00000a00000077
:105aec00224f000022200000202000002020000077
:105afc00202000004c690000676800007420000042
:105b0c00736500006e7300006f720000730d00006f
:105b1c000a000000225000002c2300002c2300005f
:105b2c00222000002020000053650000742000009b
:105b3c006d6f0000746f000072200000706f000029
:105b4c0073690000746900006f6e0000206c000027
:105b5c0065660000742c0000726900006768000024
:105b6c00740d00000a0000002251000022200000e9
:105b7c0020200000202000002020000047650000ad
:105b8c00742000006d6f0000746f00007220000024
:105b9c00706f000073690000746900006f6e000084
:105bac00206c000065660000742c00007269000017
:105bbc0067680000740d00000a000000225200000b
:105bcc0022200000202000002020000020200000c7
:105bdc00526500007365000074200000652d000004
:105bec0070750000636b00000d0a000000220000bd
:105bfc005322000020200000202000002020000064
:105c0c0020530000746f000070200000652d000010
:105c1c0070750000636b0000206100006e64000072
:105c2c0020740000757200006e2000006f6600008a
:105c3c00662000006c650000647300000d0a000013
:105c4c00002200005522000020200000202000002f
:105c5c00202000002047000065740000206d00002b
:105c6c0069630000726f0000706800006f6e0000c6
:105c7c0065200000616d0000706c0000697400000c
:105c8c0075640000650d00000a000000225600003b
:105c9c0022200000202000002020000020200000f6
:105cac005665000072730000696f00006e200000e2
:105cbc006f6600002053000065720000436f000007
:105ccc006d0d00000a000000692c00002564000026
:105cdc002c250000642c0000256400002c250000fd
:105cec00642c0000256400000d0a0000004a00002e
:105cfc002c250000642c0000256400002c250000dd
:105d0c00642c0000256400002c250000642c00008d
:105d1c00256400000d0000006a0d00000a00000060
:105d2c006b2c0000205300007461000072740000a2
:105d3c00696e000067200000636100006c69000060
:105d4c006272000061740000696f00006e20000038
:105d5c002d200000526500006d6f0000766500007c
:105d6c00206100006e790000206f0000626a000064
:105d7c006563000074200000696e00002073000051
:105d8c00656e0000736f00007273000020720000db
:105d9c00616e0000676500000d0a0000006b0000da
:105dac002c200000436100006c690000627200004e
:105dbc0061740000696f00006e20000066690000cd
:105dcc006e69000073680000656400000d0a000035
:105ddc00004c00002c250000642c00002564000001
:105dec000d0000006c0d00000a0000006d2c00007e
:105dfc00256400002c250000642c000025640000a4
:105e0c002c250000642c0000256400000d0a000005
:105e1c00006e00002c250000642c0000256400009e
:105e2c002c250000642c0000256400002c250000ab
:105e3c00642c0000256400002c250000642c00005c
:105e4c00256400000d0a0000006e00002c250000e7
:105e5c00642c0000256400002c250000642c00003c
:105e6c00256400002c250000642c00002564000033
:105e7c002c250000642c0000256400002c2500005b
:105e8c00642c0000256400000d0a0000006f000067
:105e9c002c250000642c0000256400002c2500003b
:105eac00642c0000256400002c250000642c0000ec
:105ebc00256400002c250000642c000025640000e3
:105ecc000d0a0000006f00002c250000642c00005f
:105edc00256400002c250000642c000025640000c3
:105eec002c250000642c0000256400002c250000eb
:105efc00642c0000256400002c250000642c00009c
:105f0c00256400000d0a0000005000002c25000044
:105f1c00642c0000256400000d000000700d0000d2
:105f2c000a000000712c0000256400002c250000e4
:105f3c00640d00000a000000720d00000a00000051
:105f4c00730d00000a000000542c000025640000b2
:105f5c00007400000d0a0000007400002c250000e5
:105f6c00640d00000a000000742c0000300d0000cd
:105f7c000a000000752c0000256400002c25000090
:105f8c00642c0000256400000d0a0000007600005f
:105f9c002c56000065720000736900006f6e0000e3
:105fac00203100002e3200002e3200002041000073
:105fbc00756700007573000074200000323000001b
:105fcc00303800002047000043740000726f00005e
:105fdc006e690000630d00000a00000048570000c5
:105fec002076000065720000736900006f6e00007f
:105ffc003a200000255800000d0a00000057000050
:10600c002c250000642c0000256400002c250000c9
:10601c00640d0000007700000d0a0000005900001c
:10602c002c250000642c0000256400000d000000ed
:10603c00792c0000256400002c250000640d000064
:10604c000a000000792c0000256400000d0a0000f5
:10605c0000250000643a000020250000640d0000bb
:10606c000a0000007a2c0000436f00006d6d0000e8
:10607c00616e0000642000006e6f00007420000050
:10608c00666f0000756e0000640d00000a000000d1
:10609c00536500006c650000637400006f720000b3
:1060ac00207000006f73000020250000640d0000bc
:1060bc000a0000000c0700000a0a00000d5700003f
:1060cc00454c0000434f00004d450000207400007b
:1060dc006f200000746800006520000070720000e2
:1060ec006f7400006f6300006f6c0000206f000085
:1060fc006e200000652d000050750000636b0000e1
:10610c00204200006c750000657400006f6f000089
:10611c007468000020630000616c0000696200007c
:10612c0072610000746900006f6e0000000a0000cc
:10613c000d500000726500007373000020480000d1
:10614c00202800007265000074750000726e00005b
:10615c0029200000666f00007220000068650000b6
:10616c006c700000000a00000d500000494e000049
:10617c00206300006f640000652000003d200000db
:10618c0025730000004f00002c250000730a00004e
:10619c00000a00000d450000727200006f720000d2
:1061ac00207700007269000074740000696e0000b2
:1061bc0067200000504900004e0000004d2c0000ec
:1061cc00257300000a0000000a0d00004572000053
:1061dc00726f00007220000077720000697400007a
:1061ec00746900006e670000204e0000616d0000b5
:1061fc00650000000a0d0000467200006965000091
:10620c006e6400006c790000206e0000616d00006f
:10621c00652000003d2000002573000000530000a5
:10622c002c250000730a0000006500002d70000092
:10623c00756300006b5f000025730000000a00000e
:10624c000d5200006573000065740000206f0000a3
:10625c006b20000046690000726d00007761000041
:10626c0072650000203d0000202500006400000045
:10627c000a0d0000202200004622000020460000eb
:10628c0061630000746f00007279000020720000de
:10629c006573000065740000000a00000d2000000a
:1062ac00224d00002c4e0000616d000065220000a4
:1062bc00205700007269000074650000204e000039
:1062cc00616d000065200000666f00007220000008
:1062dc0046720000696500006e6400006c79000075
:1062ec00204200006c750000657400006f6f0000a8
:1062fc0074680000206e0000616d000065000000f5
:10630c000a0d0000202200004e2200002052000046
:10631c00656100006420000061630000747500007a
:10632c00616c00002046000072690000656e000080
:10633c00646c000079200000426c00007565000060
:10634c00746f00006f740000682000006e61000024
:10635c006d650000000a00000d200000224f0000b7
:10636c002c230000222000005772000069740000ea
:10637c006520000023200000504900004e20000042
:10638c006e7500006d62000065720000000a00006e
:10639c000d20000022500000222000005265000059
:1063ac0061640000206100006374000075610000ee
:1063bc006c200000504900004e2000006e7500005b
:1063cc006d62000065720000000a00000d200000e4
:1063dc002252000022200000536f0000667400005f
:1063ec0020720000657300006574000020420000fc
:1063fc006c750000657400006f6f0000746800001d
:10640c00206d00006f640000756c000065000000da
:10641c000a0d000020220000532c00002322000053
:10642c0020570000726900007465000020230000f2
:10643c0020500000494e0000206e0000756d0000d9
:10644c006265000072200000616e00006420000094
:10645c00736100006d65000020740000696d000020
:10646c0065200000652d000070750000636b000056
:10647c005f230000000a00000d7a00002c4300008e
:10648c006f6d00006d6100006e640000206e0000f6
:10649c006f740000206600006f7500006e640000d1
:1064ac00002500006325000063250000643b00000c
:1064bc00256400003b250000646d0000000c00000a
:1064cc00075300007461000072740000696e0000d4
:1064dc0067200000636100006c69000062720000bc
:1064ec0061740000696f00006e2000002d20000018
:1064fc00526500006d6f00007665000020610000a1
:10650c006e790000206f0000626a00006563000075
:10651c0074200000696e000020730000656e00009e
:10652c00736f00007273000020720000616e000037
:10653c00676500000d0a000000430000616c00005c
:10654c006962000072610000746900006f6e0000e7
:10655c0020660000696e0000697300006865000029
:10656c00640d00000a0000000c070000002500006c
:10657c0063250000634800000d0a00004143000041
:10658c00434500004c450000524f00004d450000b3
:10659c0054450000520d00000a2500006325000040
:1065ac00633200004b250000346400002c200000f6
:1065bc0025340000642c0000202500003464000009
:1065cc000d0a00000a000000534500004c45000075
:1065dc00435400004f5200000d0a000025630000d8
:1065ec0025630000324b000025320000640d0000d2
:1065fc000a0a000000490000520d00000a250000a4
:10660c0063250000633200004b63000068650000e6
:10661c00636b0000203a0000203000007825000059
:10662c00782c00002061000064640000726500009a
:10663c0073730000203a0000203000007825000021
:10664c00782c0000206400006174000061200000c0
:10665c003a20000030780000257800000d0a000078
:10666c000a000000505200004f580000494d000035
:10667c004954000059200000534500004e530000bf
:10668c004f520000530d00000a2500006325000046
:10669c00633200004b250000346400002c25000000
:1066ac00346400002c250000346400002c2500000c
:1066bc00346400002c250000346400002c250000fc
:1066cc00346400002c250000346400002c250000ec
:1066dc00346400000d0a00000a000000414d000067
:1066ec0042490000454e0000542000004c49000077
:1066fc004748000054200000534500004e53000052
:10670c004f520000530d00000a25000063250000c5
:10671c00633200004b250000346400002c2500007f
:10672c00346400002c250000346400002c2500008b
:10673c00346400002c250000346400002c2500007b
:10674c00346400002c250000346400002c2500006b
:10675c00346400000d0a00000a0000004d490000de
:10676c00435200004f500000484f00004e450000bf
:10677c000d0a00002563000025630000324b000069
:10678c0025340000642c000025340000642c00002b
:10679c0025340000640d00000a0a000000430000cc
:1067ac00414d000045520000410d00000a2500003b
:1067bc0063250000633200004b5200003d250000b1
:1067cc00336400002c200000473d000025330000fe
:1067dc00642c0000204200003d25000033640000c2
:1067ec000d0a00000a0000000c07000057450000cd
:1067fc004c4300004f4d000045200000746f00001a
:10680c002074000068650000205200005332000024
:10681c0033320000202d00002049000032430000dc
:10682c0020740000726100006e7300006c61000047
:10683c00746f0000722000006f6e00002065000075
:10684c002d500000756300006b0d00000a20000045
:10685c003120000062790000746500002070000097
:10686c00726f0000746f0000636f00006c200000fa
:10687c00415300004c2d000045500000464c0000d8
:10688c002032000030300000360d00000a000000fd
:10689c000c070000574500004c4300004f4d000012
:1068ac0045200000746f0000207400006865000033
:1068bc00205200005332000033320000202d000023
:1068cc002049000032430000207400007261000077
:1068dc006e7300006c610000746f00007220000089
:1068ec006f6e0000206500002d50000075630000e5
:1068fc006b0d00000a2000006d7500006c74000028
:10690c0069200000627900007465000020700000ae
:10691c00726f0000746f0000636f00006c20000049
:10692c00415300004c2d000045540000485a000013
:10693c002032000030300000370d00000a0000004b
:10694c00256400002c200000256400002c20000091
:10695c00256400000d0a000000430000616c00007b
:10696c006962000072610000746900006f6e0000c3
:10697c0020760000616c000075650000733a000021
:10698c0020250000642c000020250000642c000051
:10699c0020250000640d00000a0000004672000073
:1069ac006565000020660000616c00006c3a000018
:1069bc00202500006c6400002c200000282500001d
:1069cc00642c000020250000642c00002025000011
:1069dc0064290000202d00003e2000002825000026
:1069ec006c640000290d00000a00000053680000d0
:1069fc006f6300006b3a0000202500006c640000ff
:106a0c002c20000028250000642c0000202500000c
:106a1c00642c00002025000064290000202d0000bb
:106a2c003e200000282500006c640000290d0000a9
:106a3c000a000000287800003d250000642c0000ae
:106a4c00207900003d25000064290000202d000065
:106a5c003e200000616e0000676c0000653d000088
:106a6c00256600002c2000006c650000643d0000d1
:106a7c00256400000d0a0000000000006c65000099
:106a8c006674000020250000752c000020720000a8
:106a9c00696700006874000020250000752c000058
:106aac00206c0000696700006874000065730000ca
:106abc0074200000257500002c2000006c6900007b
:106acc0067680000745000006f7300002025000000
:106adc00750d00000a000000436100006d200000ed
:106aec006c6900006768000074200000256c0000d1
:106afc00750d00000a0000000a0000000a000000ea
:106b0c00050000000000000000000000fbff00007a
:106b1c00f6ff0000f6ff0000f6ff0000f6ff000095
:106b2c00fbff00000000000000000000050000005a
:106b3c000a0000000a000000256400002c20000060
:106b4c000073000065740000737000006565000040
:106b5c00642000002564000020250000640d000066
:106b6c000a0000007370000069720000616c000084
:106b7c0020250000750d00000a00000025640000af
:106b8c002c20000000200000636100006c690000f4
:106b9c006272000061740000696f00006e200000da
:106bac00646f00006e6500000d0a0000000000001c
:020000040000fa
:106bbc0006000000260000001f000000120000006c
:106bcc0027000000180000001c0000002d00000031
:106bdc0041000000fd000000e50000003201000053
:106bec008b0200001e0200004400000024ff000085
:106bfc00b8fe0000bdfe00003dff000027ff0000b6
:106c0c003dfe000026fe00009efc0000dcf90000aa
:106c1c003bfe0000c908000044100000d60e000026
:106c2c009405000033fb00005ff600008ff70000b6
:106c3c008afa00008afb0000a3fa0000a1fb000006
:106c4c0021010000e7080000a60d00001a0c00004e
:106c5c00bb03000046fb0000a9f80000d3f90000bc
:106c6c0037fd00004aff00005afe0000c3fd000083
:106c7c00d6ff0000f90300002c060000d80100002c
:106c8c00d0f8000029f80000cf030000ff0f00002f
:106c9c007f110000d406000014f9000088f20000f7
:106cac00ddf5000006fd00007a0000009ffd0000ed
:106cbc0059fa000033fd000016060000d30d000049
:106ccc00b20d0000ec04000025f9000007f50000ef
:106cdc009bf8000020ff00001503000000010000dd
:106cec00adfd0000e6fd0000a70200002707000034
:106cfc008703000013f7000027f100003dfd0000a2
:106d0c00bd100000b41900009e100000f7fd00003b
:106d1c00c3f00000d8f000003ff900003bff00007a
:106d2c00b2fc000016f7000030f80000c6010000ad
:106d3c00a20d0000211300003a0d0000a501000077
:106d4c00acf8000082f5000006f9000051fd0000cf
:106d5c0048fd000002fb0000f7fa0000c9ff00002c
:106d6c00d70600002e0700001afd00004bf60000ad
:106d7c002dff0000980f0000d21600009b0d0000a4
:106d8c00a4fb000013ef0000a5ef00005ff800006b
:106d9c0010ff00009efd000076f900007dfa000057
:106dac0021010000390b0000b1120000501000004e
:106dbc001006000049fa0000bbf20000edf30000e1
:106dcc0083f9000095fc000066fc0000c6fb000087
:106ddc0015ff00003005000078040000befc000028
:106dec0022fb00003006000051130000be1300000f
:106dfc00bf050000a0f40000beec0000cbf00000ca
:106e0c003bf9000017fd00004ffa000009f90000e3
:106e1c007cfc00008e030000790d0000db120000ea
:106e2c00470e0000c7010000c8f40000b1ef0000dd
:106e3c00e5f300002cfa000026fc00001dfb00000e
:106e4c00d7fa00005e00000017060000d401000015
:106e5c0011fa0000f6fc0000120c000036170000be
:106e6c009511000010ff000067ee0000e5ea00003d
:106e7c005ef200002afb000032fc0000abf80000c0
:106e8c0087f900007bfe0000270800009813000023
:106e9c0000160000000d0000c8fd00004cf00000c2
:106eac0057ed0000c0f30000e1f90000cffb00003b
:106ebc0077fa000065fc00001d0400009806000035
:106ecc00ea00000094fd000044070000b414000028
:106edc008d1400003204000080f0000075e8000002
:106eec0049ee00001df90000defd00009afa0000da
:106efc00f2f9000009fe0000ec0400007a0f00001b
:106f0c007c1500000d1200004c050000ebf4000095
:106f1c00d3eb00000fef000015f70000e4fb0000be
:106f2c00d8fb0000d8fa00008d0100005c070000bf
:106f3c0079050000ef010000450600006b11000010
:106f4c00d1130000d40600006df3000041e90000ed
:106f5c0040ed00005df8000088ff000070fd0000af
:106f6c004bfc00005eff0000fe020000f109000077
:106f7c00dc110000fa1500000a0f0000d5fd00001e
:106f8c0021ee00002aeb0000e7f2000006fb0000f7
:106f9c00a4fd0000dffa000071fe0000980500005f
:106fac00cc0800008a0a0000b80b0000f50e0000a7
:106fbc00d40d0000020300002af400008cec000049
:106fcc009fef000020f8000077ff0000feff00009c
:106fdc0050010000ca030000ee0100001002000086
:106fec00e7090000ab160000bd180000ff08000008
:106ffc00daf20000b5e7000046ed00000df90000e4
:10700c00a0ff00002cfc000085fa000086010000a7
:10701c0060080000780f0000d9120000e810000092
:10702c00ae0a0000bffe0000daf2000031ee0000f4
:10703c0047f2000040f8000091fd0000f3fe000054
:10704c00c802000089080000940500002800000018
:10705c00bf0100003a0f0000181a0000db110000fd
:10706c000cfb00008ee800002ae800005ff4000032
:10707c00deff00009bff0000bcfa000037fe0000a2
:10708c00fe030000eb0a0000d31000003c130000cc
:10709c00ea1000000c05000059f5000042ec00005d
:1070ac000fef000001f60000c1fb000026fc000001
:1070bc00d9fd000011060000b908000011080000fd
:1070cc0034070000850a000086100000630c0000e5
:1070dc00c9fc00000aed0000cee90000bef1000082
:1070ec00fdfc0000530100005cff000001020000e9
:1070fc00af02000067020000190700002d0f00000e
:10710c00e31500001c0f000057fc0000eceb000026
:10711c00c0e9000065f2000030fb00001dfd00001e
:10712c0016fa0000c4ff00004f07000038090000e9
:10713c00070b0000a90b0000e90d0000950b0000e7
:10714c0065ff0000ebf00000ffea000058ef0000c4
:10715c00c1f7000087fe0000b8fe00005d020000d1
:10716c00b70600000a040000f702000059060000f0
:10717c00ca0f0000251400003c0800002ff400008a
:10718c0050e80000d7eb0000a7f60000a7fe0000b7
:10719c0024fd000006fc0000230300002306000071
:1071ac00430700009d090000110e0000b6110000fd
:1071bc004c09000040f800004deb000001eb000012
:1071cc00c6f2000032fb000078fd000085fd0000d7
:1071dc00d4040000ff07000041070000cf080000a6
:1071ec000e0b0000f60e00007a0a0000b5fb000042
:1071fc00d3ed0000e9ea0000fff1000027fb0000de
:10720c0001000000b6fe00002d030000080700007e
:10721c0058030000dc020000870700005f1100002b
:10722c001014000081060000f5f20000ade800002b
:10723c00eeec00008bf70000f8fe000096fd00005d
:10724c00f4fd0000c7050000d1070000e2070000b4
:10725c0046090000900c000027100000c108000037
:10726c0011f900009eec0000d1eb0000c4f300000b
:10727c0047fd0000d1000000d4ff000030050000e5
:10728c001807000097040000a605000089080000fc
:10729c00ab0e0000810e00005902000019f3000033
:1072ac0026ec00008ff00000f5f9000082000000d1
:1072bc00fefe0000deff00003c0500001a0400008a
:1072cc002c030000bf060000330e000089130000e1
:1072dc00fb0b0000cffa0000e0ec000072eb0000aa
:1072ec00c3f3000016fd00008dff00005ffd0000e1
:1072fc00af020000d60700002f060000e6050000d4
:10730c0039080000e00c0000640d0000da030000f6
:10731c00daf50000dfed0000b3f0000038f90000f2
:10732c001d000000fffe00002afd000041020000cd
:10733c009d0300000a030000eb060000b70b0000e1
:10734c001f0f0000fb0b000066ff0000baf20000ec
:10735c0083ef00006cf40000c2fa0000a5fc0000f2
:10736c007bf900003bfc00008a050000960600003b
:10737c00c403000037060000310c00006d10000043
:10738c00c00a0000b8fb000080ef000016ee000001
:10739c00e0f4000092fb00004cfc0000f1f800004f
:1073ac00b2fd0000c50700004c0700000a030000f6
:1073bc0077040000540b00007d100000cc09000085
:1073cc00cbfa0000f9ef000099ef00001df6000069
:1073dc0040fb000068fa00005af700008afd00002c
:1073ec002e0800005808000017040000b10400002b
:1073fc00440a0000750e0000220900002dfc00005c
:10740c0072f10000e1ef00005bf50000ccfa000027
:10741c00a4fb00007df90000e6fe0000d907000087
:10742c00e50600005602000080030000c9090000b8
:10743c00f30d0000dc09000001ff000081f50000e5
:10744c000df2000028f40000a3f80000ccfa0000b4
:10745c00b5f90000aefd000075060000e606000060
:10746c0065010000c50100003d0a00003d1100004f
:10747c00bd0e0000e901000093f4000077ef00005e
:10748c0062f200005ef8000069fa0000f9f80000f2
:10749c00ccfb00002d070000240d00008806000026
:1074ac001b010000a7030000ba0800001d0c00001f
:1074bc00650700009bfb00005ef20000def00000a0
:1074cc0054f7000074fe000031ff000046fb000082
:1074dc006afe0000c0040000ec02000087ff000000
:1074ec0082040000090e0000aa120000530e0000d6
:1074fc00a5000000e8f3000011ef0000e6f1000029
:10750c00a7f7000032fa000003fa0000a0fe00000a
:10751c00450a0000f90c0000de02000024fd00000a
:10752c0040040000490e0000da1000006e08000054
:10753c00f7f90000d3f00000a0f00000f5f6000011
:10754c00dafc000072fd0000c0fb000054010000da
:10755c00c50a0000180800004afe000030fd0000bb
:10756c0026070000de1000009d1100002907000016
:10757c00a1f800007bf0000003f20000d2f800003c
:10758c00c1fb0000faf90000f6f900007f040000ce
:10759c00cb0e0000f6080000b9fd000063fe0000f1
:1075ac00ec080000f40e0000510c00007402000006
:1075bc00cef70000d6f200000bf5000088fa0000b0
:1075cc00c6fb0000bbf9000037fa000029050000db
:1075dc001a0e000084050000f1f9000087fd000080
:1075ec00c30c00001e150000580f00000d00000019
:1075fc00d0f2000083ef000057f40000c2fa000044
:10760c0009fb000091f80000e6fa0000e507000015
:10761c0037110000e205000067f60000eef80000ec
:10762c00740b00009a170000b6110000ecff00006c
:10763c0001f10000d2ee00004af500006efb0000e4
:10764c00fff9000037f6000076f900006c08000026
:10765c0045140000eb08000002f50000aaf300003e
:10766c0002070000d91600003a130000f8010000d0
:10767c00baf20000dcf00000c8f70000edfc0000de
:10768c00f1f90000e2f3000013f5000052030000d2
:10769c00e1120000550c00006af700001ff2000018
:1076ac00180500005819000054180000b004000020
:1076bc0047f0000036eb0000f0f30000bdfd0000c9
:1076cc003bfe00006ff600008bf300005afe00003a
:1076dc00171200006d140000b0fd000037ec000024
:1076ec0004f7000036110000ac1b00007d0f0000f9
:1076fc0005fa0000dced0000a2f200000afd00001b
:10770c00b3ff000072f600000dee0000fcf3000069
:10771c002f090000601a0000750d0000e5f1000053
:10772c00c6eb0000d1030000491c0000ba19000090
:10773c003403000013ef00003fee000020fb0000bc
:10774c002d03000042fc000031ee00006eec000046
:10775c006cfd000099160000e01a00009cfe000071
:10776c0031e5000013ee0000bd100000e224000023
:10777c009b160000d5f9000006ea000096f1000007
:10778c00290100005e030000dbf4000075e7000037
:10779c00b6ee0000be070000881e0000ce160000ea
:1077ac0016f300004ddf000070f40000e01a00003a
:1077bc0031260000b50d000023f00000d2ea0000d5
:1077cc00cffc0000ed0a0000ac0100009cea0000b8
:1077dc0069e00000dcf10000bf0f00006920000030
:1077ec002f100000afea0000cfdc0000fdf9000014
:1077fc0019230000402b00007d0c0000afea0000b4
:10780c00f3e80000210200002011000091000000ac
:10781c00bae20000edd9000022f40000401800008c
:10782c0038250000220e0000e2e5000034d90000eb
:10783c003bf900000a2500008c2d00008a0d000089
:10784c008aeb000082eb0000da050000f812000061
:10785c00e7fe000075df00004fd800008cf400003c
:10786c007d180000ae220000420d00004ce9000023
:10787c0097db00001ff7000094200000f22c0000a2
:10788c003112000044f0000072eb00003a030000db
:10789c005b130000e902000015e30000c8d80000eb
:1078ac00b9f1000099150000611f0000e00a00000a
:1078bc0086ef00008ce2000050ee00007f0a000012
:1078cc0093200000261f00008d0c000032fe0000eb
:1078dc0097000000bc070000afff0000f0e80000bc
:1078ec001cda0000b2e5000039030000e6170000c6
:1078fc001a140000f803000004f5000015ef000056
:10790c0087f90000760d00008b1800004d11000067
:10791c00bc0100006dfc0000110600004c0c0000c6
:10792c00acff000061e900000fe000008ced0000ee
:10793c0045050000c71100005b0c000090ff000023
:10794c0042f300005cef000073fc0000a910000083
:10795c00f9190000c01300008c080000d6040000c8
:10796c00f40500001b00000070f000003de2000078
:10797c0057e4000095f60000260a00002d100000c8
:10798c00550900000501000046f80000acf20000ab
:10799c0099f900007b0b0000511900001016000033
:1079ac003008000031000000b7020000090300009d
:1079bc00cbf7000005e90000e9e4000043f100000a
:1079cc0051040000d60d0000fd090000b3fd0000bd
:1079dc0030f10000d0f200002106000096180000e3
:1079ec00d7170000c8070000b6fb0000cc00000051
:1079fc00de0b000089080000def4000081e40000ca
:107a0c00a5e9000032fd0000140a0000f605000094
:107a1c002efb000080f80000b7fa00008afa000084
:107a2c00f8fc000077080000d2130000dd11000004
:107a3c00d9060000750100002f070000070b00009d
:107a4c004b0100004af0000098e800007cf10000b7
:107a5c00e2fe000049020000cafc000017fb000017
:107a6c007b0100000e03000058f800009cf10000a0
:107a7c00c5000000ed170000e31a0000240a000006
:107a8c005cfb0000c3fc000052080000440b00002b
:107a9c00d8fd0000d5ec000022ea000063f70000de
:107aac0019060000f50600008bfc000048f50000ec
:107abc00fef50000faf900007aff000075090000dd
:107acc00de1200008211000097060000f3ff000098
:107adc0041020000d902000036fb000055f2000004
:107aec00c9f200000afe0000ed080000d6070000f5
:107afc00dbfd000056f3000057f0000071fa0000a7
:107b0c00c40900004f0e00000e0600007aff0000b2
:107b1c009a030000970b0000d609000011fb00002f
:107b2c00e8ec00000bee0000f4fb00002d09000057
:107b3c00c80b0000fa0500006aff000026f80000e0
:107b4c0065f20000dcf70000b906000046120000e8
:107b5c00f91100005d090000b9030000de0200000d
:107b6c00befe000081f30000c2e70000a7e70000a2
:107b7c0080f6000001090000f60f0000230a000047
:107b8c00a101000075f80000e9f20000edf9000019
:107b9c00c60b00006a190000e4150000f70700008e
:107bac002b000000c6020000f20200008ff700005c
:107bbc00d8e80000fde400008ef100009104000004
:107bcc00de0d0000da09000078fd000012f1000063
:107bdc0000f3000080060000be180000ab17000088
:107bec0082070000a2fb0000ff000000f40b000065
:107bfc005808000086f400005fe40000e7e900008c
:107c0c007dfd0000250a0000d10500000cfb0000e2
:107c1c0089f80000bafa000085fa000017fd000090
:107c2c00b0080000e8130000b8110000ae06000018
:107c3c007a0100004e070000000b00000801000054
:107c4c000cf00000a2e80000adf100002dff0000d8
:107c5c00ea020000eafc0000dcf90000b9ff0000b9
:107c6c004f0200007df90000d8f300002d02000047
:107c7c00f016000018180000a50800005dfd0000bb
:107c8c004b000000730900003e09000069fc000075
:107c9c0083ef000051ef00002ef90000bf00000040
:107cac000cfe00001ef70000dff700008afe00004b
:107cbc0023ff0000cff900009bfd00007e0c0000ac
:107ccc00851400008e0b000051ff0000a1fe000087
:107cdc00650500002b0900005c05000036fd000066
:107cec001df9000022fb000029fc0000d2f7000067
:107cfc00b1f10000caf1000066fb0000dd040000d9
:107d0c00c8000000ddf60000b8fc0000af0e00005b
:107d1c000a1400007805000041f3000054f4000040
:107d2c00320a0000a6190000e310000047fd000015
:107d3c005ff60000bfff0000880600001ffb00007c
:107d4c00a3e7000009e300008cf50000980b00008d
:107d5c006c0d00000bfe000086f2000024f8000001
:107d6c00520900006d100000ce00000089f20000e6
:107d7c0028fa0000010e00004419000089100000d0
:107d8c006601000079fe00004d0500008d05000025
:107d9c000ef90000a9e9000072e60000c6f300002d
:107dac007103000056070000b000000032f900001b
:107dbc0095fa000090010000130800008c050000eb
:107dcc0090fa000029f7000027000000680f00005f
:107ddc004c150000100e00004e0400009400000032
:107dec00e1040000f0070000670000000af1000049
:107dfc00c7e8000091ef0000d1fc0000f002000089
:107e0c00a5fe000037f900004bfa000055ff0000fa
:107e1c00fe0100005c03000061020000ccff0000ca
:107e2c00090000005c0300000d080000860900003a
:107e3c00e0080000bb0500006a0200000704000017
:107e4c00de060000740400005afe0000bcf90000bd
:107e5c0025f800008af70000dbf5000059f400005b
:107e6c001cfa0000420500001e06000005f9000087
:107e7c0044f0000025fd0000e30c00005a0a00004d
:107e8c00c7f80000d5f40000700800009111000044
:107e9c0038060000f6fc0000d9000000570800006e
:107eac000c0a0000c90500002103000003040000b7
:107ebc004102000030fd000041f90000d2f5000045
:107ecc0028f4000095f8000073fb000087fa00000e
:107edc0019fa00003ffb00000fff00005f030000d9
:107eec00d006000036020000c1f700004dfa000079
:107efc007f0800000f0c0000ab020000ee00000039
:107f0c00510a0000c90d0000b3080000c1010000b7
:107f1c00eefe00004e00000054ff0000fcfb0000d1
:107f2c0055fc00005f0000004aff000035fa00001d
:107f3c00f7f60000f8f7000060fc0000e5fc00001c
:107f4c00c9fd00003400000038f9000030f70000d3
:107f5c00ca00000098030000ea050000b509000003
:107f6c00910000005dfb00004e060000cd0d0000ee
:107f7c004e060000f7fa000082f900007b020000b8
:107f8c007209000004040000b7fc0000f4ff0000bc
:107f9c00790500002d010000e4f8000004f9000050
:107fac000fff000067ff000097fa00009df900002a
:107fbc0021fc0000aefd0000a9ff0000c80100007c
:107fcc0041ff0000fafb000000fd0000f8ff00007c
:107fdc00f40300007b040000c3ff00001302000048
:107fec002a0800000f0800003e0700008001000076
:107ffc0077fb000057000000f00400005bfd000060
:10800c000cf80000aafe00000d02000031fe00007a
:10801c00dbf90000d0f90000c0fd0000b9fe000043
:10802c00bcfe000084fe000005f900004bfa0000c5
:10803c00ac020000d2020000700400004d080000e9
:10804c00ed000000b9fc000075050000ac0b000051
:10805c00f6040000e0f9000004f80000f001000054
:10806c0036090000f5010000e1f9000093ff000063
:10807c007d070000f50100003bf800002afc000021
:10808c009d050000e00100004ff9000078f90000a8
:10809c00fafd000029ff00000100000095ff000020
:1080ac00eaf70000b5f80000930300003e0300005f
:1080bc0094fd000039fd0000dbfd000020030000f2
:1080cc00950300002f010000100700009300000032
:1080dc00daf50000b2020000fd0e000020fd0000e9
:1080ec0022ef000023fd0000ee090000ab070000aa
:1080fc004900000026fd0000600000005e03000047
:10810c0031ff0000defb000065000000ff000000f6
:10811c005bfe000097fe00001bff00000a01000040
:10812c00470000006cfb0000c0fb0000d900000001
:10813c00eb010000cffe0000d2fd0000e1020000c8
:10814c0093030000affd00006cfa000050ff00002c
:10815c008306000074020000eefd0000ccff00005e
:10816c008e0000004101000033ff0000c8fb00003e
:10817c0069010000ab0600009efe00003dfc000003
:10818c0048060000190a000026fe00004af4000010
:10819c00e1fd0000230b0000a6030000b0f5000079
:1081ac001ffd0000100700006e03000058ff0000c8
:1081bc0020ff000017fe0000170000002c05000037
:1081cc003504000088ff000016fd000063fe00006f
:1081dc00ac0100003c0000001efe00005dff000032
:1081ec006d000000c10100001b010000ac0000008c
:1081fc006d0200002601000089fe0000fdfe00005b
:10820c0019ff0000bcff0000fc020000260000006b
:10821c0088fc000048010000ae040000670000006c
:10822c00fafd0000d30000009801000017000000c8
:10823c00fcfb0000a0fe0000be0700004103000094
:10824c0077f7000041fb000063070000ff0400000b
:10825c0002fc000067ff00002b0300005000000030
:10826c00fafd00000afe000073010000f700000098
:10827c0016fe0000aefe00005ffd0000f2fc0000e8
:10828c00550300000005000085fe00004afd0000bb
:10829c00b70100000802000067ff00003c0000006e
:1082ac005700000046fd000090fd00005301000047
:1082bc00b402000037fe0000dffc0000a00100004b
:1082cc004e0200008afe00007ffd00001c02000030
:1082dc0090030000d5fc00003efb0000ce01000026
:1082ec005005000097000000e6fa00003efd00007b
:1082fc0027010000610300009203000073ff0000df
:10830c0026fb000065fd0000dd0300007f0400007b
:10831c002dfe000010fc000009000000bdff000055
:10832c0088ff00009fff0000f6ff0000190100000d
:10833c0002000000a9fd00002cfe00002a02000033
:10834c009a0100006efe00002bfe000052ff0000a0
:10835c00abff00007fff000082ff00004400000024
:10836c004101000002010000a6fc000094fd000089
:10837c00e30300000902000091fb0000fef900007d
:10838c0045fd0000fd010000db02000009000000bb
:10839c0058ff000036000000a40100005f0100003f
:1083ac00d8ff0000bffc00002dfc00004cfd0000bd
:1083bc0069fd000015020000ab000000d9fc0000b4
:1083cc0077010000c304000054020000a8fe000066
:1083dc004cfc0000e2fc00009d0000001a000000b4
:1083ec0053fe0000aa000000f300000095010000fd
:1083fc00ae0100004bfc00004bfc00000003000031
:10840c00ae010000e5fe0000e5fe000030fc0000bf
:10841c00e9fe0000c50300003b010000dbfb00008f
:10842c0098fc00005202000042040000a9ff00006a
:10843c00c7fd00001c0200001402000075fd0000c6
:10844c0024ff000069030000d700000075fc000049
:10845c0057fd000078ff0000ea0000003402000025
:10846c00dc000000020000004e000000d100000003
:10847c0036010000c4fe000062fd000024fe000076
:10848c00be00000017030000380200001d000000b1
:10849c001dfd0000b3fe0000520200007701000039
:1084ac0081fe0000b3fe000054020000b90200007f
:1084bc004bff0000c8fd00004d0100006e030000e2
:1084cc002dff00007ffc0000f5fe000064010000a1
:1084dc007300000066ff0000a30100007d02000095
:1084ec0006ff00003bfd000048020000b80300003e
:1084fc00c7fd00000cfc00006ffe0000aefe00008b
:10850c001afe000005ff00003b00000043020000c3
:10851c003d030000520200005e020000d701000083
:10852c001f00000092fe0000a8fe000064fe000088
:10853c002afd0000f9fe0000ef00000078ff0000ab
:10854c00fbfe000048010000f30100005400000095
:10855c009c00000072000000bafd000099ff0000b2
:10856c009f020000b3000000fcfd000058ff00005b
:10857c006601000097fe000011fd0000ddff000009
:10858c005302000036000000fcfc00004500000017
:10859c009a0400006f020000ecfd000030fd0000aa
:1085ac00790100008a02000041fd000071fd00000d
:1085bc00b4020000110200002dfe000073fe00004a
:1085cc00f90100006c0200001aff0000e7ff000038
:1085dc001c02000054ff000099fd0000380100004f
:1085ec005c02000009fe0000ccfc000073010000de
:1085fc00c40300009eff00006dfd0000e7010000b9
:10860c00dd030000dcfc00009cf90000d30000003e
:10861c005c0400002fff0000b1fd000034030000db
:10862c00d2040000a1ff000095fc0000edff00004b
:10863c000a02000033fe000000fc00003c000000b9
:10864c00a5020000e7ff0000befe000039ff00009d
:10865c003aff000000010000890100005bff0000f0
:10866c001aff000072000000e5000000c8ff0000c7
:10867c0086fe000023ff00005d000000f6ff0000f6
:10868c00a0fe0000c9ff0000f50000000e01000074
:10869c00ed00000012ff0000e5fe00004f0000009e
:1086ac00410000007e0000007500000033fe000059
:1086bc0091fe00005d0000004cff0000abfe0000ce
:1086cc0066000000210100007cff00005400000047
:1086dc0004020000b200000097fe00000cfe000037
:1086ec00ccff000097ff000026fe000045ff0000b5
:1086fc00ba00000076ff0000effd0000f80100005a
:10870c0077040000f4ff0000ddfd0000b80000005d
:10871c004b02000098ff0000d9fc000093fe000003
:10872c00540000009dff00001bfe00001aff00001b
:10873c006c0200006d0200002b00000051ff0000d5
:10874c0082000000a600000010fe000034fe0000b5
:10875c008c00000042ff0000e1fd0000faff000069
:10876c007d01000083000000a8fe000005ff000052
:10877c00340100001a0100007aff000037ff0000ee
:10878c0075000000f200000004ff0000b7fd0000bf
:10879c006eff00009f00000040000000c4ff0000be
:1087ac00e5fe000047000000280200000a0000005f
:1087bc00ecfd0000a6ff0000890100006100000034
:1087cc0037ff000096ff00002d0000004300000062
:1087dc00daff00000e000000fbff00007cff000031
:1087ec002800000033010000f4000000a8ff000086
:1087fc003fff00005f0000008700000080ff0000ca
:10880c007aff0000de0000001901000091ff00005b
:10881c00defe0000a4ff0000840000001f0000002a
:10882c0017ff0000d7ff0000f4010000b3010000a7
:10883c0054ff00001d000000670200006f010000e3
:10884c004fff0000fafe0000180100003202000089
:10885c008dff00000cfe0000af000000ea010000dc
:10886c006dff000021fe00007800000057020000a0
:10887c007a000000a3fe0000720000009c020000c1
:10888c000b0100001dff00009b00000047020000d0
:10889c0089000000c4fe000059000000b90100006e
:1088ac00ac00000004ff00000100000035020000d5
:1088bc000b010000e5fe000054000000b2010000b6
:1088cc0022000000f5fe000098ff000016010000d9
:1088dc000f0000007cfe000065000000eb010000b2
:1088ec000f000000c9fe000064000000010200003f
:1088fc000301000097fe000046ff00009d010000f0
:10890c00d2000000f5fe000052ff00000e01000036
:10891c0056010000f2fe00004afe0000e3000000d9
:10892c00080100008cfe000087fe00004e000000d5
:10893c007b0000003cff0000dafe00007e0000001f
:10894c003201000052ff000006ff0000c7000000cb
:10895c00f9000000a5ff00001eff00000f00000042
:10896c00b0000000120000002dff0000ceff000040
:10897c00060100007d00000069ff0000f0ff000010
:10898c00b3000000490000005fff000021ff000061
:10899c00550000006200000035ff0000caff000017
:1089ac00ed0000004800000075ff000015000000fd
:1089bc0015010000ce00000043ff000075ff000011
:1089cc00fe0000009200000079ff0000acff0000e8
:1089dc00af000000e800000058ff0000ccfe0000d3
:1089ec0099000000b6000000d0fe0000ecfe000074
:1089fc0030000000f6ff000019ff000019ff000016
:108a0c005f0000009e000000e7fe000026ff000053
:108a1c00c60000005d00000052ff000058ff00007f
:108a2c00e3ff00001b000000bbff00004bff000039
:108a3c00a5ff0000340000001b000000ceff00006a
:108a4c0096ff0000e2ff000078000000bcff000071
:108a5c00a5fe000092ff0000cb000000fdff00000f
:108a6c00fefe0000b6ff0000a80000005d00000044
:108a7c0090ff0000a1ff00009600000079000000ac
:108a8c00c1ff0000d8ff00003f000000ac00000058
:108a9c0054000000baff000022000000cb000000d0
:108aac000f0000007eff000061000000820000004b
:108abc00fbff0000d5ff0000eaff00003b000000b8
:108acc00f3ff000081ff00003c000000af0000003d
:108adc002b0000000c000000530000007d00000083
:108aec0018000000b7ff0000150000005400000043
:108afc00d0ff0000a0ff0000440000007500000043
:108b0c0016000000dbff00003d000000be0000006e
:108b1c005d000000ceff0000ceff00005a000000f8
:108b2c0091000000f0ff000075ff0000dfff000067
:108b3c005b000000070000009bff0000daff000054
:108b4c005a00000037000000d3ff0000f3ff0000c4
:108b5c001d0000002c0000000c000000d9ff0000dc
:108b6c00050000004500000051000000030000005b
:108b7c00100000006a000000610000001f000000ef
:108b8c00deff00001b00000051000000efff0000a2
:108b9c00d1ff00003e0000005c000000fdff000063
:108bac00d5ff0000380000006d0000002000000020
:108bbc00dbff00000900000007000000cfff0000f1
:108bcc00e9ff0000feff000012000000ffff0000a4
:108bdc00deff0000080000001a000000ecff00009f
:108bec00fbff00005400000047000000e6ff0000ff
:108bfc00e1ff00004a00000059000000e6ff000001
:108c0c00caff00004e00000080000000f9ff0000c9
:108c1c00e1ff0000430000005600000002000000cd
:108c2c00bfff00000f0000003e000000f9ff000035
:108c3c00caff0000f3ff00002c000000040000003d
:108c4c00d5ff0000e8ff0000150000002000000028
:108c5c00e5ff0000d2ff000005000000110000003d
:108c6c00dfff0000c7ff0000efff00000c0000005a
:108c7c00e1ff0000c3ff0000eeff00000400000055
:108c8c00d8ff0000c9ff0000e5ff0000feff000058
:108c9c00e5ff0000c5ff0000dcff0000eeff000058
:108cac00deff0000d0ff0000d8ff0000e8ff00004e
:108cbc0002000000edff0000daff0000d8ff00000a
:108ccc00a4ff000095ff0000b4ff0000b3ff0000fc
:108cdc00c1ff000093ff0000cfff000063ff000006
:108cec0065ff000032000000b50100005e010000cd
:108cfc0034fc000051fb000024040000e3020000df
:108d0c0002f9000019030000d0f6000010fa000070
:108d1c0083120000e9fb0000b8fa00006d050000aa
:108d2c0000f50000d201000046170000470a0000c1
:108d3c0008dd0000d4f50000151f000086ef0000d0
:108d4c0092f80000b00d00002cf60000f9030000b2
:108d5c007804000040090000b1f80000b3e90000fd
:108d6c0094140000c207000081eb000069010000b0
:108d7c0066130000a8fc0000e8f700004b07000099
:108d8c0016f400000dfa0000c30c00002afa0000d3
:108d9c00fdfd00005c0200004d0300005a010000c4
:108dac0059f90000ca000000c4ff00002a000000ae
:108dbc00990100007e050000e6fe00001f16000071
:108dcc00da0a0000fed10000e80900006d1800006e
:108ddc006fe100009ffe0000990e0000fafd0000fc
:108dec00890500008df3000038ef0000111e000013
:108dfc00990800009df40000860c0000240a000075
:108e0c00170d000064fa00003dee000012f20000a5
:108e1c0036030000600b00002bf60000d7030000a7
:108e2c00b90a00000f010000cffe000051fc000049
:108e3c00bcfe00000bfa0000f5010000a0070000ca
:108e4c00c4f30000990500005a0c0000cdf7000097
:108e5c0081120000800000000ae00000de0000002b
:108e6c004909000054f90000c3ff00004cff00004a
:108e7c00690a0000a20c00002df2000089fb000022
:108e8c00600a0000420100006efb0000720200004c
:108e9c00ba2000001e1b0000c2cc0000c5e200007e
:108eac0023200000a4ef0000bbf40000ba0d00006a
:108ebc00a6010000bbf9000057f400006307000096
:108ecc00af0e0000e70700007cfb0000fd05000072
:108edc00c213000027090000d3fe00003eeb000087
:108eec0036f00000b80400000500000044fa000051
:108efc00210100007f010000a4fc000005f200002d
:108f0c0084010000671d000074020000c8f100001d
:108f1c00bf010000aafd0000c7fb00000a01000011
:108f2c0027060000b10a0000f4f7000076f20000fa
:108f3c004bff000028f90000dffa000019fd0000cb
:108f4c00fbfe0000ca04000024fa000070040000bc
:108f5c0089060000f201000008110000e0f5000095
:108f6c00b5ff00000e1b0000f0fc000023f9000010
:108f7c00cdf700006dec00008dfc000050030000ec
:108f8c00dbf90000e5fd0000fa04000036f90000f2
:108f9c0080010000850a0000fdfc0000fb080000b9
:108fac000a07000066f5000061ff0000b101000037
:108fbc006efb00005d0a000033020000d8f20000d6
:108fcc008e000000f0f8000083f40000dd040000c7
:108fdc00cc000000a2f70000600400005404000064
:108fec00f2f70000b6030000b60900009ffd000078
:108ffc00f1fd0000b70d00004c0e0000b40c000099
:10900c004ef400001adf00009afc0000e7fd00009f
:10901c0031f80000f20a00009b02000038eb00005f
:10902c00a90000008b0f0000c4fd0000310e0000f1
:10903c00cd1d0000e0fe0000af0300006a0d000033
:10904c0079e50000e9ee00005104000040f3000057
:10905c0052f900007309000047fc00002cf90000d5
:10906c0035f80000110d00003113000022fd000046
:10907c0024080000c3fb000056fa00005405000051
:10908c007a010000120000006ffb0000d2fc00000f
:10909c005df70000cdf800002cff0000f5fe00008d
:1090ac008bfb000042fc0000c9fb00007f0b0000a2
:1090bc009e12000031fa00006dff0000df0a000074
:1090cc00ad000000470400008e0f0000bff200004e
:1090dc0024ef00004efd000057ed00006804000076
:1090ec0084070000a8fa00009e1000005f05000035
:1090fc0031f20000ae0300002e050000b0fb0000b2
:10910c00a6fd0000a7010000820d0000120b00005c
:10911c0018f70000d6f9000027fd0000d7f7000073
:10912c0075f900003502000074fe000075f40000b3
:10913c00bd0d00006f01000010fc0000f90b0000d9
:10914c009c03000088170000edfc00004e1100008d
:10915c00d60400003ed300000206000091ec000093
:10916c00fbf500007b0c0000e1f60000f5030000ad
:10917c0058f100002e0c0000a327000005fc000095
:10918c00c5f10000ba1600003107000086f400009b
:10919c00610b000084df0000ffec00009b0c000062
:1091ac000afc00003c040000d9020000a8ff0000eb
:1091bc008cf50000ed100000e20c0000bdee00008c
:1091cc0017f400008afe000069060000da090000ae
:1091dc0044080000180a00002ff5000001e100000f
:1091ec00d9060000b8fe0000cdf60000e9fe000034
:1091fc00fdf9000071090000f8f30000fd140000f7
:10920c00991b00005eee0000080c000093080000a3
:10921c000ff60000c70100008bf9000020f70000da
:10922c0022fd00006bfb000057f600000306000057
:10923c00540d0000b6fa0000a8f80000bffe0000b4
:10924c0078fd000084080000f102000013f9000012
:10925c0099090000c70800007cfd0000dbfe00003f
:10926c0065fb000035f000004bfc000035080000e9
:10927c00bcf5000012f900007203000004fa0000b3
:10928c007d130000c80700008f0700004319000081
:10929c005ff700009d06000034ef00007af000003c
:1092ac00880b000039e4000043f90000af10000007
:1092bc0067f7000025f300000e0800008d1d00006c
:1092cc00fe060000aff90000f00b0000a0fb000050
:1092dc00470300008401000033ea000001fc000099
:1092ec0018fd000045fd00009a0c0000c9ff0000ad
:1092fc00c0fd000058f900006ffd0000ec0e0000ee
:10930c001200000099fe00002ffb0000a0ff0000df
:10931c006411000028fd00003cf60000bcfd0000bc
:10932c003ff800005ffb000046040000e1fb00007a
:10933c00b4f90000fc0100003ef60000900e0000a5
:10934c00dc17000074fe0000d1060000830b000047
:10935c0056f8000094f8000006fd0000cafb00005f
:10936c0077ff0000ebef0000a7ff000052080000a1
:10937c005dfe00006d07000061fd0000fbff0000ba
:10938c006105000006fd0000c0050000e7090000b3
:10939c001f00000011fb00001eff0000f202000085
:1093ac0040fb00003af300001efd0000b304000077
:1093bc00bef900001306000047010000eaef0000b0
:1093cc005b110000c8090000a8fa0000b9130000e6
:1093dc006b0e0000b6f1000080f20000b903000033
:1093ec0062f600001df60000bb020000bffd00008d
:1093fc0002ff000088f900005df30000ca1b0000aa
:10940c004d1800006ffd0000d70300009f00000006
:10941c00ff00000092ed0000cd070000fbfe0000f5
:10942c00cbdd0000b1120000c00b00007ef5000087
:10943c00880a000087f300001101000047100000ab
:10944c00fdf700008a09000035fe000083f70000dc
:10945c00cc0b0000b0ff000029000000f7ff00005b
:10946c0071f10000c8f40000c6080000fdff000008
:10947c002cfa00004b070000aaf20000250c00009b
:10948c00221b00003cf900007ffe0000e0f400000d
:10949c002000000008140000bbfe0000bcf7000018
:1094ac00d4ef000074f80000b00500003903000090
:1094bc00400600004f0100003afd000024fd0000b2
:1094cc0037fe00005eff000046020000a90100000c
:1094dc009e0100008f0c000044fd000023f50000ed
:1094ec004403000014f70000f5f500004e050000e1
:1094fc0048010000e2f90000f6060000f1fd000052
:10950c000bf900005b14000053fc000031ff00005d
:10951c0011160000d3010000ef01000070ee0000f6
:10952c0089f50000bfff00005bf600009b05000002
:10953c005b00000000fc0000cb000000bcef000052
:10954c0099fd00001e1b0000810700005d0e00004d
:10955c005b0400006cf500003cfa000010f5000004
:10956c00da090000a6f6000098ee00005a08000088
:10957c005f040000160200005e010000f0f0000025
:10958c0021020000100f000050ff0000b2fe00008e
:10959c0054f90000defb0000ba060000560800007b
:1095ac009cf90000bdfc0000bd020000c7f10000ea
:1095bc00acfe0000270200004df8000023fd000067
:1095cc00e0010000ce000000bbff00007a1000009c
:1095dc009707000096fb000074030000d4fc000009
:1095ec004d05000022ff00008df4000099020000e0
:1095fc006df90000f0f70000f0ff000085ff00009f
:10960c0090ff00006402000019fc000033f8000019
:10961c000b1100003c0800009bf80000c40f000078
:10962c00a404000047f5000014fe00005bfa0000e3
:10963c0088ff0000cffd000050f80000b2fb0000d6
:10964c00ea01000049010000fdfe000082fc000060
:10965c00d1f00000920b00005a110000e1fb000059
:10966c00a508000093070000b4f9000071fd00008c
:10967c0077fe000061fb00000cff00007ffb000088
:10968c001dfa00000fff0000370200007aff0000f7
:10969c009ffe0000b80100005efd000045050000c3
:1096ac00a30800000df9000080ff0000ec0600008c
:1096bc00930000006c0400007dfb0000d9f7000053
:1096cc00f3ff000090f80000e40000005f040000cd
:1096dc00bc020000ae060000b6fc000086fd0000d7
:1096ec00bdf8000020020000740b0000c3f700005e
:1096fc000e020000ad0e00006bfe000098fd000095
:10970c00edfa000081f60000ef0400005f0200009b
:10971c0016fc00008301000082fd0000b1fd00007a
:10972c0084070000a3fa000023f80000ea0e0000f2
:10973c0084fe0000f1fa0000020a000011fb000098
:10974c00adf9000088fe0000a7ff0000a6fd000098
:10975c00730300003b0b000022ff0000d50000004b
:10976c00a500000051fe00007e050000a3f60000dd
:10977c001afe0000d10500007df6000031fc00004f
:10978c00e8ff00001dff000020010000b4010000f4
:10979c0064f80000a40000005711000064fd0000f4
:1097ac0051000000a50f0000bcfa000054f90000a5
:1097bc006efd000017fb0000f500000071fa0000c0
:1097cc0026f9000008fe0000310300000aff00002b
:1097dc0012000000edf5000060f7000054150000c9
:1097ec00680600003cfe0000670c0000ad000000a5
:1097fc009df9000069ff000063fc0000cefc000036
:10980c0092fe0000aff90000b3fb00003d01000028
:10981c0014010000ccfd00000a01000036fe00001f
:10982c00c3fd00008d0a00008d0400002ff900001c
:10983c000c0600006f0600006f0100000a03000018
:10984c00f8f5000023fb00004d0000007bfa00003f
:10985c002cfe0000fafe00008f03000068000000e0
:10986c00a2fe000085fd000088fb00005d0b0000df
:10987c00d4070000f0fc00002a0f00002e0a0000a4
:10988c00fdf7000062fb0000c9f900003bfb000083
:10989c0089ff0000ebfa0000defd000076070000f7
:1098ac00c6fc0000e3ff00000d01000059eb0000b6
:1098bc000b0d0000c91700009bfb000023100000db
:1098cc00520800005ff5000073fd00006dfb000006
:1098dc00c0fa000065fd0000b0fe000071fd000044
:1098ec00a101000058030000dcfc0000d6010000c0
:1098fc006afb00001af90000c714000039090000c7
:10990c00a8f60000c5ff0000e3fc0000d501000034
:10991c00d10300006bff00005900000003fa0000a7
:10992c00e8fe000081000000eef6000044ff00009d
:10993c001e030000c60000001afe00007cff0000a1
:10994c005d010000f9fa00007b0a0000d30700005b
:10995c0032fc00002d020000ff010000c5070000d2
:10996c00cafc0000cefc000081fd000050f5000098
:10997c00b0030000d5fc0000cdf80000d5040000b9
:10998c0080020000fafb0000b50000007cfe000025
:10999c007bf00000f1080000301000006e020000a7
:1099ac00760c00006f00000014fb0000f3fb0000bd
:1099bc00e2fa000008fc00001ffd0000b9030000e3
:1099cc00e1fd000087fc0000ddff000002ff00004d
:1099dc00acfb000058ff00006c04000083fa000090
:1099ec003d040000e70b000065f600004bfe000094
:1099fc0070020000c5f80000dc030000b600000097
:109a0c006e010000290300007cfa0000bafa000085
:109a1c0056fd0000cfff0000fefc000081ff00009f
:109a2c004e01000001000000dc000000b8fe000048
:109a3c0014fb0000bcff00006e080000b403000023
:109a4c00f604000002ff000023fa0000ed01000004
:109a5c00d4000000e5000000780000005c0300006a
:109a6c00ccff00009bfb000069fd000031fa0000f8
:109a7c0093fc00009dff0000440300004afe000020
:109a8c00fd000000b2fb0000daf80000da0d000067
:109a9c008006000055010000a60600007c030000b3
:109aac005bfe0000b40300001b0200007ff300000b
:109abc000100000034ff0000c7f8000003020000a2
:109acc0096fc0000f1010000ed030000cdfa00004f
:109adc0030020000a9ff000047f9000086040000d6
:109aec003f060000a5fd00001a080000110600004a
:109afc002bf90000bdff000003fd000087fe0000f5
:109b0c006c030000b8fc0000d40000003100000021
:109b1c004dfc000030000000bdff000063fe0000a3
:109b2c00e5ff000093030000a3fc00002ffc0000e5
:109b3c00ce050000380000004905000007070000b2
:109b4c00b5000000740200002e000000b6000000fa
:109b5c0075fb0000baff00005b050000e00300008d
:109b6c0060fe0000eefb0000c00000003afa0000ae
:109b7c004ffe0000a101000066ff00001d04000064
:109b8c000aff0000fa0000004b000000e6f700009e
:109b9c00000400005d090000e9fc000089000000e1
:109bac00f407000062000000c3030000e40400009e
:109bbc007ef6000042f80000b30100000cfe00002d
:109bcc00fcfd0000e9010000a9fd0000d00300002d
:109bdc0094020000e9f8000021fe000095fe000050
:109bec0030fe000069fe00008a01000043090000fd
:109bfc00bc0200006c000000480600006100000080
:109c0c00fafd0000f6ff0000c9fb0000e8fa0000b6
:109c1c00e8000000fe00000009fd0000ccff000081
:109c2c00ef00000057ff000086000000cdfe000092
:109c3c00b0fc00008dff0000d0fa0000f8fe000020
:109c4c00ae0a0000600300007fff0000400200002d
:109c5c00dffd00007cfd00002c0000006bfc000010
:109c6c00bcfe000066030000940000009bfe000098
:109c7c006dfe00002cff000080fe0000effe0000d7
:109c8c00cfff0000ffff000085ff0000e502000091
:109c9c00b6ff0000fefa0000b500000029fa000033
:109cac0074ff0000830b0000bbfe000043000000ab
:109cbc004e050000b5fb0000eeff0000a1ff000008
:109ccc0084fc00000d010000c0fe000021fe00001d
:109cdc00bd0100008802000002ff00009afe000097
:109cec00540000006afd000024ff00008701000002
:109cfc00b80000003a010000c5fd000001ff0000a3
:109d0c0029fc0000f4f90000130c00008e0a00007e
:109d1c004bfb0000b501000036fd000010f90000ff
:109d2c00b3ff00000bfc0000c2ff0000b6050000f2
:109d3c0026010000a2ff000024030000f4ff000035
:109d4c0076ff0000e7020000e2fd0000aefb000021
:109d5c007800000075020000140000002efe0000c8
:109d6c009cfe0000de00000095ff000007fd0000d7
:109d7c0080ff000025020000d20300000d0100004e
:109d8c00f0ff0000f0ff0000c1ff000075000000b4
:109d9c0099fe000072010000c40100009400000054
:109dac00ed0000006aff0000c60000006c0100001e
:109dbc008afe00006ffd000095ff0000700000009f
:109dcc0068ff0000da000000d701000032ff00003d
:109ddc008dff000001000000d8fe000020ff0000f5
:109dec0090fd00003eff0000830200001402000002
:109dfc00f9ff0000c1fe00008b010000a50000006f
:109e0c00bfff0000e201000001020000500400004e
:109e1c009e00000060fb000043fd00000dff0000f1
:109e2c0022fe000072fe0000080100002d00000060
:109e3c009bff000026000000fafd0000cffe000092
:109e4c00670000008cfe000079fe0000e2ff0000bd
:109e5c0041010000dd0300002f010000740100002f
:109e6c0073050000d5fd0000a1ff000013020000e7
:109e7c00f9fa00008d0000001cff000023fc00001c
:109e8c007600000071ff000050ff0000e9ff0000a9
:109e9c0037ff00002cff000049000000c5fe000049
:109eac006efe000043000000d7ff0000b1ff000071
:109ebc002f0100005f00000048ff0000b2ff00000f
:109ecc00b2ff0000b0000000a7ff0000720100000c
:109edc001a020000f5fe00007b01000030000000bb
:109eec0085fd00004e0100001c000000dffe00009c
:109efc00d3ff0000f4ff000086020000d7fe000034
:109f0c00cefd0000080200006800000092ff000077
:109f1c006bff0000a1000000370100006afe00008a
:109f2c00bd0000004300000056fe0000f9010000d7
:109f3c007c000000fefe0000b6000000d100000016
:109f4c00f0ff00003bfe0000f4fd0000c2ff00002b
:109f5c004e0200004c02000027010000cf00000060
:109f6c0043010000c3ff0000aafe0000c6fe000073
:109f7c002fff0000520100009200000070ff000053
:109f8c0050ff000073ff00000eff0000f2fe000007
:109f9c008c010000a200000050ff000036020000ff
:109fac0070000000f1fd000057ff00000d000000e4
:109fbc0099000000fcff0000bdff0000a70000009e
:109fcc00ebff0000f6fe00007fff0000a1ff000089
:109fdc0003ff0000fbff0000280000002eff000024
:109fec00f3000000cb00000039000000f20100007b
:109ffc009f0000007bff000020010000c901000051
:10a00c00acff000096ff0000e00000001d00000007
:10a01c00f0ff0000030100002101000093ff00008d
:10a02c0093ff0000c8000000ed000000d0ff00000e
:10a03c0066ff0000fcff00000a010000ce010000da
:10a04c0059ff00004aff0000620100003c000000c4
:10a05c0047000000baff0000d8fe0000c600000058
:10a06c0097000000adfe000050ff0000b7ff00009d
:10a07c00aaff00000d01000082ff00006700000035
:10a08c006702000019ff000069ff0000ec000000ef
:10a09c008bff000097ff00002600000097000000d7
:10a0ac00acff00005bff000038000000c0fe0000a9
:10a0bc00beff00002b0100008fff000085ff000099
:10a0cc0063000000b6000000deff0000c0fe0000d0
:10a0dc00cefe0000430100009401000010000000bf
:10a0ec00b9000000c2000000430000009eff000009
:10a0fc00e8fe000090fe0000bd000000f80000002b
:10a10c0099ff000097ff000030ff00001f000000c7
:10a11c004dff00005fff00001b010000bbff0000b3
:10a12c003900000076010000d7fe000055fe00004b
:10a13c00baff00002000000045000000aeff000048
:10a14c001c0000009200000087ff00000dff0000c3
:10a15c009eff00006bff00004eff0000550000004a
:10a16c0096ff0000afff0000480100002d0000002a
:10a17c00f1000000c4010000ccff0000f1ff000062
:10a18c00c7010000100100002cff00004900000076
:10a19c00ba000000d6ff00004e0000005201000083
:10a1ac008b00000044ff00001400000008010000b8
:10a1bc008f00000072ff00009dff00004c000000ab
:10a1cc00a20100001b010000a2fe00006e000000b6
:10a1dc002b010000ffff000059000000bdfe000035
:10a1ec0082ff00003901000083ff0000d4fe000054
:10a1fc0095ff00003aff0000a4000000f5000000ed
:10a20c0009ff0000a4010000be010000dcfe0000fc
:10a21c00100000004600000045ff0000f9ff0000a0
:10a22c0076000000e8ff00007cff0000c3ff000088
:10a23c0029ff0000eafe0000590000004400000065
:10a24c0087ff00007fff00006e000000bc000000d4
:10a25c001600000010ff0000fbff0000e7010000eb
:10a26c0022ff0000f6fe00000a010000c7ff0000fc
:10a27c00c9ff00004800000035fe0000b7ff0000d9
:10a28c00d20100002aff0000baff00005aff0000b4
:10a29c00b5ff0000b801000033ff00007dfe000098
:10a2ac00fbff0000200000007aff000015ff0000fb
:10a2bc0065fe0000d1fe0000d0ff00004bff000047
:10a2cc0072ff0000e6ff00001a0000009c00000076
:10a2dc00e6ff0000b6fe000068ff0000530000001f
:10a2ec001b000000b5ff0000caff0000e0ff0000eb
:10a2fc002b0000004b00000092ff000036ff000016
:10a30c00a4ff000099000000f1ff00005eff0000b8
:10a31c00780000007b000000c4fe00009dff0000e0
:10a32c00ac000000ddff000098ff000093ff000070
:10a33c00ff000000f3ff000045ff0000ba00000022
:10a34c005aff000050ff0000c9000000e6ff0000ab
:10a35c00a2ff0000ae0000004c0000009dff0000ba
:10a36c0045000000f2ff0000220000003900000050
:10a37c00c9ff0000be000000feff0000ffff000050
:10a38c00910000006bff0000e4ff000025010000bd
:10a39c0092ff0000abfe0000070100003900000036
:10a3ac0014ff0000fe000000f3ff0000e9fe0000b7
:10a3bc0090010000a00000006afe00008100000077
:10a3cc00820100002500000021ff0000a200000017
:10a3dc009a000000250000009b000000d1ff000047
:10a3ec00de0000006200000041000000a800000038
:10a3fc0051ff00008f000000b900000012000000a7
:10a40c00880000005f0000008f00000050ff00007b
:10a41c004e0000006b0000009dfe00006b00000071
:10a42c00170100003b0000001a0000007d00000036
:10a43c000200000038ff000031000000680000003e
:10a44c00d8ff000065000000ba0000002e000000dc
:10a45c00b8ff0000e9ff000011000000ddff000064
:10a46c0078000000530000004a0000006500000066
:10a47c009dff000068000000520000007cff0000ff
:10a48c002a000000760000007dff000071ff000034
:10a49c00c10000009f000000a4ff0000d6ff0000d8
:10a4ac00abff00007dff00004a000000060000002a
:10a4bc005bff00001800000056000000ebff0000de
:10a4cc001b000000ebff00002eff0000a7ff0000a8
:10a4dc005c000000e5ff00002600000099ff000072
:10a4ec0077ff0000520000002200000066ff000011
:10a4fc0005ff0000f8ff0000570000001e000000e0
:10a50c007800000091ff00001cff0000a800000074
:10a51c006800000008ff0000bfff00001e000000e4
:10a52c0042ff000020000000bcff0000c0fe000045
:10a53c00c7ff000025000000cfff000090ff0000c7
:10a54c00baff0000b6ff0000bfff0000c1ff000013
:10a55c0087ff0000b1ff000050ff0000b4ff0000b7
:10a56c00480000005aff00008dff0000ffff0000b4
:10a57c00d6ff000080ff0000cfff0000b9ff0000f5
:10a58c0037ff00003f0000002300000065ff0000c3
:10a59c00adff0000a4ff00009cff0000afff000017
:10a5ac00b2ff0000ddff000013ff0000eeff000013
:10a5bc0060000000d9fe0000b3ff0000f5ff0000b2
:10a5cc003bff0000dfff0000f6ff0000c1ff0000b2
:10a5dc00c4ff0000cbff00004a000000f7ff0000a2
:10a5ec0034ff00000500000039000000d2ff00001d
:10a5fc000d0000003b0000001e000000fcff0000ee
:10a60c004900000030000000f7ff0000430000008c
:10a61c005e0000006b000000610000002c000000d8
:10a62c005b000000410000002300000079000000e6
:10a63c005f000000f3ff0000600000007a000000e3
:10a64c000a0000003c000000500000006200000006
:10a65c005d000000430000008e000000230000009d
:10a66c00f7ff0000960000002e000000eeff000037
:10a67c00630000006d0000005c0000005100000051
:10a68c006300000053000000730000005000000045
:10a69c00ffff00004e0000004e0000001f000000f5
:10a6ac00630000006000000049000000430000004f
:10a6bc00470000003e0000001200000028000000cf
:10a6cc003a00000052000000600000005e00000034
:10a6dc00430000001b0000002000000047000000a9
:10a6ec0017000000020000002a00000020000000fb
:10a6fc0031000000feff00001200000017000000f7
:10a70c00d6ff00001e00000022000000e0ff000049
:10a71c001a00000024000000090000000d000000d9
:10a72c00060000001b000000d8ff0000e4ff000042
:10a73c0037000000edff0000f3ff000017000000e1
:10a74c00e9ff0000f3ff00000a000000d5ff000045
:10a75c00cdff00000c000000ecff0000d2ff000059
:10a76c00e8ff0000daff0000f5ff00000100000028
:10a77c00bfff0000cdff0000e5ff0000ccff000094
:10a78c00f7ff0000eeff00009fff0000d5ff000068
:10a79c00f7ff0000afff0000baff0000faff000057
:10a7ac00ceff0000cfff000007000000caff000032
:10a7bc00c2ff0000f5ff0000dbff0000c0ff00003f
:10a7cc00e8ff0000d2ff0000c2ff0000f6ff00000f
:10a7dc00b6ff0000acff0000e5ff0000a9ff000081
:10a7ec00c7ff0000f0ff0000aeff0000b1ff00004b
:10a7fc00d7ff0000bbff0000b2ff0000c9ff000044
:10a80c00bfff0000c4ff0000d7ff0000bfff000027
:10a81c00c5ff0000d7ff0000ccff0000d6ff0000f2
:10a82c00c9ff0000c4ff0000deff0000e2ff0000d3
:10a83c00d0ff0000deff0000dbff0000e9ff00009e
:10a84c0005000000fdff000000000000f6ff000006
:10a85c00f0ff0000deff0000f2ff0000fdff000033
:10a86c00e1ff0000d8ff0000ffff0000e7ff000041
:10a87c00f1ff000005000000ffff000025000000b4
:10a88c00d6ff00003e000000a0ff000075fe000097
:10a89c0015ff0000f00400003000000060f900001b
:10a8ac003e070000f502000044f6000049020000db
:10a8bc001107000099fb000051fc00005505000039
:10a8cc0087fe000033fe00005300000018fe00005d
:10a8dc00410200004efe00000bfd00007fff000057
:10a8ec0024020000ed0000000e1600001bf7000013
:10a8fc00dde0000030220000fa0200004fdf000013
:10a90c001f06000099100000fb040000b0e90000d5
:10a91c0028f20000b4320000def400004ad200003d
:10a92c00882500004a0a000095e80000bc000000e1
:10a93c00f30300000e0b0000f90d00003cdb0000df
:10a94c0067010000b21e00003fe90000a4ef000008
:10a95c004c130000250e00001ae8000059020000fc
:10a96c007a0b00000ff6000018fc0000e901000053
:10a97c0057000000abff00009e150000bae8000075
:10a98c0067ef0000ea26000026f20000c0eb000092
:10a99c002a0c00008502000051fd0000f0fc0000b4
:10a9ac0013fe0000230800009405000026f60000aa
:10a9bc00f4ff000025070000cff80000ddff0000c9
:10a9cc0068020000a2120000e902000011de000083
:10a9dc00e71400005f0e000018df0000f900000013
:10a9ec00a10e0000e6fd000071f800005df900000a
:10a9fc002308000014130000b3fc0000eef4000068
:10aa0c00610800003a060000f0f7000059fa000057
:10aa1c006c0d0000b50700009bfb00002eee000043
:10aa2c00620c000064060000ebdd0000db1000008f
:10aa3c00ba0800006ef900000aff000058ff000081
:10aa4c004c0b00008ef200009a030000af010000d6
:10aa5c0039fa00008506000086000000760600002a
:10aa6c003bf30000e3ff0000160b000020f0000099
:10aa7c00b8fc000074040000dbfb000004fe0000c6
:10aa8c0078010000bafe00002f0100005200000007
:10aa9c00b6fb00004cfc00003efe00008e090000de
:10aaac00600000001c04000018050000e7f0000026
:10aabc0016030000350100000bf1000032fc000011
:10aacc0075070000d7fb000014f40000ad0c00006b
:10aadc00edf90000c8060000fd0a000023f5000097
:10aaec00720b00001f000000a0020000e506000031
:10aafc00cdfa000035f80000b60b000001f700009d
:10ab0c00f7e90000e60a0000040300009df50000d0
:10ab1c002cff000093060000e7fe00008f000000f1
:10ab2c0073fe0000ff0900001c070000a0fc0000e1
:10ab3c007d020000e600000082fd000075ff0000b1
:10ab4c0092ff000059f40000170200002b030000d4
:10ab5c008cfb000095fc0000920800003aff0000fe
:10ab6c000cfe00002cff0000e7fa00003c0c00007b
:10ab7c00e6f40000ea030000120b00008cef00006a
:10ab8c00c10d00007101000048f10000670b0000ce
:10ab9c0085fa0000c5fb0000ba0300003e0200006d
:10abac008700000002fd0000caff0000dc0100006d
:10abbc00470000000dfa000012050000a308000079
:10abcc00d5080000d40200005df80000e1fd000093
:10abdc00d70a0000e8f700006def0000c70c00007a
:10abec00f6040000fbf4000005fc00000c0d000056
:10abfc00ccfa0000ae0500007913000072f50000dd
:10ac0c0084050000f90b00002800000081fb000007
:10ac1c00c5ff0000070a0000fbf7000021ef000051
:10ac2c00900900008b020000bbf10000e80100005d
:10ac3c003b050000c8ff00009e09000097020000c1
:10ac4c00eafc0000dc0a0000eafe0000cbf4000085
:10ac5c009f050000330600004af7000010fe0000bc
:10ac6c0034000000550800003cf400002bf40000f8
:10ac7c005710000080f40000f5fe0000bc06000038
:10ac8c00d6f900000c0200005d03000038f600004d
:10ac9c001604000010060000aff2000027050000ab
:10acac00b6040000d2f90000d1fb000045030000ff
:10acbc0027010000fbfc0000ce010000d4fa0000cc
:10accc00fe01000050ff000010fc00000405000015
:10acdc0009ff0000de07000089030000ccf700002c
:10acec001cf80000090f000081fa000058ef00006a
:10acfc0034090000eb030000fdfb000075f40000bc
:10ad0c005c09000045ff0000330200006f090000e1
:10ad1c00c10a0000400d0000eae900005c030000dd
:10ad2c0018130000d9f10000e5ed000078040000d4
:10ad3c0004130000b1f5000031e5000064110000bf
:10ad4c00ec160000ebed0000dcf20000af1400008c
:10ad5c007907000095ee00001f050000df0b0000d6
:10ad6c0003fa0000acfe000010fe000052f40000dc
:10ad7c00c2060000e80300005df40000760200004b
:10ad8c0058070000510200002bfb000008000000d7
:10ad9c00dc0900006e0100003efa0000f4fe000029
:10adac00f8010000030200007dfb000025fc000000
:10adbc005e03000018020000dffa0000fffa00003a
:10adcc005e0300002200000059010000f9fd0000a4
:10addc002f0c00009bf800003ef700004111000012
:10adec0072f6000008fc0000490400000502000097
:10adfc001dfe000018f90000760600002e01000070
:10ae0c00f4f600001702000008030000b0fd00007b
:10ae1c007bfb00001b030000fd0b0000bd020000cb
:10ae2c000bee0000e6fb0000e31b0000a5f30000a6
:10ae3c00e5e500006515000037080000c2ef0000d2
:10ae4c00d9f40000010e0000cd06000097f40000bc
:10ae5c001a0b000022070000ae050000f0f80000fd
:10ae6c0021fd0000d20a000076fc0000f9f600007b
:10ae7c0093f50000030a000016060000caed00005e
:10ae8c009efd00005b0d00007b0b0000f3fa000040
:10ae9c0071f70000df1000008f030000e1f20000ea
:10aeac00590100003d0600002d000000f5f70000e0
:10aebc0011f80000610b0000f5030000f7f0000032
:10aecc00da03000072080000d2f9000099f70000c4
:10aedc0015110000450c00003ce9000041ff00008a
:10aeec0071100000a6f80000a6ef0000b6060000e6
:10aefc0020080000a6fd000070f40000fa0200001b
:10af0c00f31d00009ae30000bef500008220000053
:10af1c006def000047f200003009000073050000df
:10af2c005307000048f1000050fe0000960f00008f
:10af3c00c7f400004ff10000b00700002b10000018
:10af4c0090ed00009a0200003610000043f400005f
:10af5c0062fc000084ff00009d0e0000460900000a
:10af6c00cee400006b0400007d1c00002feb000001
:10af7c0077f00000571200002f030000e7f20000ea
:10af8c006ef90000cb0c000099020000e4f3000005
:10af9c0052020000de09000001fe00008ef80000e5
:10afac001f160000bf02000058e1000064120000f0
:10afbc00df1200002ad800009b000000941e000045
:10afcc0057f00000f4f70000f20200004c100000f3
:10afdc00ad0100009afe0000b910000092f00000d4
:10afec00cb0400006c0f00003fe5000022040000c1
:10affc00b5170000a8e60000e80300006f0e000083
:10b00c005ff700006af3000025010000360c000019
:10b01c0025fc00002c13000097ec00006ffc0000d6
:10b02c0053200000eede0000e1f40000cc1500001f
:10b03c006dfc00008df60000250200009dff000055
:10b04c000a130000ab0100000ede0000091e000018
:10b05c00740d000071d7000042060000f51d0000c1
:10b06c00c5f400000de3000008130000ea0a00001c
:10b07c00a0e7000077f500009511000054090000ce
:10b08c00dce20000cf05000011100000fafa00000d
:10b09c005bfe0000a4000000950c000025f80000e9
:10b0ac00a7fb00002e080000bffc00001bff0000e7
:10b0bc00eeff000052fc0000acfa0000b5000000ee
:10b0cc00f5ff000072fb00003d040000d5fb000002
:10b0dc005ffe00003204000068f700005d13000002
:10b0ec00f8f90000bde80000d11900004e00000086
:10b0fc00bae80000100600006b0c00003ff70000df
:10b10c0090f40000fe08000066070000c2f3000087
:10b11c0060fe0000be060000d4000000baf800007b
:10b12c009b04000063100000cae8000026fa00002f
:10b13c00d21a0000a3ef0000b8e60000be1a00000f
:10b14c00070400007ae7000038090000f908000045
:10b15c00f9fb00006f050000561800008eef000090
:10b16c005df000001e1f0000a4f9000042e4000086
:10b17c0083100000b4090000a1ed000040fe0000a7
:10b18c00fc0e00002b02000022ed0000390900002b
:10b19c008a050000dcf60000b4fc0000df070000ac
:10b1ac00761c0000b8e30000c2ec0000022b00008b
:10b1bc0033f300009fd80000ff1d000005100000b5
:10b1cc0041e20000c005000025070000280a00002d
:10b1dc00b80a0000aef30000d0ff0000dc10000045
:10b1ec00c3f9000011ec0000670f0000b209000069
:10b1fc0029f20000b1f800006a06000051fc0000c2
:10b20c00e7f70000eaff000013030000a8060000a7
:10b21c0055fa000084fe000038100000ba07000048
:10b22c00d3ed0000c9010000661300002af10000f4
:10b23c004bf40000f8100000680100001df2000043
:10b24c001d010000fd060000d6fd00003df90000c8
:10b25c0042010000b803000086fe0000aefb0000b7
:10b26c0010060000260700008df5000062fc0000af
:10b27c004e080000a1fc000010f6000001050000c3
:10b28c00760400007cfa000062ff00003903000025
:10b29c0073000000b4020000e2010000a2fe0000f6
:10b2ac006c0a00007eff000089f00000070400001b
:10b2bc009a0a0000c0f70000f3f20000eb0900004e
:10b2cc00e006000081ee0000f9ff0000610b0000b9
:10b2dc0068f60000b5f90000511500007808000070
:10b2ec00c1e9000004000000cf11000076fb000053
:10b2fc00a0ee0000b8030000b00f000032f5000013
:10b30c007cf30000d40c00006e05000052f200002b
:10b31c00d5010000050d00009c0300009600000004
:10b32c0013f7000085fc0000ae070000f5ff0000dd
:10b33c00d3f00000aefa00007a1800002ff50000e0
:10b34c0036eb0000d51400001f02000052e4000090
:10b35c00cc1500008d2e0000a6d8000010e90000ce
:10b36c00942c0000b802000095dc000070f700007f
:10b37c00701e0000d5fc00003ddf00000f0a00002d
:10b38c00fc1d0000e3f2000015ee000004180000a4
:10b39c004c000000aaef0000b30d000004070000f1
:10b3ac00a9f20000e6ff0000c705000062ed0000f6
:10b3bc00defe0000760c000041f60000b0f8000044
:10b3cc00e6080000b90e000086fc000044fc0000fa
:10b3dc00590800007f0100006af8000086fd00009b
:10b3ec00d5030000a3ff00007afe00008df80000da
:10b3fc00ec010000a906000038f4000077f9000009
:10b40c005c0b0000a5010000dcfa0000f800000055
:10b41c00fdfc000048060000aa01000003f2000039
:10b42c000f0500004e0b0000b9f50000fef80000ff
:10b43c003f0800002e01000059f90000e8fc000054
:10b44c006c030000e302000079f80000dafe000053
:10b45c003009000015040000effd00002efa00007a
:10b46c00cdff0000c6030000d5ff000074f80000fb
:10b47c003e000000fb0a000056f80000d7f7000061
:10b48c00090700001f02000049f800005a000000e4
:10b49c00241100001606000021f6000039fe000001
:10b4ac004a070000b9fc0000e6fa0000bcfd0000f1
:10b4bc0042ff00001f0800000cf800002cf80000f0
:10b4cc00a50a00004bff0000aeec0000c20d00000e
:10b4dc00b1270000dbed0000f4e50000ab13000029
:10b4ec00500e000090ed000044f00000540d0000e0
:10b4fc00d7090000eeef000013f4000087180000dd
:10b50c008a060000beeb000073030000400b000035
:10b51c006dfa0000b6fc0000730f000095ff0000f0
:10b52c00b7f000001b050000e204000054ed000021
:10b53c00f6fa0000c40f0000bdf90000e5f30000ae
:10b54c007e090000ea0a00001c080000b708000091
:10b55c002afd0000caf60000eeff000032030000d6
:10b56c005bfc00002af80000c4ff0000e70b0000a1
:10b57c0061fc000098ec000023000000490c000066
:10b58c004bfb0000fefa00002e0d0000d203000061
:10b59c00cff5000021ff00009b060000adff00006e
:10b5ac0062f800008d00000039090000f90100006c
:10b5bc00f9f8000071fc0000b3050000fd0000006c
:10b5cc00fcf70000e9ff0000ba0d0000380600008f
:10b5dc00a5ef000084f900006d0e0000970100003b
:10b5ec00dff20000e4fb00007c0c0000b60500005c
:10b5fc004ff3000040fc000004090000590000005b
:10b60c0032fb000087030000cb0c00003d0600005d
:10b61c002df6000002fc0000bc0500009d0100009e
:10b62c00bbfa00000ff60000190400001d0b00000f
:10b63c0055f7000088f50000900b00003e09000053
:10b64c003cfa0000ae010000f60d000015070000ea
:10b65c004ef300004afa0000bc0a0000b2010000e0
:10b66c00e9f1000022f60000c10a00000b06000000
:10b67c0018f2000053f90000da0e0000a9080000cf
:10b68c0000fc0000030200002f060000590100001e
:10b69c00a6f800006efc0000a5050000f7fe0000f7
:10b6ac00e6ef000040fb00007e0c000096fe000060
:10b6bc002bf50000320200009a0c00004806000036
:10b6cc000efc0000ddfc0000af04000019010000be
:10b6dc00f0f7000087fc0000ac0400003ffd000008
:10b6ec00cdf20000df000000360a00007ffa0000f7
:10b6fc00aff50000c4070000770d0000e4f900006e
:10b70c00c9f50000bd060000060c0000cafc0000d4
:10b71c00b2f40000db010000b7090000e2fc0000fd
:10b72c0063f0000002fe0000ad0b00004eff0000b5
:10b73c00d2f4000081010000e90e00003f0500007a
:10b74c002ef700000ffd000082070000150300001b
:10b75c002cf90000ecf9000098040000250500000d
:10b76c0056f80000f8f80000cc070000c5050000f2
:10b77c003efb0000480100003d0900004cff0000aa
:10b78c0066f5000064040000bb0e0000fafc00002b
:10b79c0052ed000012fb0000d80e0000e404000083
:10b7ac0015f00000c3f70000a90e0000d40800003b
:10b7bc00a1f90000eafe0000470700001502000096
:10b7cc009bf8000018fd0000690500008efe0000cb
:10b7dc000bf500008b010000560800008bf90000ef
:10b7ec00b4f70000ae040000ac09000046020000f3
:10b7fc00e3fb0000a5ff0000c204000030fe0000c7
:10b80c00a3f800004e0000008306000039fb000086
:10b81c00c8f200001a030000610800005ef8000086
:10b82c00e4f70000f40a0000e20a000088f60000c9
:10b83c00eaf80000db090000270a0000dbf9000031
:10b84c0038f60000b1040000f8070000ccf8000046
:10b85c005df00000730100000a0c000021fc0000e8
:10b86c0031f30000f8030000940f0000ed0200001b
:10b87c0041f70000b9fe00001009000009020000a9
:10b88c0072f80000d6fc0000ea030000e80100009a
:10b89c006cf9000063fa00004a0500002404000063
:10b8ac007afb00008f00000034040000a5f90000b2
:10b8bc009efa0000b80d0000851000001ff6000075
:10b8cc00a3ea0000b30100006612000002040000ad
:10b8dc004aec0000cef30000ca0f0000640a00001e
:10b8ec00f7f2000085fa0000060b00005e04000071
:10b8fc0063f80000e9fb0000270500004a04000083
:10b90c00f70400008d06000092fa000017f4000006
:10b91c00f2fe00004303000070fc0000f1f900008f
:10b92c008b000000da07000087ff000040f80000e1
:10b93c0056020000e812000001150000e8fc0000af
:10b94c00aae9000079f30000420500007c08000021
:10b95c009e0000007ef7000092f9000096030000a4
:10b96c00360900004604000046f80000e7f4000029
:10b97c00a9fb000058030000fb0600009f0c000010
:10b98c00ce0a0000d6f9000005ee0000dcf5000040
:10b99c0002060000fe07000012fc00009ff90000e8
:10b9ac000805000010070000defd0000fdfe000091
:10b9bc00080b00002d0b000090fb000031f2000082
:10b9cc0054fc0000f10900004406000094fb000048
:10b9dc00fffa000079000000cafd0000e5f6000047
:10b9ec0053fb00001105000060060000dafe0000a9
:10b9fc006afa0000ea0200003d1100000813000082
:10ba0c005501000097ee0000e3ef0000220000005b
:10ba1c00010a0000510400006df900002ef900002d
:10ba2c00b40200002e05000054ff000016fd0000bb
:10ba3c00c3fe00007efb0000cff80000b40800003d
:10ba4c0053170000980800007cef000003eb000087
:10ba5c00c7fc0000c8090000650300009ff9000046
:10ba6c0008fc0000e00300000f020000aafe00002a
:10ba7c00570700005d0c000083020000d5f40000a5
:10ba8c0044f200009cfe0000cd0a0000d109000029
:10ba9c0089fe0000b2f6000054fa0000dafe000045
:10baac003cfd00005afc000010000000da0400000d
:10babc001402000013fb0000960000002c0f000085
:10bacc0094110000a601000066ef000061ee00007a
:10badc00d6fd0000300a0000f908000099fe0000b5
:10baec007ff500009cf7000034000000ee0400001d
:10bafc00c40100001bfc0000e5f80000da000000a7
:10bb0c002c130000c713000058fe00001aec0000b4
:10bb1c00aced000040ff0000560a0000c30300001b
:10bb2c00a7f900006bf90000940100005305000018
:10bb3c00b2020000de020000f00400000704000066
:10bb4c005dfd0000f7f4000029f700003704000049
:10bb5c00a20c00005b080000bffd0000a7f600006f
:10bb6c009cf4000040f6000015fd00006c0600007f
:10bb7c005a0a000092030000bbf900000afd000005
:10bb8c006c0c0000e313000086090000faf50000bd
:10bb9c0093ea000092f0000011010000920c0000ea
:10bbac0002090000b6fd0000b4f7000018fa00000e
:10bbbc00ad0000007e0300009100000017fc0000a7
:10bbcc0066fc00006d070000da110000db0d0000c0
:10bbdc00aefd0000f7ec00000eea0000e7f60000f6
:10bbec00c1050000490b0000a7070000640100001c
:10bbfc0066fc000007f9000075fc00004607000019
:10bc0c00e70e0000500c0000630200004bf800002f
:10bc1c0093f300001ef5000092fb00006c04000082
:10bc2c0023080000690300009afc0000fdf90000e5
:10bc3c00e3fb000059fe0000b70000003e050000c9
:10bc4c00760a00009a0c000042090000b9000000be
:10bc5c00e3f50000a4ee00007ef20000d5ff00002a
:10bc6c0080090000250900009a030000affd0000c8
:10bc7c00f0f80000fbf700007cfe0000cc07000091
:10bc8c00d00b00005d0800006501000014fd0000f1
:10bc9c0097fb00000ffb000049fc000040ff000078
:10bcac0077000000ddfd00006efb0000cafc000008
:10bcbc00feff0000c2010000b6010000830200007c
:10bccc0061060000330b0000cb0c0000de06000008
:10bcdc0035fa000019ef00002aed0000aef5000067
:10bcec0048020000380a0000c00a000005050000e8
:10bcfc003dfc000089f60000ccf80000f4000000c8
:10bd0c00f5070000a90900006c060000a301000063
:10bd1c00f1fd000000fc0000b0fb0000d1fb0000b6
:10bd2c002dfb000030fa000093fb0000ceff00005a
:10bd3c002d040000ce0500001d0300009efe000037
:10bd4c009ffd0000c1020000900a0000a60e00003a
:10bd5c00eb090000bdfc0000cbee000048e9000040
:10bd6c0050ef00005bfc000044090000670f00006e
:10bd7c00570c0000c903000033fb000021f7000042
:10bd8c000ef90000d3fe00008e0400003407000002
:10bd9c00ce0600008b0400006401000064fd00006e
:10bdac00acf80000c7f4000042f400008ff800006b
:10bdbc0047000000d3070000940b00009b08000014
:10bdcc006601000079fe0000b0010000d5060000fd
:10bddc00bc0800008f0300001ffa0000f4f1000003
:10bdec0033ef0000bff3000075fd00009b0700005f
:10bdfc00ad0c0000740a00001704000036fd0000b2
:10be0c0086f900007afa00007ffd0000990000001e
:10be1c00980300003b060000f606000074040000c6
:10be2c00a3ff000053fa00004ff500006bf2000076
:10be3c00bcf40000b9fc000063060000e20b00003b
:10be4c00420a0000db050000ba040000b90500003e
:10be5c00eb050000e40300003cfe000045f600008a
:10be6c005df0000060f0000083f60000daff0000d7
:10be7c005b080000c80c0000f00b00003506000049
:10be8c00a3fd000046f70000e1f600000efb0000e9
:10be9c008f0000007c05000088080000a20800004c
:10beac00050600008401000005fc000057f60000a8
:10bebc0012f200003bf20000fbf70000da00000079
:10becc00db0800009a0b0000f6090000b80800001f
:10bedc002c080000720700003b0500001aff000050
:10beec00b2f600005af00000cdee000062f2000045
:10befc0034fa000040040000cf0c0000a00f00003a
:10bf0c004a0c0000f9040000bafb0000eff400003a
:10bf1c00f7f30000e8f800006b01000025090000b1
:10bf2c00d20c0000050c000066070000edff0000bd
:10bf3c00b5f7000050f100005cef0000fff20000cc
:10bf4c00b0fa0000c6030000370a0000270b0000ff
:10bf5c000e0a0000240a0000f90900005e08000027
:10bf6c0059040000c7fd0000eef5000028ef0000aa
:10bf7c0017ed00001cf10000cbf9000030040000ac
:10bf8c00ae0c0000f0100000760f000081070000de
:10bf9c00abfc00008af5000081f4000072f8000090
:10bfac00140000002a080000ce0c0000290c000030
:10bfbc003b060000bcfd00000ef6000023f1000063
:10bfcc0099f00000faf40000e0fc0000e604000028
:10bfdc0046090000a20900001409000049090000ec
:10bfec00a509000030090000ee05000056ff000016
:10bffc000af7000073ef0000d1eb000017ee000011
:10c00c0025f60000bc0100002c0c00006f11000094
:10c01c00b6100000470a00008e000000bdf80000ba
:10c02c00c9f5000077f80000a7ff0000e206000049
:10c03c005f0a0000f00800003f030000adfb0000a9
:10c04c00cff400003df10000e0f20000e4f8000045
:10c05c00720000002106000073080000c1080000f7
:10c06c005d080000e4070000a7070000ba06000006
:10c07c00e6030000ccfe000011f80000e4f1000023
:10c08c00daee000043f0000005f60000e8fe0000c8
:10c09c00c90700002a0d0000040e0000650a00000c
:10c0ac00b10400009d0000004eff0000a500000040
:10c0bc00dc020000fd020000e1ff0000a0fa00001d
:10c0cc0075f5000090f20000aaf30000edf80000f6
:10c0dc00860000005d070000d80a0000630a00001b
:10c0ec00df06000039020000cefe00001ffe00003b
:10c0fc00e4ff0000570200007f030000490200002b
:10c10c0003ff0000b4fa0000cff600001bf500009e
:10c11c0091f60000e0fa00007300000054050000e6
:10c12c001008000010080000b006000053060000c4
:10c13c002f07000095070000fe050000a701000076
:10c14c0026fb0000ecf30000c1ee000071ee0000d5
:10c15c0074f300007dfc0000500600007f0d000011
:10c16c00211000000f0d00002b050000c9fc000081
:10c17c0037f800006cf800007cfc0000a002000006
:10c18c00a4070000ef080000f1050000a0ff00006c
:10c19c00caf80000f2f3000072f2000006f500008d
:10c1ac00fffa0000270200008d070000490900007b
:10c1bc00b00800005c080000b1080000f5080000a1
:10c1cc00d3070000790300003ffc000014f40000ca
:10c1dc00b1ed00001bec000084f0000028fa000018
:10c1ec00e1050000c10e0000db110000030f000090
:10c1fc00e606000048fd00000ff7000016f60000f0
:10c20c00b7fa000085020000ab0800006c0a0000c1
:10c21c004c0700009600000000f9000000f300003d
:10c22c0037f10000acf400009dfb0000db020000c5
:10c23c004f070000b2080000a90800002c080000fd
:10c24c00cb07000078070000fe0500005302000039
:10c25c0074fc0000a4f5000058f00000d1ee0000c2
:10c26c00e0f10000fcf80000540200003b0a000062
:10c27c00010e00002e0d00005b080000ec02000017
:10c28c00cfff00006bff00005a01000021030000eb
:10c29c00430200007dfe00002df900008af400002e
:10c2ac00a5f20000cff40000b6fa00000c0200006a
:10c2bc00f20700009e0a0000d0090000cc06000026
:10c2cc005703000011010000bb00000067010000d3
:10c2dc008d01000030000000fcfc0000dff80000c5
:10c2ec004ef5000003f4000070f600002efc000078
:10c2fc00f80200001c080000cd090000fd0700003a
:10c30c00170500009d0300000304000066050000f3
:10c31c00e4050000e00300003fff0000d7f8000038
:10c32c008ff200000cef0000e9ef0000a1f5000017
:10c33c00b2fe0000970700006d0d0000830e000098
:10c34c001b0b0000a3050000a500000001fe00006f
:10c35c0050fe00005a000000eb0100001e0100001e
:10c36c00b9fd000015f90000f0f4000037f30000ef
:10c37c0070f500007efb00002103000000090000a6
:10c38c00b50a0000e20800006d060000e60400009b
:10c39c003e04000046040000170400005702000091
:10c3ac0030fe00002ff800003ff2000009ef000003
:10c3bc004ef000001cf60000dcfe000094070000ac
:10c3cc00c70d0000530f00001a0c000017070000e7
:10c3dc00a1020000deff000015ff00001aff0000a4
:10c3ec00ddfe00008cfd00009efa0000def6000071
:10c3fc0014f4000020f4000009f800009cfe00007a
:10c40c0052050000fe090000620b0000f10900005b
:10c41c001e0700006f040000de0200005102000045
:10c42c00a8010000ddff00009afc00006ff800007e
:10c43c0077f400002df2000025f30000d3f7000084
:10c44c00edfe0000fb050000010b0000a30c00003a
:10c45c004d0b0000bd0800001c060000330400005a
:10c46c00db0200005e0100001dff000083fb0000ea
:10c47c0023f7000038f300001ef1000093f20000d7
:10c48c00e6f70000cbff00009f070000b80c00008f
:10c49c00c50d00007a0b0000f2070000a20400009a
:10c4ac0090020000bc010000fb00000060ff0000d7
:10c4bc0059fc000058f8000056f40000c5f10000cb
:10c4cc0047f2000061f6000081fd00007b050000d2
:10c4dc008c0b0000c40d0000580c00003b09000040
:10c4ec0009060000c3030000540200004a010000ca
:10c4fc008aff000020fc000099f70000fdf200000c
:10c50c0034f00000eff0000067f50000d2fc0000f2
:10c51c0030050000fd0b0000f00e0000a40d000023
:10c52c00150a0000390600003d03000067010000f9
:10c53c0025000000e2fe0000d4fc000081f90000a0
:10c54c006ef50000e8f100003bf1000063f4000020
:10c55c00a0fa00007b0200007e090000760d0000ae
:10c56c005e0d0000a40a00007b0700009f04000081
:10c57c009c02000079010000620000003ffe0000f8
:10c58c00bffa000085f6000063f200005cf00000ca
:10c59c00f0f1000030f700001fff00001b07000047
:10c5ac00b90c0000a70e0000240d0000130a0000b7
:10c5bc00e3060000630400008e020000d4000000bb
:10c5cc00aefe000049fb00000ff70000e9f200008e
:10c5dc0020f00000b6f00000fcf4000032fc00007b
:10c5ec00820400003f0b0000a00e0000220e000091
:10c5fc00560b00002108000090050000e30300002a
:10c60c00770200009c00000072fd000008f9000099
:10c61c0055f400006cf0000039ef0000b3f100009d
:10c62c0083f7000095ff000095070000310d000016
:10c63c00d70e00003e0d00004a0a00003107000032
:10c64c00fa0400006b030000dd010000caff0000cb
:10c65c0035fc00006cf70000c5f200009aef0000fa
:10c66c006fef0000d3f2000061f9000085010000bb
:10c67c00f6080000a20d00007c0e0000990c0000d2
:10c68c00ab090000d5060000e90400008a03000095
:10c69c000b020000d8ff000013fc00003bf7000069
:10c6ac0063f2000017ef00001fef00009cf2000087
:10c6bc0026f900004d010000c8080000a90d00007b
:10c6cc00ce0e00002d0d0000820a0000be070000f7
:10c6dc009e050000ee030000f401000047ff00007f
:10c6ec005ffb0000adf6000060f2000086ef00007a
:10c6fc00a4ef00003cf3000091f900004d01000094
:10c70c008c080000320d00003d0e0000be0c000035
:10c71c00490a0000fd0700002f060000b7040000c6
:10c72c00150300006b0000002cfc0000f5f6000067
:10c73c0044f2000047ef0000f8ee000012f2000097
:10c74c0046f8000036000000e5070000560d00001a
:10c75c00fb0e00005a0d0000b60a0000370800005e
:10c76c005a06000023050000b70300007201000008
:10c77c00b7fd000090f8000056f300007eef0000bb
:10c78c0044ee0000b0f0000062f6000042fe000033
:10c79c0065060000510c0000d70e0000c10d000012
:10c7ac000c0b000094080000ae060000830500008e
:10c7bc0086040000dc020000aaff0000c7fa00009b
:10c7cc0015f5000050f0000012ee000042ef0000e2
:10c7dc00e5f3000026fb000060030000370a0000b0
:10c7ec00ec0d0000c60d00006c0b000041090000b0
:10c7fc008d070000a106000034060000fa040000ba
:10c80c003302000056fd00004af700009ff10000c3
:10c81c00f4ed0000aeed0000ebf000001bf70000a3
:10c82c001eff00009a060000d40b0000090e000049
:10c83c000c0d0000b00a0000de08000081070000ab
:10c84c004c0600004205000069030000d5ff000003
:10c85c00d0fa000050f50000aaf0000052ee0000e3
:10c86c000cef0000d3f2000020f900007300000070
:10c87c0017070000bd0b0000320d0000370c000044
:10c88c00a40a0000f8080000940700008b060000c2
:10c89c0036050000f1020000e4fe000084f90000ff
:10c8ac0010f40000a3ef0000bded00001fef00002e
:10c8bc0075f3000045fa0000a30100000808000011
:10c8cc00300c0000f30c0000c40b00000a0a00003e
:10c8dc006c0800005c0700007806000051050000a1
:10c8ec001803000015ff0000aff900001af4000057
:10c8fc00a1ef00008bed0000f5ee000074f30000da
:10c90c0038fa0000a6010000f8070000240c000013
:10c91c00e50c0000e20b0000710a0000da080000d0
:10c92c00fc070000fe060000a80500005c030000e8
:10c93c001bff0000b5f9000007f4000094ef0000a5
:10c94c00d6ed000059ef0000c6f300001efa0000ff
:10c95c00160100002d070000410b0000620c0000c6
:10c96c00570b0000f3090000c70800001308000073
:10c97c00780700006a0600004b0400005e0000000f
:10c98c001bfb000060f5000078f0000007ee0000d3
:10c99c00e0ee000066f20000f2f70000acfe0000d2
:10c9ac0005050000dd090000d50b0000270b000079
:10c9bc00e7090000d8080000a6070000d806000010
:10c9cc003d060000f90400006a02000023fe00008e
:10c9dc00b7f8000052f300007bef00004aee0000b5
:10c9ec001af0000060f400005bfa00003d0100004a
:10c9fc00f9060000ce0a0000ed0b0000710a0000e1
:10ca0c001609000000080000ee060000a806000051
:10ca1c0033060000b4040000810100007dfc00001e
:10ca2c00cff60000a6f10000a8ee0000d6ee000044
:10ca3c00b9f10000aaf60000fffc00005003000052
:10ca4c001b080000eb0a0000b80a000014090000e3
:10ca5c0064080000b00700003e0700005b07000000
:10ca6c00b2060000a2040000cb0000007efb000018
:10ca7c0000f60000a6f100007def0000f6ef0000cc
:10ca8c00c8f200006bf7000004fd000096020000e5
:10ca9c007b0700005e0a0000b40a0000e6090000f3
:10caac000909000054080000d707000079070000ae
:10cabc00ad060000c20400003701000054fc000069
:10cacc00f7f6000064f20000aaef0000a0ef0000ef
:10cadc0051f2000005f7000024fd00004d0300009a
:10caec0076080000420b0000450b0000520a0000c3
:10cafc00340900002c08000079070000e006000053
:10cb0c00e50500008103000077ff000043fa0000f8
:10cb1c00caf40000b3f0000033ef0000b5f00000e1
:10cb2c00acf4000068fa0000ad0000002206000022
:10cb3c00d6090000030b0000620a00002709000060
:10cb4c0042080000c40700001d0700002906000071
:10cb5c00ff0300002e00000033fb0000c9f50000ad
:10cb6c0067f1000077ef000071f00000e8f30000bf
:10cb7c0064f90000b9ff000081050000890900007c
:10cb8c00c10a0000330a00006509000056080000c5
:10cb9c0043070000a0060000d20500001f0400009f
:10cbac00c6000000cefb000035f6000050f100007e
:10cbbc0097ee0000bbee0000c6f10000def60000b0
:10cbcc0072fd00000c040000f1080000b80b00001e
:10cbdc006d0b0000b7090000a608000072070000ea
:10cbec00b90600008e060000ae05000082030000ae
:10cbfc006dff0000f3f9000059f40000f0ef0000a5
:10cc0c005aee0000d9ef0000b9f3000063f9000000
:10cc1c00f4ff0000ac050000ad090000360b00006d
:10cc2c00f0090000ad080000220800005f070000ba
:10cc3c00490700003a070000f80500001e03000039
:10cc4c0076fe0000c5f800008ff300001ef0000017
:10cc5c0051ef000042f1000046f50000aefa000072
:10cc6c005c0000008805000065090000900a0000c7
:10cc7c00dc090000f808000058080000f20700006a
:10cc8c00bd070000660700002e0600005d030000d3
:10cc9c00fdfe0000c6f90000caf4000049f10000d6
:10ccac000df0000076f10000e2f40000c8f900007d
:10ccbc006fff0000ce040000f6080000900a000090
:10cccc000e0a00003e09000077080000a2070000d1
:10ccdc004f070000350700005c0600002804000028
:10ccec00650000004efb0000f8f50000e9f10000c3
:10ccfc001df00000dbf00000c2f300006af8000039
:10cd0c00dffd00002e0300008e070000ba090000b2
:10cd1c00560900003f080000cb0700006a0700001e
:10cd2c004c0700008c070000220700006205000081
:10cd3c00f301000032fd0000f3f7000061f3000086
:10cd4c00b3f000009df00000f5f20000bdf600000d
:10cd5c008cfb00007a000000f9040000330800008e
:10cd6c00140900005f0800004b070000f0060000eb
:10cd7c0005070000fa060000fc0600005e06000035
:10cd8c0054040000d00000004dfc00008af70000a5
:10cd9c00c1f30000f3f1000037f2000067f400006b
:10cdac00fbf7000056fc0000df000000200500002f
:10cdbc00c10700001b080000af07000002070000bd
:10cdcc00800600009e060000ce060000d60600007d
:10cddc003406000032040000e7000000b9fc00003b
:10cdec005bf80000d6f400000ef300003ff30000e7
:10cdfc0017f5000014f80000f4fb0000e4ff00003d
:10ce0c00890300008e060000a40700003407000010
:10ce1c007d0600001b0600000c0600002706000023
:10ce2c00620600002a060000d90400004c02000033
:10ce3c00bafe000082fa0000a5f600002df40000f6
:10ce4c006ef3000063f40000b2f600000efa00006e
:10ce5c00effd00009f0100002405000016070000f4
:10ce6c0076060000b30500009405000044050000a0
:10ce7c00a905000064060000990600002f060000ba
:10ce8c006a0400003201000032fd0000f7f80000d7
:10ce9c008cf50000ebf30000ebf3000063f50000f1
:10ceac0038f80000c4fb000058ff0000900200009e
:10cebc000e050000c1050000f2040000a3040000f0
:10cecc0025050000910500005e06000040070000eb
:10cedc003f0700004b060000ef0300005a00000063
:10ceec0052fc00007ef80000b0f5000088f4000051
:10cefc00f6f4000097f6000033f900005afc00002d
:10cf0c006cff0000170200002d0400002305000038
:10cf1c00100500001105000081050000fa05000055
:10cf2c0080060000f1060000d5060000dd050000bb
:10cf3c00d5030000e400000069fd0000fdf90000cd
:10cf4c004af70000c1f5000079f5000070f600000a
:10cf5c0068f8000013fb000011fe0000ff00000049
:10cf6c00d2030000a7050000a7050000140500006f
:10cf7c001505000036050000890500004606000076
:10cf8c00ca0600008a06000045050000c602000023
:10cf9c0046ff00006dfb0000eff700009bf5000062
:10cfac00daf400007bf5000051f70000fef90000f8
:10cfbc0003fd0000f8ff0000ac0200009e0400001e
:10cfcc0012050000890400009c0400002b050000e1
:10cfdc009f0500007406000000070000ca06000050
:10cfec00b20500004f030000f0ff000032fc00000f
:10cffc00bcf8000038f6000032f5000089f500009e
:10d00c0001f700006af9000051fc000034ff000039
:10d01c00c7010000f9030000f8040000e60400005a
:10d02c00e70400004d050000dc0500005806000078
:10d03c00c4060000b3060000ad0500009d0300000f
:10d04c00a200000029fd0000d4f900003ff7000009
:10d05c00d7f50000bff50000e0f60000f3f8000083
:10d06c00b2fb0000a3fe00008301000034040000aa
:10d07c008d05000042050000e404000006050000d8
:10d08c0037050000c205000088060000de0600001f
:10d09c004b06000093040000b10100000afe0000e2
:10d0ac004ffa000044f7000094f500005bf5000017
:10d0bc006ff6000080f800001cfb0000d9fd00009a
:10d0cc0080000000db02000066040000ac040000dd
:10d0dc0054040000ae04000034050000b905000043
:10d0ec0078060000b50600005d0600002105000072
:10d0fc00d1020000b3ff000055fc000044f9000011
:10d10c00f7f60000f3f5000007f600002cf700001e
:10d11c002af90000aefb00004cfe0000df0000000e
:10d12c0079030000b00400009304000053040000d5
:10d13c00bc0400005e050000aa0500005f060000ac
:10d14c00b70600001f0600009a040000040200004d
:10d15c00ddfe00009bfb0000b7f80000f1f60000bc
:10d16c005ef60000b4f60000e6f70000c6f9000019
:10d17c0008fc000057fe0000d30000004403000030
:10d18c00c5040000eb0400008e040000cd04000078
:10d19c003c0500009c050000110600003a0600004a
:10d1ac00c30500004c040000f001000004ff000067
:10d1bc00e4fb000028f900006cf70000c0f600004a
:10d1cc00fcf6000019f80000daf90000f4fb00008e
:10d1dc0049fe0000a300000027030000a304000088
:10d1ec009e0400005c04000049040000bd04000023
:10d1fc00400500009c050000f5050000ae05000090
:10d20c007a0400005402000082ff000084fc00003d
:10d21c00dcf9000015f8000062f7000081f700004f
:10d22c0045f80000aaf9000099fb000096fd0000eb
:10d23c00a1ff0000c8010000b50300007504000048
:10d24c00ed030000f30300002b0400007b0400003e
:10d25c0042050000a5050000b80500003a050000d5
:10d26c00bb03000062010000a6fe0000e3fb00000f
:10d27c00a6f900005bf80000f0f7000030f80000a1
:10d28c0014f9000085fa000052fc000021fe000099
:10d29c001d0000006e020000d9030000e70300002f
:10d2ac008d030000b003000065040000e3040000df
:10d2bc00830500002c06000010060000500500003d
:10d2cc00900300000b01000058fe0000c2fb0000a0
:10d2dc00d8f90000c8f8000072f80000b4f800009b
:10d2ec006ff900009dfa000015fc0000befd000067
:10d2fc00beff0000c701000048030000ba03000095
:10d30c0098030000ce03000048040000d504000080
:10d31c009c0500004b06000071060000be050000d5
:10d32c0025040000da01000027ff000082fc000049
:10d33c004bfa0000d0f800002df8000036f8000081
:10d34c00d4f80000f8f900007dfb00004cfd000053
:10d35c0061ff0000a5010000830300001b04000016
:10d36c00c9030000b8030000f903000065040000c5
:10d37c000b050000cc05000043060000f205000080
:10d38c00d3040000d60200004a000000adfd0000ee
:10d39c0053fb000098f900009ff8000088f800008b
:10d3ac0019f9000005fa000038fb0000b0fc000081
:10d3bc0060fe00004c000000390200006603000013
:10d3cc00850300001d0300000a0300005703000042
:10d3dc00c40300009f04000080050000d905000074
:10d3ec00a10500009a040000ae02000044000000f9
:10d3fc00bafd000070fb0000c5f90000e1f8000068
:10d40c00d2f8000046f9000027fa00005efb00008d
:10d41c00b8fc000057fe0000330000000d020000b5
:10d42c000e030000ea0200008b020000a5020000bf
:10d43c00ff020000a3030000a1040000a2050000ed
:10d44c0051060000340600002e0500004b030000be
:10d45c00e30000005afe0000f9fb000027fa000070
:10d46c000ef90000c2f8000029f90000edf90000e7
:10d47c00edfa00003afc0000b5fd000074ff00005e
:10d48c0066010000ce0200003f030000d90200003c
:10d49c0099020000aa020000dc020000b4030000a4
:10d4ac00be0400008c050000da05000055050000e4
:10d4bc00fa030000e001000063ff0000f3fc000031
:10d4cc00eefa00009cf9000010f9000034f900009d
:10d4dc00d0f90000c0fa0000e3fb00003cfd0000a6
:10d4ec00d7fe0000b00000004d020000e702000073
:10d4fc009b0200005202000064020000990200002e
:10d50c0057030000750400007805000006060000b3
:10d51c00bd05000089040000840200001d0000000d
:10d52c00a7fd00007bfb0000f4f900002bf90000c4
:10d53c002af90000aff900007bfa000093fb000011
:10d54c00edfc000072fe000054000000030200001d
:10d55c00f0020000d90200006a020000650200001f
:10d56c0056020000ea020000090400000305000056
:10d57c00c7050000be050000e10400003e030000ea
:10d58c00f400000081fe00003efc000093fa000055
:10d59c0097f900004ef90000abf9000053fa0000b7
:10d5ac0029fb000039fc000072fd0000fbfe0000ae
:10d5bc00ce0000004a020000b30200002c02000062
:10d5cc00bd010000530100003a01000022020000de
:10d5dc00530300009304000095050000e4050000cf
:10d5ec0039050000a00300008c01000038ff00008a
:10d5fc000bfd00004afb000038fa0000c2f90000e5
:10d60c00d3f900005dfa000017fb0000fafb0000e4
:10d61c0008fd000062fe000015000000c5010000be
:10d62c005202000008020000ca0100006d01000057
:10d63c00300100005f0100005f020000ae0300003b
:10d64c00b7040000840500007c0500009b0400006a
:10d65c00210300004e0100004cff00005bfd0000a8
:10d66c00c3fb00009ffa000018fa000000fa00004b
:10d67c0068fa00002afb000029fc000065fd000090
:10d68c00d7fe0000b3000000fe0100002a020000db
:10d69c00dd0100003f010000a80000006b0000004d
:10d6ac009b0000005c010000a902000005040000c2
:10d6bc000705000064050000f7040000f2030000f9
:10d6cc0060020000880000009dfe0000defc0000ef
:10d6dc008ffb0000b3fa00005ffa00007bfa000039
:10d6ec0009fb0000d7fb0000defc00000dfe000073
:10d6fc007fff0000d90000007601000061010000ee
:10d70c0013010000b60000003f00000024000000e0
:10d71c00720000002e010000580200007a03000085
:10d72c004c040000d3040000d904000029040000bc
:10d73c000303000087010000ccff000016fe000070
:10d74c0092fc000054fb000093fa000066fa000003
:10d75c00aafa00006afb00006dfc000086fd0000c8
:10d76c00e0fe00003e000000320100006a010000f3
:10d77c002b010000cb000000680000001d00000021
:10d78c00ffff0000490000001f0100002002000004
:10d79c003203000041040000f40400002b050000db
:10d7ac00c1040000d30300005e020000a7000000cb
:10d7bc00f6fe000061fd00001dfc000037fb0000c0
:10d7cc00ddfa0000f3fa00005ffb000039fc0000fa
:10d7dc004dfd000081fe0000ecff0000e5000000a4
:10d7ec002b01000021010000ea000000970000005e
:10d7fc003e00000020000000260000004b0000004e
:10d80c00e7000000a10100004c020000070300002b
:10d81c008f030000e2030000d40300003d0300006e
:10d82c00480200000a010000a2ff000038fe0000c0
:10d83c00f3fc0000f9fb000063fb00003dfb000063
:10d84c0072fb0000edfb0000c3fc0000d1fd0000ea
:10d85c0005ff00002d000000be000000db000000f2
:10d86c00d2000000910000004700000006000000fc
:10d87c00daff00001d0000004d0000006d000000ec
:10d88c00f00000007d010000df0100006e020000ce
:10d89c00f10200002c0300004e030000f80200000f
:10d8ac00520200005a01000017000000ddfe0000cb
:10d8bc00b3fd0000bdfc00001dfc0000dafb000005
:10d8cc00f3fb000071fc000034fd000043fe00007f
:10d8dc0083ff00007b000000f4000000ff0000004c
:10d8ec00f3000000b0000000410000002500000023
:10d8fc001a000000100000003b0000006100000056
:10d90c007f000000b5000000ee0000004c0100009c
:10d91c00b40100001202000085020000da020000cf
:10d92c00ca02000075020000e8010000ff000000c0
:10d93c00f7ff0000ebfe0000f7fd000030fd0000db
:10d94c00b0fc000083fc0000a0fc000017fd0000f0
:10d95c00d5fd0000cdfe0000c1ff00005d00000001
:10d96c00aa000000a9000000770000005100000090
:10d97c001b000000070000001f0000003b0000001f
:10d98c00600000007a00000083000000a00000008e
:10d99c00be000000ed0000003c01000095010000fd
:10d9ac000a0200006f0200008602000072020000f2
:10d9bc002802000076010000a4000000b6ff000061
:10d9cc00cbfe0000fffd000069fd000016fd00000d
:10d9dc000dfd000053fd0000defd0000a9fe00005f
:10d9ec007aff0000070000005200000062000000f7
:10d9fc00390000001900000001000000f7ff0000d2
:10da0c001a0000004e0000007b0000009000000097
:10da1c009200000099000000a2000000a700000086
:10da2c00ce0000001901000082010000ed01000091
:10da3c0028020000610200006c0200000e020000cf
:10da4c007f010000c5000000e9ff000019ff000085
:10da5c0062fe0000d4fd000085fd00007afd000090
:10da6c00a6fd00000bfe0000a5fe000046ff000016
:10da7c00bfff0000f8ff0000150000000d000000c3
:10da8c00f0ff0000f7ff0000140000003c00000055
:10da9c007a000000aa000000b5000000bd000000e4
:10daac00bd000000a8000000a30000009c000000c6
:10dabc0091000000a2000000ca000000f00000006d
:10dacc002f0100005a0100004d0100003c01000034
:10dadc00ef000000820000000a00000072ff00004e
:10daec00f6fe00008bfe000033fe0000fdfd000082
:10dafc00fefd000037fe00008dfe0000e7fe00007a
:10db0c0054ff0000a7ff0000ccff0000e2ff000064
:10db1c00e1ff0000e2ff0000d7ff0000d6ff00008d
:10db2c00e0ff0000f2ff0000180000002b000000d6
:10db3c0028000000270000003a0000004900000007
:10db4c004900000048000000510000005400000093
:10db5c004c0000005000000059000000690000005b
:10db6c00800000009a000000d1000000ed000000d1
:10db7c00ed000000cc0000009d00000075000000ce
:10db8c0018000000d4ff0000a7ff00005fff00009a
:10db9c0046ff000042ff000045ff00005eff000052
:10dbac007fff000096ff0000acff0000cdff0000df
:10dbbc00d6ff0000d2ff0000ebff00000b000000be
:10dbcc000d000000300000004c000000430000007d
:10dbdc0060000000660000005f00000044000000d0
:10dbec0036000000410000001c000000180000007e
:10dbfc001a000000160000002700000022000000a0
:10dc0c00150000001300000021000000250000009a
:10dc1c001e0000002a00000012000000e9ff0000b6
:10dc2c00d9ff0000c9ff0000c4ff0000c1ff0000c5
:10dc3c00b9ff0000bdff0000bfff0000bcff0000eb
:10dc4c00c3ff0000c4ff0000c6ff0000c8ff0000b7
:10dc5c00c6ff0000c5ff0000c3ff0000baff0000b4
:10dc6c00c8ff0000e1ff0000e6ff0000edff000030
:10dc7c00fcff0000f8ff0000ecff0000e3ff0000d9
:10dc8c00f4ff0000f0ff0000edff000002000000b8
:10dc9c0003000000fcff0000f4ff0000f6ff000092
:10dcac00f4ff0000feff0000100000001400000054
:10dcbc0026000000310000002800000026000000b3
:10dccc0026000000220000001b00000012000000d3
:10dcdc0023000000410000004f0000005a0000002b
:10dcec005e0000004f0000003b000000330000000d
:10dcfc003a00000048000000410000004300000012
:10dd0c005d0000006600000073000000650000006c
:10dd1c007000000087000000550000007300000038
:10dd2c0048000000200000005d0000001f00000003
:10dd3c004600000061000000300000005e000000a2
:10dd4c004400000033000000300000000d00000013
:10dd5c00300000002600000026000000300000000b
:10dd6c000c0000001c00000002000000f6ff000088
:10dd7c00150000000f0000002a0000001b0000002e
:10dd8c000d0000000c000000e0ff0000daff0000b6
:10dd9c00cfff0000d6ff0000f4ff0000efff0000f3
:10ddac00f7ff0000f7ff0000d8ff0000e0ff0000c5
:10ddbc00daff0000daff0000e7ff0000e9ff0000d7
:10ddcc00f4ff0000f6ff0000f5ff0000f8ff000074
:10dddc00010000000a0000000a0000000e00000014
:10ddec00080000000a0000001300000010000000f2
:10ddfc0012000000140000001d0000001a000000ba
:10de0c0017000000120000001c000000270000009a
:10de1c00240000003400000040000000420000001c
:10de2c0050000000480000004a0000005d000000a7
:10de3c00550000005c000000550000005b00000075
:10de4c00550000004f000000570000003c0000008f
:10de5c0031000000360000003f00000026000000ea
:10de6c00520000005400000050000000e8ff0000c9
:10de7c001400000086000000f9ff000024000000e0
:10de8c001b00000028000000faff0000d6ff000075
:10de9c00200000009dff0000a3ff0000b2ff000067
:10deac0085ff000066ff000063ff00005fff0000bd
:10debc0051ff000063ff00005cff0000cdff00007d
:10decc001700000052000000fd000000c000000020
:10dedc001b00000049000000580000001400000066
:10deec00b9ff0000a8ff00006fff000081ff0000d9
:10defc0065ff00002cff00005fff000030ff0000fa
:10df0c0033ff000040ff000057ff00002eff000011
:10df1c0048ff000037ff000042ff0000b9ff00007f
:10df2c001b00000087000000d70000005e0100000d
:10df3c001e010000510000006d000000ad0000004b
:10df4c003e000000daff0000c7ff0000b2ff000037
:10df5c009bff000075ff000064ff00005fff0000e6
:10df6c0047ff00004bff00003dff00002cff0000ae
:10df7c002cff000024ff000035ff000095ff00007f
:10df8c000400000079000000e10000006c010000ba
:10df9c0094010000e0000000a4000000bb000000a1
:10dfac008100000020000000f7ff0000d3ff0000fc
:10dfbc00c3ff0000a4ff00009dff0000a2ff0000b3
:10dfcc007eff00008bff00006cff00005eff000076
:10dfdc0067ff00006fff000078ff0000d6ff000015
:10dfec008b0000001e010000b4010000270200009d
:10dffc005902000097010000e10000003701000009
:10e00c00f6000000580000001b0000000a00000091
:10e01c00f3ff0000f4ff0000faff0000eeff000029
:10e02c00f6ff0000cfff000099ff000088ff000002
:10e03c0074ff000079ff000082ff0000eeff00007b
:10e04c00930000001b010000f601000052020000ca
:10e05c00d401000092010000a50100004b0100005a
:10e06c009b0000003900000001000000c7ff000009
:10e07c00adff000093ff00008fff000090ff000039
:10e08c007eff00007eff000037ff000023ff000032
:10e09c002fff00002aff00007dff0000adff0000f5
:10e0ac0025000000b90000004d0100001102000025
:10e0bc00190200009c0100009a010000a801000058
:10e0cc0027010000830000002c000000e6ff000088
:10e0dc00b2ff000088ff00006fff000093ff0000fc
:10e0ec0030ff000030ff0000fefe0000b5fe000017
:10e0fc0009ff0000ecfe000010ff000082ff000092
:10e10c00f7ff00005c000000e1000000a00100002f
:10e11c0009020000d0010000cd01000088010000c0
:10e12c00c90000001b00000082ff00006dff000012
:10e13c0012ff00009afe0000d4fe0000affe0000ab
:10e14c0045fe000092fe0000dffe00005bfe0000ba
:10e15c009efe000069ff00003dff000063ff000011
:10e16c009dff000002000000440000006e00000053
:10e17c00940000007100000052000000fefe000040
:10e18c0067fe000050fe0000f2fd0000fafe0000e9
:10e19c0068ff0000b8ff00009c0000001c0000009d
:10e1ac0084000000db00000095ff0000a7ff0000ca
:10e1bc0024ff000001ff0000d2fe0000c4fe00009e
:10e1cc0040ff000010fe000078fe000000fe000082
:10e1dc00e0fd000086fe000066fe00004aff000025
:10e1ec0084ff0000b400000051010000a6010000f3
:10e1fc00120200009d0100002501000083000000b8
:10e20c00c5ff0000f9fe0000b9fd000089fd00000b
:10e21c00d9fc0000e0fc00004cfd0000f4fd000007
:10e22c004dfe000010ff0000e6ff00006c00000037
:10e23c0069010000d1000000c60000004f00000082
:10e24c00c8ff00006aff0000d2fe0000d4fd0000f1
:10e25c0057fd00004afd000008fd000079fd00009c
:10e26c006bfe000075ff000036000000aa020000e3
:10e27c005b030000e40200003e0300008d0100007f
:10e28c0096000000c8fe000075fd0000f6fb0000c3
:10e29c00d7fa00005cfb000085fb0000affd00001e
:10e2ac0080ff00002001000062030000a3020000b8
:10e2bc0050050000db02000017020000d500000032
:10e2cc0082fe00007ffd000016fc000077fb0000c2
:10e2dc0081fa000040fc000078fc000050000000b7
:10e2ec00c8020000800500002d070000f4070000a4
:10e2fc00130600007d0400005301000013fd000014
:10e30c00f0fb00002cf900006ff9000090f9000000
:10e31c000afb000012fd0000afff000062030000ca
:10e32c00c0040000c209000003090000c60a000076
:10e33c00180800002404000076000000b4fa000065
:10e34c008ef8000084f40000aef6000001f7000027
:10e35c0048fd0000b7020000dd080000260e00009a
:10e36c00c40d0000e80d00006d040000ee0100007b
:10e37c00f1f90000ccf2000042f8000078f1000046
:10e38c0019ff00009dfd0000c00500008d06000077
:10e39c008f0700002b080000d4030000a406000027
:10e3ac00a9ff00009dff000071060000e2fa0000ca
:10e3bc006c040000fafd000016fd000077ff000061
:10e3cc00aefa0000b000000001f9000046020000a7
:10e3dc002efd0000110300004b0400004c0b00004c
:10e3ec00c8070000590a0000eb050000aff9000057
:10e3fc009d0500009cf20000d9fb000045fe0000ca
:10e40c0055f700003808000092f700002d060000b8
:10e41c0058ff00001c0500003609000060050000d4
:10e42c001d090000d90000002fff00005f04000050
:10e43c0060f2000036ff000070fa0000cff8000018
:10e44c009308000087fd0000d107000031fc00009c
:10e45c00d0ff0000bcf900006af90000d5060000ee
:10e46c00ce0d0000c90c00007315000079010000ee
:10e47c00e1f7000006020000b8e000001f020000f7
:10e48c001ff80000f0fe00003512000072f60000cc
:10e49c00a510000060f80000cf030000fb03000093
:10e4ac004efa0000a909000095f80000530800007e
:10e4bc003d08000012f20000880800001ff1000067
:10e4cc00aef500000f080000bef4000028090000a3
:10e4dc000efd000008ff000087fc000092fa00000f
:10e4ec00d012000073050000920f0000fd07000021
:10e4fc006ce90000a2fa00003bfa00000eee0000ee
:10e50c001414000059fd000037fc00002a0600001e
:10e51c0013e60000730a000025000000100700003d
:10e52c00a20c000026f4000091000000b4eb0000e7
:10e53c00e40b000089020000b4f40000f4170000a2
:10e54c008bdd0000470500002000000051eb0000af
:10e55c0015150000d3f400003cfc00001302000071
:10e56c00d40c00002e1400006e060000edfe00001e
:10e57c0090e1000018f00000b0130000c2f600009b
:10e58c004f1900005200000007d9000021040000c0
:10e59c0083f20000f4120000381c00004a02000054
:10e5ac0082f300002ee300009df30000ad08000094
:10e5bc00901b0000c30f00002bf4000058e7000074
:10e5cc00fdeb000049020000671b0000900a0000f0
:10e5dc0034f000001ef1000043e90000c803000005
:10e5ec0029230000bf180000de080000b2ef000075
:10e5fc00aadf000046fa00005e18000027090000a0
:10e60c00630200005cf2000032e10000f4fd000047
:10e61c00210c00000b1b0000f20f000034f1000075
:10e62c0097f3000002f40000cfff0000531000002d
:10e63c009b02000010fc0000a9fc0000ceee0000c4
:10e64c00bb090000870e0000b0f700003e0400007c
:10e65c0074ee000094ee0000b30f0000f40900000b
:10e66c0018030000ea050000abf60000e5fb000013
:10e67c00ff25000002080000c4e100001afb0000a6
:10e68c00f8ee0000db0200009213000020f5000001
:10e69c0047f90000100100005d0700008b0400002a
:10e6ac0040030000920100005e0b000061120000ac
:10e6bc007af50000b4f20000e2fb0000b0ff0000ad
:10e6cc00cd0b0000160300000ff000003cfa000018
:10e6dc006809000091000000e4050000faf8000051
:10e6ec00d4fe0000db0d00006bf000000c020000fb
:10e6fc00b10800001ff80000960700003f0300005f
:10e70c0063ec0000dff900007d150000940b0000a5
:10e71c0016fc0000b6fe0000e0f10000b90100009c
:10e72c00a20c000044fb00004b1a00006fe5000037
:10e73c000ee400000e25000011ff00004ef1000059
:10e74c002d0d0000d50d0000a0e4000072fd0000ae
:10e75c00b4160000b5ed0000b8fd00007a12000000
:10e76c002df800009bf600007806000088ff0000e2
:10e77c0078f90000880200001204000044fa00003e
:10e78c005bff0000d0030000c2fa000064ff000031
:10e79c006efa0000d3020000db00000077120000cc
:10e7ac00780b000045cb0000420300003a1f00002c
:10e7bc0030f800008ef6000065fe0000120200002a
:10e7cc0068f400001d0e0000e310000022e80000b9
:10e7dc0040ff00008a15000066fe000011010000d9
:10e7ec005df200008df10000e5080000e909000071
:10e7fc0021fe00006ef0000001050000d2090000af
:10e80c00aaf80000d6fa0000f4fa0000d5000000c7
:10e81c0085040000f0110000b0f600006add000075
:10e82c00880e000007110000bdf90000fef5000085
:10e83c00aff90000f80000006f000000830d00002d
:10e84c007b05000009eb0000570500005610000086
:10e85c001d0600004602000066de000015f70000f1
:10e86c00d61600007709000038f20000d6ed000043
:10e87c00560f0000d60a00009bf5000040f900007e
:10e88c0060fa000059010000e3090000cd0200000d
:10e89c004cf60000fff300005e060000340b000095
:10e8ac0003fb000090f6000050fa000097040000f3
:10e8bc00d503000065fc000059ff000098fc000027
:10e8cc0083ff0000fc03000020110000e0fc0000ae
:10e8dc00f4dc00006e060000ef1b0000420100009b
:10e8ec0051e8000074f20000f60c00002405000052
:10e8fc009f050000050100007bfb00004f0300009a
:10e90c00c3130000de0b0000e7dc000084e900000c
:10e91c00231400003614000084f700004af10000b4
:10e92c00f10100002c02000047060000a5070000c2
:10e93c009df70000adf000002e000000fa0e000064
:10e94c00e70400001cf40000e2f700009907000047
:10e95c00f50700001dfd0000c1f90000c3fc00001c
:10e96c00e4ff0000f30100003c0300005aff00002c
:10e97c00f2fb000070ff0000f90a000044040000e4
:10e98c0035f00000a0fa00009a0d0000b00a00005b
:10e99c00b1f800002ded0000c0fe0000bf0a000021
:10e9ac006d020000ae01000066fe0000a413000022
:10e9bc0024110000e0ee0000a5ec0000d4f90000ea
:10e9cc00b8100000b00700003ced0000ccf20000d5
:10e9dc00fe0a0000a9190000130700004bf200000a
:10e9ec0041f80000100100007207000073040000e1
:10e9fc0095f80000c5fa000013ff00004904000060
:10ea0c00490700009ffd000031f90000c9fd00001e
:10ea1c007a0500004c05000042fb000032fd0000ae
:10ea2c00a902000067fd000063fd00004702000022
:10ea3c00bf05000061010000e8f80000c6fb000003
:10ea4c00d0020000ba020000c4fe00004dfc000021
:10ea5c00d201000030010000d8020000580c000068
:10ea6c0076fa000088ef0000e4fb0000f50c0000d3
:10ea7c00fc0f0000eaf6000081eb000033fb000005
:10ea8c00d90f00009e1000001efd0000e0f70000f2
:10ea9c00f0080000bf0a000065f70000ddec000084
:10eaac00a1fb0000fc1000002a0800001af3000073
:10eabc0033f80000930d000022140000cff7000083
:10eacc007ee400000afe000076160000990f00009c
:10eadc0030f200007feb00008e04000036140000c2
:10eaec000909000064ef000007ed0000ad04000010
:10eafc00301300006b0800003ef6000097f7000092
:10eb0c00540400000405000064fc0000f0f900004f
:10eb1c004b0100003a080000470300002afa0000ed
:10eb2c0001f8000061ff0000780600009e02000062
:10eb3c0000fe0000a2fb0000c5080000300d000024
:10eb4c001cfa0000f3ef000043f6000099090000e6
:10eb5c006e0f00009e01000064f300003df5000004
:10eb6c00ad0600005c0e00004a070000b1fa000080
:10eb7c0071f600008c020000ca070000acfe000019
:10eb8c00eff6000021fa00007106000028070000d3
:10eb9c005afb000060f6000078fe00002f0b00000e
:10ebac007c0a000042030000c6fd00004cfa000085
:10ebbc0022fd00004efd000069fd00004602000031
:10ebcc0072060000440600009dfe000023f70000c2
:10ebdc002df9000045000000a8040000ae04000060
:10ebec000102000008fe000023fb0000ccfc00002a
:10ebfc00f0020000210600009802000053fc000007
:10ec0c00dcfb0000550000008e020000f601000045
:10ec1c0055fe0000d4000000b10500000c020000fd
:10ec2c005bfb0000b8f70000bbfe0000dd07000036
:10ec3c006e060000b1fd00005ff700008dfc0000c7
:10ec4c00ce050000130a0000c6050000fafc000007
:10ec5c0075fb0000a9ff0000c60200001cff0000ad
:10ec6c003ffa000013fc0000bb0200000c06000081
:10ec7c006902000075fe0000ecfd00002902000096
:10ec8c00d80400002c0300007a0200001e010000d2
:10ec9c0008fe00006af80000ccf900002c0500000a
:10ecac00d80a0000ab03000041f6000055f5000047
:10ecbc00670100000e0b0000c5070000ccfa000035
:10eccc0059f6000044fe00008f060000b00500005d
:10ecdc0046ff00007ffd0000c4ff0000dbff0000ca
:10ecec000bff0000250100007504000098030000d4
:10ecfc00bdfc0000a4f80000a6fb0000b803000057
:10ed0c002d0700005601000029fc00005efa0000ef
:10ed1c00cb040000f6080000f2fd000039f70000fb
:10ed2c0017fa000066060000ea0900000e01000058
:10ed3c00e6f70000c1f9000080050000ed080000b6
:10ed4c00ed0200008dfa0000c1f900005d04000026
:10ed5c005c060000fefc0000cbf600006ffb000020
:10ed6c0026070000a406000065fb000024f7000045
:10ed7c0079ff00003b0b0000ad090000d60200003b
:10ed8c0049fd00005efa000065fd00002ffd00004b
:10ed9c00b3fd0000b8020000a3060000e40500006b
:10edac00c5fd0000e9f60000b5f90000d400000034
:10edbc00d204000087040000ac010000b5fd000087
:10edcc0011fb000038fd000071030000120600006a
:10eddc000c020000f2fb00002ffc0000a50000005c
:10edec00a2020000b601000029fe0000660100002e
:10edfc00b80500007d010000d0fa0000dbf7000030
:10ee0c00b4ff000035080000dc050000ddfc00004c
:10ee1c0057f7000060fd00006f0600000e0a0000ae
:10ee2c00e1040000bffc00005dfc00001d000000c0
:10ee3c00a90100003dfd000019fa0000d5fc0000fe
:10ee4c003b0200009d050000430400004f01000040
:10ee5c00bdfd000037ff0000f90400007e07000034
:10ee6c005204000044fc00003cf7000037fa00009c
:10ee7c00ea010000ff06000069050000b5fe000075
:10ee8c00e7f80000baf9000047ff00007a0600001e
:10ee9c000208000007020000e3fa0000b1f80000cd
:10eeac0035fe00006e050000da060000dc000000f4
:10eebc00e5fa000011fc0000d60200005a08000020
:10eecc007b06000062fd0000c3f50000e6f70000c1
:10eedc00f3000000d0080000a707000063ff00004b
:10eeec0070f90000a0f70000b7fb0000da03000087
:10eefc00c10800005f060000f9fe000059fb00008d
:10ef0c001dfe0000dc030000cb06000071030000b6
:10ef1c009ffc000003f6000095f60000b7fe000011
:10ef2c0072060000840700003300000018f800008f
:10ef3c00cdf700002eff0000bd06000052090000b6
:10ef4c00cf0400001bfe000036fc00000100000096
:10ef5c0028050000f7040000d6fe000007f70000ab
:10ef6c00c0f400001cfb00008204000088080000b4
:10ef7c004304000036fc0000d7f9000084fd0000bb
:10ef8c0087020000c6040000dbff0000b7fa000097
:10ef9c00e7f90000d2fd0000ad03000019050000e8
:10efac000d03000007ff000009fc000053fd0000ea
:10efbc0035010000aa050000c6050000b8000000dd
:10efcc00e5f9000062f60000ddf80000d2fe00005a
:10efdc001805000017050000430000008bfc000022
:10efec004efa000047fc00006c0100004a060000cd
:10effc003209000031070000ec020000b2fe0000f4
:10f00c008cfa00004bf80000a4f8000023fb000071
:10f01c00d7fe0000730300003c0600004204000011
:10f02c0046ff00007df90000abf9000087ff0000ef
:10f03c006b0400003d0600004103000008fd0000c9
:10f04c0054f7000071f600002ffc00004c04000087
:10f05c009a090000af0900000104000037fd000010
:10f06c00edf8000091f900004aff000032040000a6
:10f07c007f060000f50300006ffc00005bf600004b
:10f08c003ff50000f1f90000c9000000ec0600009b
:10f09c0032080000a803000001000000b7fd0000ca
:10f0ac0059ff00006f0400003407000057050000f2
:10f0bc0064fe00000ef70000f4f2000080f4000083
:10f0cc001efc00003e050000a70b00001a0c0000ff
:10f0dc00060600004dfc000053f500001ef6000073
:10f0ec0087fc0000f8030000d40700008f05000027
:10f0fc0058ff000034f9000062f6000037f80000f9
:10f10c0012fe0000df060000840c0000de0b000085
:10f11c006106000095fe0000e6f9000025f90000ec
:10f12c0017fb00008dfd000029ff000022ff0000ee
:10f13c000bfe00005afe00001fff0000a2000000a2
:10f14c00d90100009f0200007e0200005a0100005d
:10f15c0052010000cc0000009eff0000edfd0000fd
:10f16c0000fc000043fb0000a0fc00007cfe000043
:10f17c00610000000a030000b1040000a7040000b5
:10f18c0048030000f7010000ac0000002aff00005b
:10f19c002efe000099fd0000edfd00008cfe00002d
:10f1ac00effe0000caff00001a000000c5ff0000bf
:10f1bc00fafe000088fe000054ff0000420100002f
:10f1cc00fe0300007b050000bc040000b30100003e
:10f1dc007dfd000026fa000090f80000faf900000e
:10f1ec0031fe0000bf0200009e050000ce050000ad
:10f1fc008f030000f6ff00000cfd00008bfb0000ed
:10f20c0049fc0000f6fe0000740200006a060000d3
:10f21c001a0900006109000081060000e4000000ea
:10f22c000afa000049f40000faf10000e1f30000d2
:10f23c0019fa000041030000760c0000d811000000
:10f24c00a910000076090000f5fe000078f500001a
:10f25c0005f000004bf1000051f800004a010000dd
:10f26c0010080000a90a00006e080000e20100006e
:10f27c006dfc00003bf8000032f70000e0fb0000e2
:10f28c00a6030000810c000049120000f4110000dc
:10f29c00b30a000039fe00006ff100009ce800008a
:10f2ac0018e700008ded000083f9000067070000ef
:10f2bc00d81200001a180000c1140000a80a00009f
:10f2cc00ccfd0000c5f200004fed00008fee0000f9
:10f2dc00a0f5000066fe00006e050000700800003e
:10f2ec002f0700003203000045ff00002ffd000037
:10f2fc0035fc000020fe0000100200009306000008
:10f30c00f5090000930900005f060000970000005b
:10f31c005af90000b6f2000091ee000087ef0000f1
:10f32c006cf500006efe0000ec070000860e00007d
:10f33c00d6100000570e000059070000dafd00003f
:10f34c00b9f50000adf20000b5f4000061f9000061
:10f35c007afe0000ab010000330200000f01000038
:10f36c00fcff0000fbff00004600000061020000f3
:10f37c00460600007b090000f60a00002109000087
:10f38c00900400001bfe0000c7f60000c8f000004f
:10f39c00e7ed00004df00000e2f60000d3ff0000a6
:10f3ac0047090000f60f000086120000cf0f000086
:10f3bc006c080000f0fe0000d0f60000eef2000039
:10f3cc008df30000a1f700003efd0000df010000fe
:10f3dc00fc030000690300007901000057000000e5
:10f3ec00d9ff0000e5000000010400006e070000da
:10f3fc00560a00009d0a000046070000300100007c
:10f40c001afa0000f8f30000ebef000074ef0000b4
:10f41c00f5f200002cfa000077030000610b0000ed
:10f42c000d100000871000000d0d00006406000098
:10f43c00bdfd0000d7f60000d5f30000a5f40000d8
:10f44c0005f8000028fc0000a0ff000015010000da
:10f45c00680100007c010000a901000032020000dc
:10f46c00bf030000a30600005a0900006b0a00004d
:10f47c008f080000ea03000058fd00006af6000047
:10f48c0034f10000fbee000071f0000090f500007c
:10f49c00c7fd0000960600008a0d000068110000f0
:10f4ac00f8100000520c000087040000effb000075
:10f4bc00b6f500004df3000096f400004bf8000088
:10f4cc00cefc00007b0000001e0200003702000092
:10f4dc002a0200007c020000cd0200001c04000087
:10f4ec009a060000c50800007e090000e70700002e
:10f4fc00f5030000d9fd00003cf7000043f20000ca
:10f50c0001f000001bf100007af50000cffc0000b8
:10f51c00410500009c0c000012110000fb100000c3
:10f52c00e50c0000d7050000b0fd000037f7000027
:10f53c00f6f3000036f400002cf7000080fb00000e
:10f54c00bafe0000230000009b00000087010000b1
:10f55c00c20200001303000076040000d006000075
:10f56c001f090000390a00001f0800008f0300006b
:10f57c003afd000061f600000af100007cee00008c
:10f58c0090ef000011f40000cafb0000b904000069
:10f59c00e80b00002910000071100000070d00009e
:10f5ac00820600009cfe000034f80000aaf4000063
:10f5bc0040f400001ff6000073f90000b7fc0000d7
:10f5cc0097fe000096ff00005f000000e0010000c5
:10f5dc004c03000092040000cf060000b8080000a5
:10f5ec007a090000110800002704000095fe0000b5
:10f5fc0021f80000cef2000004f0000027f000001b
:10f60c0035f3000018f900001a0100007f08000013
:10f61c00990d0000860f0000ed0d00008709000019
:10f62c001703000066fc000070f700005bf500009b
:10f63c00a1f50000a6f7000094fa0000cefc000033
:10f64c006afe0000baff000053010000070300002f
:10f65c0083040000f30600009f0900002f0b00003c
:10f66c00860a00000a0700007e010000a9fa0000cb
:10f67c001cf40000c5ef0000acee000024f100000b
:10f68c00a0f6000091fe0000d5060000020d00005f
:10f69c0051100000f60f0000450c0000d7050000cb
:10f6ac0089fe0000c7f800008ef50000faf4000097
:10f6bc0074f6000067f900003dfc000003fe00003a
:10f6cc004bff0000aa0000008f0200002a0400007b
:10f6dc00e90500004a080000060a00002d0a000097
:10f6ec00d40700001e030000ebfc00005cf60000d9
:10f6fc0084f100007bef00007ef0000061f400005c
:10f70c0009fb000029030000020a0000560e00004d
:10f71c005d0f0000170d000035080000a601000069
:10f72c0055fb000011f700008cf5000004f60000fa
:10f73c000ef80000a5fa00009dfc00004cfe000035
:10f74c00d2ff0000a10100007c030000770500003f
:10f75c0058080000f30a0000cb0b0000140a00004c
:10f76c00c305000096ff00008bf8000070f200004b
:10f77c0015ef00002def0000bdf20000f7f80000bf
:10f78c00fa00000092080000de0d0000641000007a
:10f79c00770f0000900b000058050000aafe000037
:10f7ac007bf9000066f6000077f500006df60000ae
:10f7bc00e9f8000062fb000036fd000013ff0000ba
:10f7cc003c0100008d030000be0500001b0800007a
:10f7dc00b10a00003e0c00006c0b0000dc070000be
:10f7ec00e8010000b7fa0000faf30000a7ef0000f0
:10f7fc00a5ee0000d7f000000ff6000089fd000018
:10f80c00650500007a0b0000f20e0000880f000066
:10f81c003f0d000052080000da01000013fc00004c
:10f82c000ff80000ccf500007af50000bdf60000e2
:10f83c00c2f80000fbfa000077fd00004600000053
:10f84c00d60200003d050000fa070000d80a0000af
:10f85c00d40c0000650c00006209000019040000c3
:10f86c0045fd000083f600004bf1000029ef00007d
:10f87c0043f0000031f400008cfa0000c5010000d8
:10f88c00610800003f0d00008c0f0000070f000006
:10f89c009a0b0000110600003900000040fb00002c
:10f8ac007cf700006bf500005cf50000d5f600005d
:10f8bc00eff8000087fb0000aafe0000b201000078
:10f8cc0098040000960700008a0a0000010d000051
:10f8dc00820d0000410b000074060000ebff0000dd
:10f8ec0026f9000057f30000c0ef000054ef0000b1
:10f8fc00d7f10000e3f6000081fd000025040000b4
:10f90c00c30900007d0d0000030f0000e70d00008f
:10f91c00190a0000ee0400008dff0000aefa000092
:10f92c00e1f60000acf4000085f40000f8f50000ee
:10f93c0034f8000025fb00008cfe0000f1010000f3
:10f94c0065050000f8080000400c0000340e0000b3
:10f95c00b30d0000720a0000f404000005fe000064
:10f96c0020f70000b8f10000e5ee000012ef0000f7
:10f97c001df200009df7000069fe00000705000065
:10f98c002b0a0000850d0000cd0e0000640d000058
:10f99c00910900008e04000066ff0000bdfa000013
:10f9ac0018f70000faf4000081f400003df50000a7
:10f9bc000af70000d5f9000054fd00002b010000ef
:10f9cc0047050000c5090000ab0d00006b0f0000df
:10f9dc00630e0000710a00006a04000077fd00004d
:10f9ec008df6000034f1000092ee0000ddee000018
:10f9fc00fcf1000068f7000004fe00007f0400002a
:10fa0c00d1090000ae0d0000420f0000c20d000035
:10fa1c00250a000087050000740000009cfb000014
:10fa2c00acf7000034f5000053f400008cf4000037
:10fa3c00eff500008af8000015fc00004b000000f8
:10fa4c00a6040000be090000810e00009c100000fe
:10fa5c009b0f0000b60b00007c0500001bfe000095
:10fa6c0015f7000094f10000e5ee000041ef0000f6
:10fa7c001df200003af700007bfd0000a803000017
:10fa8c00be080000950c0000930e0000d70d00007e
:10fa9c003b0b0000960700003f030000adfe00008a
:10faac0048fa0000fcf600000cf5000038f40000e9
:10fabc00d0f40000d8f600000efa00004dfe000055
:10facc001d030000e6080000710e00002a11000062
:10fadc00b4100000780d0000f0070000e7000000f3
:10faec00dff90000f6f3000037f0000060ef0000d3
:10fafc0008f1000013f50000aafa0000b2000000a3
:10fb0c001b060000910a0000d60d0000590e0000e3
:10fb1c00650c0000350900002c050000c600000033
:10fb2c003cfc00005af80000a6f5000025f400008b
:10fb3c00ecf3000039f50000d0f700008efb00005c
:10fb4c0025000000780500006a0b00005e0f000025
:10fb5c0078100000f70e0000980a00006d040000f9
:10fb6c0062fd0000bff60000c2f1000075ef00005e
:10fb7c00e0ef0000abf2000090f7000062fd000027
:10fb8c001103000007080000f40b0000f00d00004a
:10fb9c004c0d0000140b0000d8070000b00300004f
:10fbac0039ff0000d7fa000062f7000025f50000cd
:10fbbc0007f4000071f400005bf6000088f9000007
:10fbcc00d0fd0000bd020000be080000600e000069
:10fbdc00de100000621000004c0d0000d507000084
:10fbec00fd0000000efa00002bf4000081f0000074
:10fbfc00adef000053f1000058f50000defa0000f4
:10fc0c00cc000000170600008c0a0000c20d00009a
:10fc1c00150e0000140c0000ed080000fb040000a1
:10fc2c00ac00000034fc000066f80000b0f50000e9
:10fc3c000cf40000baf300000bf50000aaf700006a
:10fc4c0083fb000044000000160600005f0c00005f
:10fc5c00c70f000056100000800e0000ce090000f7
:10fc6c00a8030000cafc000069f60000d8f10000ef
:10fc7c00e3ef000066f0000025f30000e1f7000060
:10fc8c0043fd000072020000490700003f0b00001a
:10fc9c00310d0000b40c0000040b00004d080000f6
:10fcac006e0400002d000000d0fb000017f80000cf
:10fcbc0055f50000a3f300009cf3000031f50000a3
:10fccc0016f800005cfc00006e010000ce0700007e
:10fcdc00c40d0000ee0f0000ba0f0000610d000013
:10fcec00710800008002000009fc000051f60000c1
:10fcfc0098f20000f1f0000088f1000039f40000e7
:10fd0c0056f800004efd00003202000024070000ef
:10fd1c00670b00002c0d0000d70c0000140b00002a
:10fd2c002a08000054040000c1ff00002efb000054
:10fd3c0049f7000075f40000fbf2000028f3000006
:10fd4c00e0f4000021f80000abfc00001102000000
:10fd5c0096080000820d0000080f0000910e0000b4
:10fd6c00a50b0000d5060000480100004ffb000069
:10fd7c004df600001cf30000b1f100004cf2000045
:10fd8c00baf4000086f8000018fd0000b301000072
:10fd9c00bf060000240b0000d40c0000cf0c0000a8
:10fdac00a60b0000a008000069040000c1ff0000c1
:10fdbc0003fb0000f8f600005cf4000014f30000f4
:10fdcc0076f3000068f5000090f80000e8fc0000f5
:10fddc00f901000039080000220d0000b90e0000e6
:10fdec00810e0000e00b00007007000049020000cb
:10fdfc0088fc0000a9f7000054f40000bbf20000de
:10fe0c00fdf20000c9f4000001f800002bfc00001a
:10fe1c006b00000071050000770a0000dc0c00008c
:10fe2c00aa0d0000df0c0000bb09000098050000c3
:10fe3c00b0000000c9fb0000a6f70000cef40000e3
:10fe4c0084f30000c8f30000a3f500007af800006a
:10fe5c006bfc0000c50000005a060000e30b00001c
:10fe6c00f90d0000940e0000dc0c0000b808000036
:10fe7c0036040000d9fe0000d0f9000022f6000084
:10fe8c00d7f3000058f3000078f40000ecf6000003
:10fe9c0068fa000038fe0000c502000048080000a7
:10feac00930c0000dc0d0000620d0000520b0000f2
:10febc006b070000bf0200009cfd00000df9000064
:10fecc00b7f50000d5f30000b1f30000def400003c
:10fedc003cf7000092fa00006ffe0000fd020000eb
:10feec00c70800009d0c0000b20d0000cd0d0000f5
:10fefc00540b00001d07000025020000b1fc00009f
:10ff0c00f2f70000b3f4000011f300004bf3000013
:10ff1c000ef50000dcf700008bfb00006eff00000c
:10ff2c00c9030000ec080000a40c00009d0d0000ab
:10ff3c00200d0000890a00003e060000930100001d
:10ff4c0061fc0000daf70000e6f400006cf300003e
:10ff5c009cf3000044f5000014f800005ffb000067
:10ff6c0009ff00005c030000500800007e0c00003c
:10ff7c00fa0d0000b50d00005f0b0000f00600004c
:10ff8c00eb0100007cfc0000bef7000073f40000e5
:10ff9c00f1f2000064f3000064f5000088f8000042
:10ffac0010fc0000b9ff0000cc030000f2070000b9
:10ffbc00880b00008d0d0000650d0000510b00003a
:10ffcc00aa070000dc02000099fd0000d2f8000036
:10ffdc003df5000063f300007cf3000014f5000015
:10ffec00b6f7000020fb0000a3fe00005902000041
:10fffc00a3060000dc0a00008b0d0000fc0d0000c5
:020000040001f9
:10000c00860c0000180900005c040000dafe0000f9
:10001c0076f9000069f50000f5f200008df20000a1
:10002c0028f40000eff6000093fa00005efe0000da
:10003c0007020000f7050000c5090000940c000041
:10004c00770d00005c0c00008e09000057050000c5
:10005c004100000011fb0000c8f60000f1f30000a5
:10006c00fdf20000f0f300002bf600005ff9000039
:10007c0006fd00008c00000049040000710800001f
:10008c00190c0000e80d0000830d00001c0b000093
:10009c0010070000dd01000024fc000035f7000013
:1000ac00c8f300002bf20000d7f2000032f500007c
:1000bc008ef8000092fc00004e000000e9030000e6
:1000cc00ad070000030b0000ea0c0000e40c00007c
:1000dc00180b0000a707000016030000defd00004f
:1000ec00f9f8000041f500001ff3000003f30000d5
:1000fc009df400006bf7000005fb0000b3fe000050
:10010c0015020000b1050000bf090000e30c00005f
:10011c00fa0d0000c70c0000b10900002b0500000f
:10012c0090ff000005fa000075f500008bf200004e
:10013c00c6f1000024f3000013f60000ecf90000f7
:10014c0003fe000099010000f104000059080000b2
:10015c000f0b0000740c0000320c0000150a00009c
:10016c00a60600003702000037fd00009df80000d5
:10017c0010f5000026f3000011f30000bef400009f
:10018c00b2f700004efb00000dff00007b020000e8
:10019c0004060000ef090000ec0c0000a70d0000a5
:1001ac00620c00006909000002050000acff0000b1
:1001bc002afa0000b7f50000f2f2000032f200005b
:1001cc0080f300006cf6000040fa000049fe0000cd
:1001dc00c0010000e404000006080000be0a000094
:1001ec00560c0000f30b0000160a00001407000068
:1001fc001603000054fe0000b2f900002af60000bd
:10020c00f5f30000a9f30000eff4000068f700001c
:10021c00e2fa000073fe0000c90100001e05000098
:10022c00f8080000470c00003f0d0000660c0000b1
:10023c00d4090000df05000039010000fafb0000c2
:10024c0089f70000adf4000076f30000f8f300002d
:10025c0004f6000017f90000bcfc00004000000090
:10026c00420300006e0600009f090000e60b000030
:10027c00790c00003b0b000085080000c204000054
:10028c0046000000b0fb0000d2f7000039f500007a
:10029c002df400009cf4000072f600006bf90000d5
:1002ac00d9fc00000c00000034030000cb06000059
:1002bc00540a0000660c0000be0c0000490b000044
:1002cc001d0800001904000044ff00007dfa000026
:1002dc00d6f6000086f40000d2f30000d2f4000041
:1002ec0023f7000063fa0000ccfd0000f6000000cc
:1002fc001204000060070000a60a0000100c0000a9
:10030c00e40b00006b0a00004107000071030000c1
:10031c0000ff000096fa00002ef7000019f500000f
:10032c004ff4000018f500003ff7000032fa00000f
:10033c0092fd0000cb0000001f040000ce0700005f
:10034c00400b0000a80c0000360c00006e0a0000e8
:10035c001c0700003a030000bafe000074fa00000b
:10036c0052f7000047f50000b5f40000a6f50000b8
:10037c00fbf70000edfa000019fe0000340100004c
:10038c00490400001c080000190b0000550c00006b
:10039c001d0c00000c0a0000da060000ee02000042
:1003ac006afe000043fa00001ef7000025f500006d
:1003bc00a6f40000a8f50000f1f70000defa00003a
:1003cc00f3fd0000000100004e04000029080000ad
:1003dc00ee0a0000fd0b0000650b00004609000052
:1003ec0069060000910200003bfe000052fa00007a
:1003fc0039f7000035f500009cf4000090f5000082
:10040c00c1f7000082fa000091fd0000aa00000074
:10041c00320400002a080000c70a0000f10b00009b
:10042c002b0b0000f1080000320600005602000001
:10043c002ffe000045fa00001ef700002ff500000b
:10044c008ef4000074f5000081f7000027fa00001c
:10045c002cfd000046000000f5030000ff07000023
:10046c00980a0000970b0000f20a0000c208000076
:10047c00e20500002d0200000dfe00003dfa000018
:10048c0023f700002cf500008ef400004bf5000063
:10049c0044f70000e4f90000cdfc0000e6ff00008a
:1004ac00cf030000d6070000490a0000740b0000bf
:1004bc00a00a0000dd08000075060000b002000074
:1004cc009cfe000093fa000044f700001cf50000ad
:1004dc005af4000019f5000010f70000cef90000e6
:1004ec00eefc000014000000c2030000ac0700008a
:1004fc006c0a0000ab0b00001c0b0000780900001c
:10050c00d0060000fd020000cffe00009efa0000a5
:10051c003ff7000021f500004ff4000019f5000032
:10052c000ff70000d0f9000006fd00002d000000c0
:10053c00e1030000dd070000e30a00000f0c0000df
:10054c00820b0000b3090000b2060000f2020000aa
:10055c00a1fe00008bfa000063f700004ff50000cd
:10056c00a5f4000083f50000b4f700007dfa00004c
:10057c0096fd0000b00000000b040000fe07000018
:10058c00bc0a0000fa0b0000d60b0000c6090000e4
:10059c00b1060000d40200005afe000045fa00002b
:1005ac0018f700001df50000a7f40000abf50000e3
:1005bc00f7f70000e0fa0000f4fd0000080100006d
:1005cc00790400005d080000030b0000ef0b000035
:1005dc00380b0000100900001c060000230200006c
:1005ec00cafd0000f7f90000f9f6000010f5000054
:1005fc00a6f40000c0f5000003f80000cffa0000dc
:10060c00e5fd0000fe0000009d04000085080000d0
:10061c00fd0a0000f90b0000f50a0000b308000009
:10062c00da050000e2010000bffd0000e6f9000061
:10063c00def600000df5000093f40000a2f50000ba
:10064c00c0f7000072fa00007dfd00009d00000064
:10065c006504000058080000c70a00009f0b00004a
:10066c00c30a00007c0800008c050000bf010000dc
:10067c009efd0000def90000e1f600000af5000026
:10068c0090f4000076f5000084f700002dfa0000cd
:10069c001dfd00003e000000460400002a0800007a
:1006ac00760a0000700b0000530a0000840800005a
:1006bc00060600003002000028fe00003ffa000091
:1006cc0017f7000015f5000072f4000043f5000068
:1006dc003ef70000e1f90000f3fc000017000000f9
:1006ec0008040000fe070000710a00008c0b0000db
:1006fc00b10a0000ff0800006f0600009302000022
:10070c0083fe00006efa000026f7000011f50000d1
:10071c004ef400001ef50000fff600009df90000ed
:10072c00aefc0000c8ff0000d9030000ef0700007a
:10073c00820a00007d0b0000c70a000002090000bd
:10074c0055060000b7020000b1fe0000c2fa00001e
:10075c008ef7000061f5000078f4000024f500002d
:10076c00faf600006df9000052fc00006bff00006f
:10077c0034030000350700009a0900001d0b00002f
:10078c005e0b0000870900000e0700009c030000b0
:10079c004fff000040fb0000bdf7000066f50000b5
:1007ac0065f40000dcf40000baf600002af9000041
:1007bc00fefb00001cff0000e4020000100700001c
:1007cc00bf090000f60a0000250b0000d909000043
:1007dc0076070000450400003d00000033fc0000db
:1007ec00b9f8000027f60000f9f4000032f500001b
:1007fc00d3f600003ef90000fdfb0000d8fe00001f
:10080c00490200005406000045090000fa0a0000e5
:10081c008e0b0000700a000077080000be05000077
:10082c00d7010000c9fd00001cfa000029f70000e8
:10083c007bf5000029f500005af6000072f8000064
:10084c0008fb0000f4fd0000260100002f0500004d
:10085c0073080000730a00007a0b0000840a000081
:10086c00e808000093060000f5020000f8fe000006
:10087c001afb0000eef70000e4f5000016f500008e
:10088c00d1f5000093f70000e6f90000bafc000077
:10089c0096ff000044030000e30600001c09000062
:1008ac00c30a0000ae0a0000040900003e07000065
:1008bc005704000080000000c3fc000059f9000040
:1008cc00d4f600006cf5000067f50000aff60000f0
:1008dc00cef800006cfb000026fe00007f0100003b
:1008ec002005000032080000ee090000810a00001b
:1008fc00ef0900004308000027060000d8020000a2
:10090c00effe00004bfb00002bf800001df6000072
:10091c0044f50000f6f50000b9f7000026fa0000d7
:10092c00c9fc0000bcff0000550300006906000074
:10093c0076080000b10900002d0a000049090000ea
:10094c00d107000059050000ac01000005fe0000b5
:10095c004efa000073f70000bcf5000053f50000e0
:10096c0097f60000a1f800002afb0000e8fd00004b
:10097c00f400000066040000e50600008208000098
:10098c009e09000091090000cf0800003607000006
:10099c00860400001701000029fd0000bef90000cc
:1009ac0010f7000091f50000a4f50000d9f6000046
:1009bc00ddf8000076fb000007fe000019010000c6
:1009cc0046040000660600004108000034090000df
:1009dc0064090000c4080000180700009604000019
:1009ec00fc0000003afd0000d4f900001ef70000e6
:1009fc009cf500009ff50000dff60000f4f8000005
:100a0c0081fb000012fe00002e0100003b040000e0
:100a1c0038060000e1070000320900005009000010
:100a2c00840800001b0700009a040000300100003d
:100a3c0062fd0000e9f9000027f7000094f50000c2
:100a4c0097f50000d9f60000d7f8000074fb000001
:100a5c0012fe00003201000033040000d205000039
:100a6c00a8070000d408000004090000a108000039
:100a7c0014070000bd0400004d01000078fd0000cb
:100a8c0016fa000044f70000a3f50000b3f50000cf
:100a9c00e6f60000ebf8000084fb0000fffd000010
:100aac002c010000180400008f0500002307000033
:100abc00a60800000a09000048080000050700000d
:100acc00c204000062010000cdfd00004bfa0000e2
:100adc006ef70000b7f500007ff50000aaf60000e5
:100aec008ff800001bfb0000c2fd0000f5000000a9
:100afc00ad030000a60400006c06000026080000f0
:100b0c00b00800009408000089070000fb050000f5
:100b1c000d03000068ff0000f2fb000099f80000d4
:100b2c0060f6000098f5000038f60000cbf70000e6
:100b3c0026fa0000bffc0000deff000032030000bc
:100b4c0004040000ef040000ed060000fb070000a9
:100b5c00a8080000730800007d070000870500004e
:100b6c0072020000c4fe000010fb000022f800001e
:100b7c0025f60000caf50000b2f6000061f800008e
:100b8c00f0fa0000affd000083010000b303000089
:100b9c00f70300003605000098060000bc070000b3
:100bac00660800007208000092070000ad05000006
:100bbc0076020000abfe000014fb000016f80000eb
:100bcc0047f6000004f60000caf6000080f80000aa
:100bdc0022fb0000f0fd0000da010000ad03000074
:100bec007c030000b8040000bd050000fa060000fc
:100bfc0017080000480800001d08000068060000e7
:100c0c0079030000fcff00001bfc00000af9000047
:100c1c00c8f60000f3f5000055f60000abf7000035
:100c2c0029fa000002fd00001301000099030000e6
:100c3c00cd030000b3030000c50400004006000013
:100c4c00190700007e0800007908000092070000d8
:100c5c00bd0500003e0200007bfe0000d9fa00003a
:100c6c00e8f700002bf60000c1f500006cf6000060
:100c7c0067f800000efb000099fe0000b7020000b0
:100c8c0007040000c3030000380400008b040000bc
:100c9c008f050000fa060000c90700002a080000b2
:100cac0068070000540500004302000071fe0000bc
:100cbc00d6fa0000f4f700002ff60000bff5000094
:100ccc0070f6000066f800003dfb000003ff00001a
:100cdc003a03000050040000160400002e0400002b
:100cec007103000057040000820500009806000004
:100cfc006b070000e2060000d50500006003000051
:100d0c00dcff00005dfc000046f900000ef700005f
:100d1c00fff5000008f6000065f70000cef90000b2
:100d2c002cfd0000e501000022040000030400007b
:100d3c009a030000b0020000610200008f02000064
:100d4c002f040000a8050000920600003c070000dc
:100d5c00ed05000056030000050000006afc0000d1
:100d6c0070f900001ff7000004f6000018f60000f0
:100d7c0053f70000acf9000040fd0000be0100007c
:100d8c00580300003d03000019030000e9010000b6
:100d9c001701000018010000bf0200008e040000c3
:100dac002106000061070000d706000021050000a5
:100dbc005d020000f2fe0000bbfb0000def800004c
:100dcc00eef6000040f6000086f600002ff800005a
:100ddc00bbfa000038ff0000c8020000e20200006d
:100dec002703000078020000860000004f0000007e
:100dfc00060100004b02000013050000ac060000c9
:100e0c001f0700004c07000095050000e3020000de
:100e1c00c3ff00005afc000074f9000080f70000ca
:100e2c0077f6000045f600008cf7000015fa00007c
:100e3c0075fe000010020000910200001703000074
:100e4c00f102000051010000710000004c00000094
:100e5c00a8000000af02000025050000b10600004c
:100e6c00ac0700006a070000d90500006e03000003
:100e7c006200000014fd000013fa0000dcf7000013
:100e8c0090f6000055f600005df70000edf900004b
:100e9c0011fe000089010000200300008203000005
:100eac00c5020000e201000068000000abff00007a
:100ebc005c0000004701000006040000460600002c
:100ecc00e8060000af0700008f0600005904000080
:100edc00da01000083fe00008cfb000017f9000013
:100eec0078f70000a7f6000030f7000024f90000a6
:100efc00d5fc00003b01000063020000bf020000b3
:100f0c00120300006c01000064000000ecff000004
:100f1c00bcff0000200100001903000005050000c3
:100f2c009d0600001d070000ae0600001a0500001b
:100f3c00a3020000a7ff00009afc000012fa0000b8
:100f4c0040f800004ff700007df700000ef900009c
:100f5c006dfc000005000000f3010000f50200002c
:100f6c00a7020000d6010000c2000000b6ff00007e
:100f7c0006000000920000009f0200003b050000ec
:100f8c002206000042070000fd06000033050000a9
:100f9c00540300004f00000046fd00008cfa0000d6
:100fac0063f800002af7000007f7000078f800004b
:100fbc0065fb000010000000360200005c0200001f
:100fcc001b0300009801000050000000bbff000054
:100fdc00d3fe00009dff0000bb0000006b02000070
:100fec00d6040000070600001c0700003e070000a6
:100ffc000c0600002b0400009401000010ff000000
:10100c008efc000072fa0000e2f8000010f80000fc
:10101c007bf80000f7f90000ddfc0000ceff0000bb
:10102c00fe0000009e0100008b010000e4000000a7
:10103c005d00000099ff000079ff0000cdff00006b
:10104c00b60000003e0200006b030000af0400007d
:10105c00a905000000060000f5050000d6040000fc
:10106c0002030000230100000cff0000d1fc000073
:10107c00e5fa000092f900001ef90000aaf9000040
:10108c005dfb0000cdfd000091ff00007d00000025
:10109c001d010000e9000000860000000f000000a8
:1010ac00a8ff0000c7ff0000d5ff0000760000007d
:1010bc007e010000c701000092020000d80300006e
:1010cc002f040000bf040000ec04000040040000ea
:1010dc0067030000c6010000a2ff0000bcfd000079
:1010ec00defb00004afa00008ef9000096f90000c1
:1010fc00abfa00002ffc0000cbfd0000e5fe000069
:10110c007aff00005500000088000000a2000000db
:10111c00770000004c0000003800000099ff000030
:10112c00e5ff00002a00000058000000fd00000050
:10113c005e0100000b020000e40200004f030000ff
:10114c006b0300002b030000780200003401000048
:10115c00a8ff000040fe000007fd0000effb0000b0
:10116c004dfb000053fb0000eefb0000c0fc000038
:10117c0090fd0000b9fe000056ff0000bcff00000f
:10118c00d3ff0000c8ff0000ecff0000b2ff00001e
:10119c003c000000f0ff0000d7ff00009f000000a3
:1011ac0076000000b30000002f010000c101000018
:1011bc000d02000010020000bb0200004003000002
:1011cc000d0300009d020000060200001801000043
:1011dc00f7ff000004ff00000cfe0000bcfc000048
:1011ec0058fc00007dfc00005afc0000eefc0000e6
:1011fc00d5fd000094fe000061ff0000daff000046
:10120c00ebff000033000000820000008a000000a9
:10121c008c000000ad000000c5000000c5000000ff
:10122c0097000000920000007e0000007300000098
:10123c00b9000000be000000e800000060010000e2
:10124c008d010000950100001402000057020000ff
:10125c00cc0100006a0100001e01000047000000e4
:10126c0097ff0000bffe00000afe0000fffd00001b
:10127c008dfd0000bffd0000c0fe000015ff00004a
:10128c0059ff00001d00000051000000b0000000dc
:10129c00270100002c0000009d0000000e01000042
:1012ac009900000018010000c10000003a00000085
:1012bc00470000005f00000081000000cc0000002f
:1012cc00c8000000ba000000d0000000d6000000ea
:1012dc00230100002c010000e90000009c0100002b
:1012ec00880100000901000009010000c100000094
:1012fc0081000000f9ff000061ff0000ecfe00001f
:10130c0010ff0000f3fe00000fff000010ff0000b4
:10131c00befe00001eff000074ff000080ff0000f6
:10132c00efff0000fcff000028000000a1000000ff
:10133c00280000005200000038000000b4ff00003c
:10134c00e5ff000007000000020000003000000074
:10135c008400000028000000daff00005f0000009d
:10136c004e000000030000000c000000f1ff000024
:10137c004800000071000000d2ff0000d7ff000001
:10138c00aeff000030ff0000b1ff0000cfff0000f7
:10139c0098ff0000b3ff0000f9ff00006d00000093
:1013ac005d000000270000000e0000008eff000012
:1013bc0066ff0000cfff0000ffff000031000000bf
:1013cc00750000006e0000003a000000f1ff000004
:1013dc0014000000750000005e00000054000000c6
:1013ec00d1000000cc000000a1000000ad00000006
:1013fc006200000005000000efff0000a2ff0000eb
:10140c001dff00006fff00004aff000035ff0000c9
:10141c006cff000056ff000094ff0000b4ff0000ba
:10142c0098ff0000c9ff0000cdff00001000000075
:10143c00760000002c000000510000001e0000008f
:10144c00cdff0000eeff0000f1ff000000000000e7
:10145c00100000005c00000009000000bdff00004f
:10146c004a0000003b0000000b00000038000000a8
:10147c0042000000bd000000030100003c00000021
:10148c0019000000c8ff000022ff000092ff0000be
:10149c00a2ff00002fff000034ff0000f5ff00004a
:1014ac004e0000000e000000ecff000085ff000065
:1014bc00e8fe0000f5fe00008bff0000c8ff0000f6
:1014cc00ffff00003b0000002e000000d0ff0000da
:1014dc003aff000076ff0000d6ff00009fff0000df
:1014ec00c6ff0000fbff00000f0000002f000000f3
:1014fc0044000000e6ff000067ff0000f6ff00005c
:10150c00090000006aff000012000000d6ff000076
:10151c0075ff000030000000840000007e00000019
:10152c0037000000c7ff000058ff000058ff000004
:10153c00a7ff00000500000044000000330000007d
:10154c00d6ff00003800000001000000aeff0000d4
:10155c003e000000c7ff00001c000000420000001d
:10156c00d2ff0000e1ff00009eff0000a6ff00007c
:10157c00a6ff00000e00000068000000e0ff000065
:10158c00b7ff0000d7ff0000cfff0000f5ff000001
:10159c001d000000600000008b00000056000000e1
:1015ac006200000043000000ecff00001d00000082
:1015bc00070000000b000000400000002b000000a2
:1015cc006700000039000000140000002d0000002e
:1015dc00e6ff0000e3ff0000ffff0000e4ff000057
:1015ec00050000003a000000230000001f0000006e
:1015fc002600000013000000390000006e000000ff
:10160c00720000005c000000ebff0000e8ff00002f
:10161c00e0ff0000cbff00002a0000000c000000df
:10162c001000000026000000fcff0000daff0000a4
:10163c000600000039000000730000005d0000008f
:10164c00c9ff0000d0ff0000aaff0000a5ff0000aa
:10165c00f6ff00000d00000019000000e9ff00007b
:10166c00c2ff000007000000220000000400000080
:10167c0015000000feff0000f9ff0000d7ff00007e
:10168c00c5ff0000daff0000efff0000f3ff0000d1
:10169c00e1ff0000f1ff0000e1ff0000daff0000b5
:1016ac00b0ff000088ff0000b7ff0000caff000079
:1016bc00070000002d0000001a00000020000000b0
:1016cc00d6ff0000c9ff0000e4ff0000deff0000b1
:1016dc00fdff00002d0000001a000000d8ff0000e4
:1016ec00d2ff0000c2ff0000bcff0000d0ff0000d2
:1016fc00f4ff00000c00000015000000e7ff0000e4
:10170c00c8ff0000e2ff0000e6ff00002800000018
:10171c002a000000fbff0000f8ff00000900000099
:10172c001f0000000700000006000000e3ff00009f
:10173c00cbff0000e0ff0000e0ff0000f7ff00001f
:10174c00eeff0000caff0000d0ff0000beff00004b
:10175c00cdff0000f4ff0000d5ff0000b7ff000034
:10176c00a4ff0000baff0000ccff0000b6ff000091
:10177c00bcff0000abff0000aaff00008bff0000c5
:10178c007aff000093ff0000a0ff0000a9ff0000fb
:10179c0090ff00008dff00008dff0000a5ff0000f2
:1017ac00b0ff0000a6ff0000b2ff0000b0ff000079
:1017bc00a3ff000082ff000075ff00007cff00000b
:1017cc0095ff0000bfff0000daff0000daff000009
:1017dc00b3ff0000bdff0000b6ff0000b7ff000024
:1017ec00f0ff0000f1ff0000f1ff0000e5ff00003a
:1017fc00d2ff0000ddff0000edff0000fbff00004a
:10180c00b8ff000078fe0000c2fd00005afd000089
:10181c0063fd0000c8fe00004cff00007cff0000d0
:10182c0065ff000080ff0000cb000000df0000001f
:10183c00670000005afe000030fc00006efe000045
:10184c007e0000004e020000930200002101000007
:10185c0097020000c2020000c20300005404000002
:10186c004102000060010000b5ff00001000000004
:10187c00f5000000bf000000e000000003000000c5
:10188c00940000006a000000fdfe000030fe000025
:10189c00aafc0000f0fc000054fe0000c1fe000099
:1018ac004aff0000bcfd000054fd00006cfc000071
:1018bc00cafa000054fe0000c900000061020000da
:1018cc000e02000047000000b7020000dd0300001c
:1018dc008905000042060000cf030000c002000092
:1018ec00ae0000000c000000a0ff000056fe00003f
:1018fc00f1fe000037fe00002afe0000bdfe0000d5
:10190c009bfd000060fd0000c6fc00008ffc000089
:10191c00c1fc000061fc0000e1fc0000f0fc0000d8
:10192c0005fb0000cbfb000070000000230300004f
:10193c0013040000b4010000ed000000540200008c
:10194c0090020000460500000f050000790300001e
:10195c0039020000700000007600000095ff0000c6
:10196c00cdfe00002ffe00000bfd000035fd000039
:10197c00a0fd00007ffc000083fb00006cfa00005f
:10198c0008fa00006df9000064f70000ecf90000a3
:10199c0070fe0000b70100007a0300006a0200002c
:1019ac005b0300009304000059050000e1060000f1
:1019bc001505000008030000840100004a00000027
:1019cc00b6ff000081fe000080fd0000b9fc0000a5
:1019dc0068fc000011fd00000afd000036fb000051
:1019ec0082f9000012f900000efa000001f8000064
:1019fc0067f90000a9ff0000600300002b05000040
:101a0c00a40300006a030000d00300001d030000c3
:101a1c002a0500006d04000023020000fd000000f8
:101a2c00f9ff00002b00000065fe000070fc0000b8
:101a3c00b3fb00001ffa000080fa0000fefb000060
:101a4c00a2fc000074fc000043fa0000c3f6000086
:101a5c001bf80000040000001c05000040050000fd
:101a6c003802000047010000370300003204000078
:101a7c00c70600004906000044020000afff00004a
:101a8c00e9ff00007d00000031fd00007ff900003f
:101a9c004ff8000064f80000c9fa00000afd0000cd
:101aac003efc0000b5f6000050f3000042fa0000c6
:101abc00f90100003a060000a40500002b03000009
:101acc006b040000aa050000cf0800007508000098
:101adc00f302000005ff000080fc0000ebfb00009f
:101aec006cfc0000cefb000030f900004ff700004a
:101afc006ef900005afd0000e3fa00001ef600002b
:101b0c0052f9000079ff000077030000590500002e
:101b1c00280600008a0600006d0500008206000001
:101b2c00400700003103000054ff000095fc00004a
:101b3c007ffa0000d2f8000052f8000010f9000003
:101b4c0097fa00006cfb00008ef800005dfa0000b4
:101b5c005a0100006c05000048060000e704000074
:101b6c00240600002d070000010500000f040000f2
:101b7c00ef000000e7fd000033fc0000def9000080
:101b8c0033f8000008f600003bf600002cf60000cd
